:020000040800F2
:1000000000000120F53F0008892700088B27000821
:100010008D2700088F2700089127000800000000A6
:10002000000000000000000000000000932700080E
:10003000952700080000000097270008992700086E
:1000400045400008454000089D270008454000083D
:100050004540000845400008A9270008AF270008D0
:100060004540000845400008E127000845400008D9
:10007000B5270008B7270008B9270008C5270008DA
:10008000D1270008DD27000845400008454000084A
:100090000000000045400008E32700084540000834
:1000A000454000084540000845400008454000081C
:1000B000454000084540000845400008454000080C
:1000C00045400008454000084540000845400008FC
:1000D00045400008ED27000845400008454000085D
:1000E00045400008E9270008F927000845400008B6
:1000F00045400008000000000000000045400008E6
:100100004540000845400008052800084540000813
:1001100045400008454000084540000845400008AB
:10012000454000084540000845400008454000089B
:080130004540000845400008AD
:1001380010B5054C237833B9044B13B10448AFF319
:1001480000800123237010BD4C0100200000000036
:10015800280E010808B5034B1BB103490348AFF348
:10016800008008BD0000000050010020280E010892
:1001780014214160704714207047406A704700009E
:10018800790100087F01000883010008990100082F
:1001980010B5044604F1100000F05CFCC4F8F80047
:1001A8000148C4F87C0110BD88010008F8B5E6B024
:1001B80004460D4616461F460A4906A800F0CAFE20
:1001C80070996F9A05910492009733466E996D9ACB
:1001D800039102922A466C990191214600F060F839
:1001E80067B0F0BD94010008F8B5E6B004460D46C6
:1001F80016461F46094906A800F0ACFE6F996E9A8C
:100208000491039200976D996C9A0291019233467A
:100218002A46214600F087F867B0F0BD940100082F
:1002280038B500281CBF01680029184A23D1184B8B
:100238001C684FF6F0710C404CF24025AC421FBFD1
:100248001B6819404CF27024A14212D1114D296843
:1002580079B911490B68C3F30B03B3F58A6F1FBF54
:100268000968C1F30B0140F28343994204BF01219D
:10027800117028B905E0094B994204BF012111709A
:100288004068BDE8324001F09FBE00BF6801002011
:1002980000ED00E0002004E00010005C000037489A
:1002A8002DE9F04104460D46216816464A681F4666
:1002B80090478046B8F5403F2ED122680A99936846
:1002C800204698478046B8F5403F25D12368089ACC
:1002D8000799D3F80CC02046E0478046B8F5403F60
:1002E8001AD12368069A39461F692046B8478046BE
:1002F800B8F5403F10D1236829465D69324620464B
:10030800A8478046B8F5403F06D123680B9A09995B
:100318009D692046A847804621680A68204690477C
:100328004046BDE8F0812DE9F04104460D462168BC
:1003380016464A681F4690478046B8F5403F2ED17A
:1003480022680A999368204698478046B8F5403F46
:1003580025D12368089A0799D3F80CC02046E047AE
:100368008046B8F5403F1AD12368069A39461F6976
:100378002046B8478046B8F5403F10D12368294643
:100388005D6932462046A8478046B8F5403F06D109
:1003980023680999DD6900222046A847804621681C
:1003A8000A68204690474046BDE8F0814FF4403047
:1003B80070470000F0B50C4685B0114600281A4673
:1003C8001CBF0568002D0B4B11D082B104B971B95F
:1003D8000D9860B10F9E0E9F0A9B0290049603979A
:1003E8000B980C9E009001962046A8470346184695
:1003F80005B0F0BD020003002DE9F04F0646D0B06D
:100408000868F56DD6F860E0726EB76EF36E00BAE4
:1004180000906C46486800BA60600DF14008886832
:1004280000BAA060C86800BAE060086900BA206134
:10043800486900BA6061886900BAA061C86900BAF1
:10044800E061086A00BA2062486A00BA6062886A95
:1004580000BAA062C86A00BAE062086B00BA2063FA
:10046800486B00BA6063886B00BAA063C86B00BAB7
:10047800E063402058F80C1C58F820CC58F838ACE9
:100488008CEA010158F840CC8AEA01018CEA01099A
:100498004FEAF979401E48F8049BEBD187EA02003D
:1004A80000EA0E00784010EBF5610098DFF824C4EC
:1004B80041186144C81882EABE032B404FEAF06134
:1004C80053405918636859186144CF194FEAB50366
:1004D80083EABE01014081EABE0111EBF765A1681C
:1004E8004D196544A91883EAB0023A404FEAF1650C
:1004F8005A405519E26855194FEAB70282EAB0071F
:1005080065440F4005EBBE0E97EAB00717EBFE6592
:1005180027697D194FEAB10782EA0701654401EAB4
:100528000E01EB18514011EBF36561694D194FEA63
:10053800BE0187EA010E65440EEA030E15EBB00012
:100548008EEA070E0EEBF065D4F818E075446544A2
:10055800AA1881EAB30505404FEAF26E4D40AE4451
:10056800E569AE44E64477444FEAB00080EAB30E4A
:100578000EEA020E8EEAB30E0EEBF765D4F820E011
:1005880075446544691880EAB2053D404FEAF16E4A
:100598004540AE44656AAE44E6440EEBB3034FEA09
:1005A800B70787EAB20E0EEA010E8EEAB20E0EEB1C
:1005B800F365D4F828E075446544281887EAB1053E
:1005C8001D404FEAF06E7D40AE44E56AAE44E64415
:1005D8000EEBB2024FEAB30383EAB10E0EEA000E45
:1005E8008EEAB10E0EEBF265D4F830E0754465443E
:1005F800EF1983EAB00515404FEAF76E5D40AE4447
:10060800656BAE44E6440EEBB1014FEAB20282EAF2
:10061800B00E0EEA070E8EEAB00E0EEBF165D4F8B6
:1006280038E075446544EB1882EAB7050D404FEA97
:10063800F36E5540AE44E56BAE44E6440EEBB000B5
:100648004FEAB10181EAB70E0EEA030E8EEAB70E41
:100658000EEBF065D4F840E07544654481EAB30ECA
:10066800AA180EEA000E4FEAF2658EEA010E7544EA
:10067800DDF844E04FEAB000754480EAB30E654403
:100688000EEA020E15EBB7078EEAB30E0EEBF7650E
:10069800DDF848E04FEAB202754480EA020E65448C
:1006A8000EEA070E69188EEA000E0EEBF165DDF80A
:1006B8004CE07544654405EBB3034FEAB70E1427C5
:1006C8000DF1500CDFF810528EEA010B82EA0B0B89
:1006D8000BEBF36A5CF804BBDA44AA44504483EA9F
:1006E800B10B4FEAF06A8EEA0B0BDA445CF804BBF4
:1006F800DA44AA44524480EAB30B4FEAF26A8BEA1E
:10070800B10BDA445CF804BBDA444FEAB000AA44FF
:1007180080EA020BD6448BEAB30B0BEBFE6A5CF85B
:1007280004BBDA444FEAB202AA4482EA0E0B0AEB8F
:10073800B10180EA0B0B0BEBF16A5CF804BBDA44FD
:100748007F1DAA44282F0AEBB3034FEABE0EBBD382
:100758003C2F61D3502F4DD204EB870CC7F15407BF
:100768005E4CA7FB04A504465D4FA8088EEA010A63
:1007780082EA0A0A5CF804BB0AEBF3655D447D195A
:100788002C1983EAB10A4FEAF4658EEA0A0A55443D
:100798005CF804AB5CF804BB55447D19AA1884EADC
:1007A800B30A4FEAF2658AEAB10A55445D444FEA52
:1007B800B4047D1984EA020AAE448AEAB30A0AEB51
:1007C800FE655CF804AB55444FEAB2027D1982EA33
:1007D8000E0A15EBB10184EA0A0A5CF804BB0AEBBD
:1007E800F1655D447D1915EBB303401E4FEABE0E5B
:1007F800BCD12046F46D1B19F365336EC9183166F8
:10080800716E71447166B36ED218B266F16E40189B
:10081800F06650B0BDE8F08F4EEA010B0EEA010A0F
:100828000BEA020B4BEA0A0A0AEBF36554F827A015
:10083800DFF8B0C0554443EAB10B654403EAB10A96
:100848000BEA0E0B28184BEA0A0A7F1C0AEBF06524
:1008580054F827A0554440EAB30B654400EAB30AAC
:100868000BEAB10BAA184BEA0A0A7F1C0AEBF265DD
:1008780054F827A055444FEAB00040EA020B6544FB
:1008880000EA020A0BEAB30BAE444BEA0A0A7F1CE1
:100898000AEBFE6554F827A055444FEAB20242EA33
:1008A8000E0B654402EA0E0A0BEA000B15EBB101C8
:1008B8004BEA0A0A7F1C0AEBF16554F827A0554455
:1008C8007F1C65443C2F05EBB3034FEABE0EA3D350
:1008D80040E700BF9979825AA1EBD96ECDCCCCCC38
:1008E800D6C162CADCBC1B8F00B581B00168074A5B
:1008F800914200D110B9064801B000BD7C2110F02A
:10090800F7F94FF4003001B000BD00BFFC09000842
:10091800030002002DE9F0410B4A92E8F85188B033
:10092800694681E8F8510268084B9A4200D118B923
:10093800074808B0BDE8F0811422083000F04FFBEA
:1009480008B0BDE8F08100BFDC090008FC09000818
:1009580003000200152904D20268044B9A4200D110
:1009680008B903487047083000F048BBFC09000884
:100978000300020010B481B013460268074CA2427B
:1009880000D118B901B010BC0548704701B000F19A
:10099800240210BC083000F035BB00BFFC09000879
:1009A8000300020010B481B013460268074CA2424B
:1009B80000D118B901B010BC054870470A4601B00B
:1009C80000F1240110BC083000F070BBFC090008DD
:1009D800030002000123456789ABCDEFFEDCBA981E
:1009E80076543210F0E1D2C300000000000000008D
:1009F80000000000F10800081D0900085D09000852
:100A08007D090008AD09000801040008790F0008F5
:100A1800C50F0008810F0008F0B5A3B004460B48C5
:100A280002900D4616461F46094B0822402104A88D
:100A380000F0D1FA28980190009733462A462146BB
:100A480002A800F01BF823B0F0BD00BFFC090008A5
:100A5800100A000810B5040008BF002408D0054893
:100A6800054B20600822402104F1080000F0B3FA89
:100A7800204610BDFC090008100A00082DE9F041C5
:100A880004460E46216817464A681D469047804628
:100A9800B8F5003F19D1226806999368204698470F
:100AA8008046B8F5003F10D123683146DE683A46E3
:100AB8002046B0478046B8F5003F06D12368079A1C
:100AC80029461D692046A847804621680A682046AD
:100AD80090474046BDE8F08110B500F033FA4FF476
:100AE800403400280EBF034C4FF4C07110F000F9D9
:100AF800204610BD0200030010B5044600F022FA9B
:100B080008B9054810BD0021A160D0F87C21116802
:100B180088474FF4403010BD0200030070B504460A
:100B28000D4600F00FFA064E40B1D0F87C0141683E
:100B38008847A84224BF65604FF44036304670BDF0
:100B4800020003002DE9FF4715000C4600D02CB128
:100B5800064600F0F7F95FEA000801D16448C3E0EF
:100B6800D8F8F80001684A689047B0F5003F17D1F7
:100B7800D8F87C118A68404690478146B9F1810FC0
:100B880080F09E80A94508F1FC0A17D2D8F8F80031
:100B98000368D3F80CC02A462146E047B0F5003F69
:100BA80040F08E80D8F8F8000368D3F810C06A4681
:100BB8005146E047B0F5003F76D10AE0002004E056
:100BC800215C0AF800100098401C00900098A84288
:100BD800F6D34FF0000C4749474A484B01AC009800
:100BE800844558D2D3E9007001ADC5E9007010788A
:100BF80000281ABF042086464FF0000E085854F803
:100C08000E5028443E4D05600127D0F800E087606B
:100C1800019D4F681AF80C007D408EEA050585F0A5
:100C2800040E65680F687D4085F0FC05754485F005
:100C3800A30568400AF80C000CF1010CCFE7D3E9D2
:100C4800004501A8C0E9004510782E4D002814BFC2
:100C58004FF0040E4FF0000E01A8744651F80EE054
:100C68000459A6440127CEF80050DEF80040CEF81B
:100C780008704D68019F40687D406C400D68684071
:100C880084F0040480F0FC00041984F057040AF886
:100C98000C400CF1010CCC45D1D3D8F8F800016810
:100CA8004A689047B0F5003F0AD1D8F8F8000368C1
:100CB800D3F80C804A465146C047B0F5003F01D0F2
:100CC800114811E0002006E05AF8201081F06A313E
:100CD8004AF82010401CB0EB990FF5D3B06840F0EB
:100CE8000100B0604FF4403004B0BDE8F08700BFA9
:100CF80002000300C00E010868010020240F00084C
:100D0800ADBE4ED70DBE75A10100030038B50C4627
:100D1800017A1546CA0702D500F014F908B908483F
:100D280032BDD0F8F80003682146DC682A46A0479F
:100D3800B0F5003F01D0034832BD4FF4403032BD1A
:100D480002000300010003002DE9F84191B00546B7
:100D58000E461746402101A80FF0CAFF297AC80796
:100D680004D5284600F0EEF8040002D1DFF8A4808C
:100D78004BE0D4F8F800DFF8A0800368D3F810C07F
:100D88006A4601A9E047B0F5003F3ED1D4F8F80023
:100D980001684A689047B0F5003F36D1D4F87C1115
:100DA8008A6820469047D4F8F830024618461B68EF
:100DB800D3F80CC004F1FC01E047B0F5003F24D1A2
:100DC800D4F87C0141688847D4F8F83002461846C0
:100DD8001B68D3F80CC001A9E047B0F5003F14D157
:100DE800D4F8F8000268696893689847B0F5003F3E
:100DF8000BD1D4F8F80003681C693A463146A0477D
:100E0800B0F5003F08BF4FF44038404612B0BDE887
:100E1800F08100BF02000300010003002DE9F84142
:100E2800A5B0074688461646402115A80FF060FF72
:100E380000220492402105A80FF05AFF387AC10712
:100E48005ED5384600F07EF8050059D0D5F8F80090
:100E58002D4C0368D3F810C06A4605A9E047B0F5E1
:100E6800003F3CD1D5F8F80001684A689047B0F5D2
:100E7800003F34D1D5F87C118A6828469047D5F8C8
:100E8800F830024618461B68D3F80CC005F1FC017F
:100E9800E047B0F5003F22D1D5F87C01416888478A
:100EA800D5F8F830024618461B68D3F80CC005A9D7
:100EB800E047B0F5003F12D1D5F8F800026879682C
:100EC80093689847B0F5003F09D1D5F8F800036852
:100ED8001D6904AA15A9A847B0F5003F01D020460E
:100EE8000FE00A4B0A490B4A0396029101924046C9
:100EF8001C68049B009415AA796800F0E5F900E0E5
:100F0800054826B0BDE8F08101000300C80E0108BD
:100F1800936E030026C703000200030004B001011A
:100F280000170145E10A0008010B0008250B00081D
:100F3800B50300084D0B0008150D0008510D0008F9
:100F4800250E00080168024A914218BF0020704728
:100F58002C0F000810B5040008BF002404D0034873
:100F68002060204609688847204610BD2C0F0008DD
:100F780020225C300FF0BABEF0B58468A3080022C6
:100F880004F0030407E000F15C0555F8226035BA67
:100F980041F82250521C9A42F5D300220BE000F18E
:100FA8005C0502EB830755F82360D500C5F11805E9
:100FB800EE40CE55521CA242F1D3F0BD30B5C46804
:100FC80003690022E31AD5188C5C0544521C082AD0
:100FD8002C77F8D330BD0360C1600261704738B523
:100FE800044615460022626023685A68904700202C
:100FF8006061A061A5604FF4003032BD81604FF49C
:10100800003070472DE9F84304462079D4F80C8065
:10101800450748BF244845D466691D46A8F1010024
:1010280000EAD60306EBC506B6EBC50F666102D229
:10103800A669761CA6611746A66906EB5576A661D1
:101048000E46E918884225D2A8EB03094A463146DC
:10105800F8180FF04BFE2268136839460FE0424635
:1010680038460FF043FE23681A68394620469047F1
:1010780007E0311811F00300F1D122681368204607
:101088009847484600EB0809A9F10101A942F0D3A5
:10109800002300E000202A1A3118F8180FF026FE65
:1010A8004FF40030BDE8F283040002002DE9FC4F44
:1010B800024685B0D0681369DFF86CC1DFF86C812F
:1010C800A0EB030A506840F004005060002703A812
:1010D80002900DF10C0ED8E9003403A8544DC0E974
:1010E80000342878534D00280CBF00230423994668
:1010F8005CF803305EF80940234401261D601C6833
:101108009E60DCF80430039DDCF80090DEF8046093
:101118005D406540484C654089EA0606474C664094
:101128007519474C6540D8E9006B03AC0028C4E941
:10113800006B0EBF002404200424029E5CF800000B
:10114800345920183F4C04600126046886600398CF
:10115800029E43406340384C7068634089EA00004F
:10116800364C6040034438484340280018BF0120EB
:101178005B1E9B41042F2CBFC0B2D80F02F1140391
:1011880053F8200007F00303C3F10303DB00D84042
:101198000DF807007F1C082F9DD315460C466A6979
:1011A800AB69E868D20842EA4372401E00EA0207C7
:1011B800002302409B420AD8524508D28020E055BD
:1011C8007F1C574516D2AAEB0701E01910E08020D2
:1011D800E05500E0E355E8687F1C8742FAD32A68A7
:1011E800136828469847BAF1000F03D051462046A5
:1011F8000FF07EFD2A68069E059F9368694628467B
:1012080098472A68D2F8009021462846C8472B6894
:10121800DA683946284690470EB1A86830604FF41E
:10122800003007B0BDE8F08FC00E01085412000866
:10123800680100205FC5109304850012FC68017ADC
:10124800C0F524FF24AF33D426AF698B04B0010165
:1012580000170145F8B501240094002300240DE08F
:10126800009D065D0F5D7E40F643761CF60F86F006
:10127800010635400095641C009DEB189442EFD39D
:101288001846F2BDF8B5002301240094002A11E0A5
:10129800009C85188F1815F8016C17F8015C6E40D2
:1012A800F643761CF60F86F0010634400094009C45
:1012B800E318521EECD11846F2BD00005D1200087A
:1012C8008D120008010000002DE9F84F1D46DDF8D9
:1012D80028900B9F0D9C4FF0FF3300930E469246CB
:1012E800D9F800B0804632465146D847834664B3A1
:1012F800D9F8043032465146404698476FEA0B0207
:10130800521C42EA0B0200996FEAD2735B1C194027
:10131800C2430091521C024300996FEAD2735B1CCE
:101328001940009186F05531484087EA000181F064
:101338005531216080F05531C943491C0843009A52
:101348006FEAD070401C82430092D9F80800012847
:1013580009D17540E943491C0D4300986FEAD572DD
:10136800521C90430AE0F11C85EA9102D243521CB8
:10137800154300986FEAD5735B1C984386F0AA362C
:10138800009086EA0B0686F0AA33F243DB430C98FA
:10139800C2F3C0725B1C42EAD3720099D243521C5A
:1013A80091430091774000998843009987F0AA37C4
:1013B8000F403843BDE8F28F034613F8012B002A8B
:1013C800FBD1181A0138704781F0004102E000BFD4
:1013D80083F0004330B54FEA41044FEA430594EAED
:1013E800050F08BF90EA020F1FBF54EA000C55EA28
:1013F800020C7FEA645C7FEA655C00F0E2804FEAF9
:101408005454D4EB5555B8BF6D420CDD2C4480EADA
:10141800020281EA030382EA000083EA010180EA0A
:10142800020281EA0303362D88BF30BD11F0004F58
:101438004FEA01314FF4801C4CEA113102D040428E
:1014480061EB410113F0004F4FEA03334CEA1333C9
:1014580002D0524263EB430394EA050F00F0A780E1
:10146800A4F10104D5F1200E0DDB02FA0EFC22FADC
:1014780005F2801841F1000103FA0EF2801843FAD0
:1014880005F359410EE0A5F120050EF1200E012AC1
:1014980003FA0EFC28BF4CF0020C43FA05F3C018FF
:1014A80051EBE37101F0004507D54FF0000EDCF178
:1014B800000C7EEB00006EEB0101B1F5801F1BD321
:1014C800B1F5001F0CD349085FEA30004FEA3C0C25
:1014D80004F101044FEA445212F5800F80F09A801B
:1014E800BCF1004F08BF5FEA500C50F1000041EB1F
:1014F800045141EA050130BD5FEA4C0C404141EB23
:101508000101013C28BFB1F5801FE9D291F0000F1D
:1015180004BF01460020B1FA81F308BF2033A3F1CC
:101528000B03B3F120020CDA0C3208DD02F1140CC3
:10153800C2F10C0201FA0CF021FA02F10CE002F1FE
:101548001402D8BFC2F1200C01FA02F120FA0CFCF7
:10155800DCBF41EA0C019040E41AA2BF01EB045140
:10156800294330BD6FEA04041F3C1CDA0C340EDC3E
:1015780004F11404C4F1200220FA04F001FA02F381
:1015880040EA030021FA04F345EA030130BDC4F13F
:101598000C04C4F1200220FA02F001FA04F340EA34
:1015A8000300294630BD21FA04F0294630BD94F0E5
:1015B800000F83F4801306BF81F480110134013DCC
:1015C8004EE77FEA645C18BF7FEA655C29D094EA3D
:1015D800050F08BF90EA020F05D054EA000C04BFBB
:1015E8001946104630BD91EA030F1EBF00210020A6
:1015F80030BD5FEA545C05D14000494128BF41F045
:10160800004130BD14F580043CBF01F5801130BDA8
:1016180001F0004545F0FE4141F470014FF0000033
:1016280030BD7FEA645C1ABF194610467FEA655CE4
:101638001CBF0B46024650EA013406BF52EA033586
:1016480091EA030F41F4002130BD00BF90F0000F74
:1016580004BF0021704730B54FF4806404F13204B0
:101668004FF000054FF0000150E700BF90F0000F69
:1016780004BF0021704730B54FF4806404F1320490
:1016880010F0004548BF40424FF000013EE700BF60
:1016980042004FEAE2014FEA31014FEA02701FBFF0
:1016A80012F07F4393F07F4F81F06051704732F022
:1016B8007F4208BF704793F07F4F04BF41F4002179
:1016C800704730B54FF4607401F0004521F00041D7
:1016D8001CE700BF50EA010208BF704730B54FF061
:1016E80000050AE050EA010208BF704730B511F062
:1016F800004502D5404261EB41014FF4806404F19A
:1017080032045FEA915C3FF4D8AE4FF003025FEA1F
:10171800DC0C18BF03325FEADC0C18BF033202EBA3
:10172800DC02C2F1200300FA03FC20FA02F001FAFD
:1017380003FE40EA0E0021FA02F11444BDE600BFA0
:101748004FF0FF3C06E000BF4FF0010C02E000BF85
:101758004FF0010C4DF804CD4FEA410C7FEA6C5C68
:101768004FEA430C18BF7FEA6C5C1BD001B050EA0B
:10177800410C0CBF52EA430C91EA030F02BF90EAF6
:10178800020F0020704710F1000F91EA030F58BFB5
:10179800994208BF90422CBFD8176FEAE37040F017
:1017A800010070474FEA410C7FEA6C5C02D150EAB5
:1017B800013C07D14FEA430C7FEA6C5CD6D152EA70
:1017C800033CD3D05DF8040B704700BF8446104635
:1017D80062468C461946634600E000BF01B5FFF734
:1017E800B7FF002848BF10F1000F01BD4DF808ED04
:1017F800FFF7F4FF0CBF012000205DF808FB00BFD5
:101808004DF808EDFFF7EAFF34BF012000205DF82E
:1018180008FB00BF4DF808EDFFF7E0FF94BF01207B
:1018280000205DF808FB00BF4DF808EDFFF7CEFF7C
:1018380094BF012000205DF808FB00BF4DF808EDBB
:10184800FFF7C4FF34BF012000205DF808FB00BF8C
:101858004FEA410212F5001215D211D56FF47873D0
:10186800B3EB625212D94FEAC12343F0004343EA73
:10187800505311F0004F23FA02F018BF404270474E
:101888004FF00000704750EA013005D111F00040D8
:1018980008BF6FF0004070474FF00000704700BF6E
:1018A80080F0004002E000BF81F0004142001FBF0D
:1018B8005FEA410392EA030F7FEA226C7FEA236C16
:1018C8006AD04FEA1262D2EB1363C1BFD21841400B
:1018D80048404140B8BF5B42192B88BF704710F0A1
:1018E800004F40F4000020F07F4018BF404211F044
:1018F800004F41F4000121F07F4118BF494292EAAC
:10190800030F3FD0A2F1010241FA03FC10EB0C00D7
:10191800C3F1200301FA03F100F0004302D5494264
:1019280060EB4000B0F5000F13D3B0F1807F06D311
:1019380040084FEA310102F10102FE2A51D2B1F109
:10194800004F40EBC25008BF20F0010040EA0300FE
:101958007047490040EB0000013A28BFB0F5000F7E
:10196800EDD2B0FA80FCACF1080CB2EB0C0200FA34
:101978000CF0AABF00EBC25052421843BCBFD04083
:101988001843704792F0000F81F4000106BF80F4FD
:1019980000000132013BB5E74FEA41037FEA226CC0
:1019A80018BF7FEA236C21D092EA030F04D092F08B
:1019B800000F08BF0846704790EA010F1CBF0020BF
:1019C800704712F07F4F04D1400028BF40F000401C
:1019D800704712F100723CBF00F50000704700F03C
:1019E800004343F0FE4040F4000070477FEA226263
:1019F80016BF08467FEA23630146420206BF5FEA34
:101A0800412390EA010F40F4800070474FF0000333
:101A180004E000BF10F0004348BF40425FEA000CFA
:101A280008BF704743F0964301464FF000001CE0A2
:101A380050EA010208BF70474FF000030AE000BFF8
:101A480050EA010208BF704711F0004302D5404236
:101A580061EB41015FEA010C02BF844601460020A8
:101A680043F0B64308BFA3F18053A3F50003BCFAC3
:101A78008CF2083AA3EBC25310DB01FA02FC634470
:101A880000FA02FCC2F12002BCF1004F20FA02F277
:101A980043EB020008BF20F00100704702F120026A
:101AA80001FA02FCC2F1200250EA4C0021FA02F2CB
:101AB80043EB020008BF20EADC7070474FEA40029F
:101AC800B2F1FE4F0FD34FF09E03B3EB12620DD964
:101AD8004FEA002343F0004310F0004F23FA02F0CE
:101AE80018BF404270474FF00000704712F1610F75
:101AF80001D1420205D110F0004008BF6FF000404C
:101B080070474FF00000704753B94AB9002908BF21
:101B180000281CBF4FF0FF314FF0FF3000F070B9C4
:101B2800ADF1080C6DE904CE00F006F8DDF804E02C
:101B3800DDE9022304B070472DE9F047089E0D4601
:101B480004460F46002B4AD18A42944665D9B2FA18
:101B580082F343B102FA03FCC3F120029F4020FA4A
:101B680002F217439C404FEA1C4E1FFA8CF5B7FB54
:101B7800FEF1220C0EFB117742EA074201FB05F049
:101B880090420AD91CEB020201F1FF3780F01B8159
:101B9800904240F2188102396244121AA4B2B2FB90
:101BA800FEF00EFB102244EA024400FB05F5A542B4
:101BB8000AD91CEB040400F1FF3280F00681A5422B
:101BC80040F203816444023840EA0140641B00216A
:101BD8001EB1DC400023C6E90043BDE8F0878B4214
:101BE80008D9002E00F0EC800021C6E9000508465F
:101BF800BDE8F087B3FA83F1002949D1AB4202D39B
:101C0800824200F2F780841A65EB0302012017462E
:101C1800002EE2D0C6E90047DFE702B9FFDEB2FADC
:101C280082F3002B40F08F808A1A4FEA1C471FFA74
:101C38008CFE0121B2FBF7F507FB1520220C42EAC6
:101C480000420EFB05F0904208D91CEB020205F198
:101C5800FF3802D2904200F2CA804546121AA4B256
:101C6800B2FBF7F007FB102244EA02440EFB00FE29
:101C7800A64508D91CEB040400F1FF3202D2A645A0
:101C880000F2BA801046A4EB0E0440EA05409FE734
:101C9800C1F120078B4022FA07FC4CEA030C05FA35
:101CA80001F420FA07F3FD40234300FA01F94FEA53
:101CB8001C401FFA8CFEB5FBF0F81C0C00FB1855F5
:101CC80044EA054408FB0EF5A54202FA01F20BD9D5
:101CD8001CEB040408F1FF3A80F08780A54240F22B
:101CE8008480A8F102086444641B9DB2B4FBF0F33D
:101CF80000FB134445EA044403FB0EFEA64508D93D
:101D08001CEB040403F1FF306BD2A64569D9023BF2
:101D1800644443EA0840A0FB0283A4EB0E049C42FF
:101D2800C6461D4655D352D056B1B9EB0E0364EBE7
:101D3800050404FA07F7CB40CC401F43C6E90074FA
:101D48000021BDE8F087C3F1200102FA03FC20FA64
:101D580001F225FA01F19D402A434FEA1C471FFA78
:101D68008CFEB1FBF7F007FB1015110C41EA054199
:101D780000FB0EF58D4204FA03F408D91CEB0101AF
:101D880000F1FF382FD28D422DD902386144491B0A
:101D980092B2B1FBF7F507FB151142EA014205FBC8
:101DA8000EF1914208D91CEB020205F1FF3816D258
:101DB800914214D9023D6244521A45EA004139E77A
:101DC8003146304609E73946E7E61046FCE6C145A4
:101DD800AAD2B8EB020E63EB0C050138A4E745461E
:101DE800EAE7034695E74046D1E7D0467CE7023D5F
:101DF800624433E708460BE76444023843E700BF10
:101E0800704700BF1348144A08B54FF00043C0E9B3
:101E180000230422002342610122C2614FF4805151
:101E280007220383C0E90233C0E90933C0E90C1271
:101E38000361837680F8203080F82C30826380F844
:101E48003C30C36402F052F918B1BDE8084000F014
:101E5800F3BB08BD6C010020002401400268084B58
:101E68009A4282B00AD14FF0B0431A6E42F400721F
:101E78001A661B6E03F400730193019B02B070474E
:101E8800002401400268054B9A4201BF4FF0B0425E
:101E9800136E23F400731366704700BF00240140DB
:101EA80030B585B000240546CDE901440394FFF719
:101EB800A9FF144802F0B2FC08B100F0BDFB1148BC
:101EC800039401A9CDE9015402F06EFA08B100F0BB
:101ED800B3FB0C4802F0CCFB08B100F0ADFB4FF0AF
:101EE800FF31084802F002FA064802F079FC05487A
:101EF80002F056FA0446034802F01CFC204605B0DE
:101F080030BD00BF6C010020014B024A1A607047C7
:101F18006C0100200024014008B50948FFF7C0FF04
:101F280068B1084BB3F8AA304FF6FF72934216BF58
:101F380040F6E442044B5343B3FBF0F398B208BDB8
:101F4800002000B40075FF1FD8084C0013B500230B
:101F5800ADF80630FFF7E0FF04461948FFF7A0FF89
:101F6800184BB3F8C820B3F8A8108A4204FB00F055
:101F780018D040F6E443B0FBF3F364205B1A434304
:101F8800521A93FBF2F31E331BB2ADF80630BDF8BC
:101F980006305BB21B02ADF80630BDF8060000B291
:101FA80002B010BD4FF47A7240F6FF73B0FBF3F342
:101FB8005343A3F53923A3F50C6340F6C412E0E7B5
:101FC800001000B00075FF1F4FF0B04382B09A6A4E
:101FD80022F480529A629A6C42F480529A649B6C02
:101FE80003F480530193019B002002B070474FF027
:101FF800B04382B09A6C02439A649B6C034001938D
:10200800019B02B0704708B50420FFF7F0FF0120DC
:10201800FFF7EDFF0220FFF7EAFF002211460B2031
:1020280002F09AFC0B2002F0C9FC002211460C2099
:1020380002F092FC0C2002F0C1FC002211460D2097
:1020480002F08AFC0D2002F0B9FC002211460E2095
:1020580002F082FC0E2002F0B1FC002211460F2093
:1020680002F07AFC0F2002F0A9FC00221146102091
:1020780002F072FC102002F0A1FC0022114611208F
:1020880002F06AFC112002F099FC00223620114669
:1020980002F062FCBDE80840362002F08FBC000068
:1020A80008B502F0D3FE10B16FF0040008BD064B6E
:1020B8009A6942F040429A614CF2FA321A6102F08F
:1020C800D7FE0028F2D0EFE700400058F0B585B001
:1020D80000230C4600930646A8B3FFF7E1FF054628
:1020E80070BB02F0B3FE88BB1A481B4A0223019357
:1020F800D0F8E01506F1784302EA8121B3FBF1F745
:1021080001FB1733DB0A0293D0F8E00504F17841AC
:102118000139314402EA8022B1FBF2F002FB1011CE
:10212800C3EBD1230133694601A8039302F020FFD2
:1021380020B102280CBF01256FF0010502F098FEBE
:10214800284605B0F0BD6FF00505F9E76FF0040506
:10215800F6E700BF0070FF1F00FCFF03014B18608B
:1021680000207047D00100202DE9F04F89B0B0F170
:10217800006F06460F460092C0F0C580DFF89881D0
:10218800664DD8F8E03505EA832303F10063013B87
:10219800984200F2B880002800F0B880002900F0CA
:1021A800B58040EA02035B0740F0B080FFF778FF94
:1021B8000446A0BB02F04AFE002840F0AA80D8F8E6
:1021C800E01506F1784205EA8121B2FBF1F301FB43
:1021D8001322009B03F17843013B3344B3FBF1F036
:1021E80001FB1033DB0A01334FEAD22AA3EBD222D8
:1021F800012A039388BFC6F30A050AF58038C6F199
:10220800080398BF009D069388BFC5F500654FEA8F
:10221800C828B346039B9A4505D302F029FE2046F9
:1022280009B0BDE8F08FA6F10803069A1A44954252
:1022380019D804950197CDF814B04FF00009059B03
:1022480009EB0301049B99453ED3009BAB442F4403
:102258005D1BB5F5006F28BF4FF400650AF1010A50
:1022680008F50068D6E753F8081F5A68B2F1FF3F2F
:1022780008BFB1F1FF3FD8D0294B186810B96FF0EB
:102288000504CAE7B8F1000F04D04FF400624146D4
:102298000EF0C8F8DFF88890D9F80030CBF30A00C0
:1022A80039461844AAB20EF0BDF84FF40061404612
:1022B800FFF70CFF08BBD9F8003001934FF4006317
:1022C800CDF814800493B8E7019B07914B4402931F
:1022D8000120D3E9002302F005FE88B90799019B84
:1022E800D1E9000259F80310029B5B689A4208BFC3
:1022F800884205D109F10809A1E76FF001048CE7CC
:102308006FF0030489E74FF0FF3488E76FF00504A6
:1023180085E76FF0040482E70070FF1F00FCFF03ED
:10232800D0010020B1F1006F70B511D30B4BD3F879
:10233800E0650B4B03EA862303F10063013B9942F6
:1023480006D840B139B192B20EF06CF8002070BDD9
:102358004FF0FF30FBE76FF00500F8E70070FF1F54
:1023680000FCFF03B0F1006F10B40DD3084BD3F895
:10237800E045084B03EA842303F10063013B9842DC
:1023880002D810BCFFF7A2BE4FF0FF3010BC704758
:102398000070FF1F00FCFF034FF0B04382B0DA6CFF
:1023A8000243DA64DB6C03400193019B02B070477F
:1023B80030B5012087B00024CDE90444FFF7ECFFD5
:1023C8000220FFF7E9FF0420FFF7E6FF01250222BC
:1023D8000DEB00014FF404134FF09040CDE90123B9
:1023E800039502F013FE4FF4441301A94FF09040F7
:1023F800CDE90235019502F009FE04230DEB030136
:102408000C48CDE90135CDE9034402F0FFFD224631
:102418002146062002F0A0FA062002F0CFFA224652
:102428002146072002F098FA072002F0C7FA07B001
:1024380030BD00BF0004004808B51248124A134BCB
:10244800C0E9002300230122C0E90232C0E90433B5
:10245800C0E90633036202F011FF08B100F0ECF89E
:102468000848002102F05BFF08B100F0E5F80548D4
:10247800002102F07AFF18B1BDE8084000F0DCB88E
:1024880008BD00BF94020020005800405D3E302087
:1024980070B596B005461422002103A80EF0FAFB89
:1024A8003822002108A80EF0F5FB2A68304B9A4222
:1024B8005BD18023089308A84FF440230E9303F0C0
:1024C800AFFC08B100F0B8F84FF0B0444FF4C0507A
:1024D800E36C43F00103E364E36C03F0010302934C
:1024E800029B12230026CDE903030323CDE90563EC
:1024F8004FF09040042303A9079302F087FDA36DD2
:10250800DFF870C043F48003A365A36D1A4C03F48D
:1025180080030193019B26620D23C4E900C3204672
:102528008023C4E90266C4E90436C4E9066602F0F9
:10253800A5FA08B100F080F8104AEC63A562104CC7
:102548000E23C4E900231021002380222046C4E979
:102558000213C4E90423C4E90633236202F08EFAA5
:1025680008B100F069F8AC63A56216B070BD00BF91
:102578000058004044000240D401002058000240A6
:102588003402002000B59BB04822002108A80EF0B4
:1025980081FB1822002102A80EF07CFB02F00AFF42
:1025A8004FF0B0420120D2F8903023F01803C2F85F
:1025B8009030D2F8003423F4C06343F40073C2F8B7
:1025C8000034D2F8003403F4C0630193019B242340
:1025D800089381230B930023CDE91003B02208A8A8
:1025E800CDE9122303F05EF808B172B6FEE74F2377
:1025F800CDE90230CDE90400CDE90600022102A8A8
:1026080003F0EAFA08B172B6FEE71BB05DF804FB06
:1026180008B501F019FDFFF7B5FFFFF7C9FEFFF791
:10262800F2FCFFF709FF00F0A7FD40F6B83000F014
:102638003FFA00F0A8FDFCE772B6FEE700B58DB0E2
:102648002C22002101A80EF025FB1748174B036028
:102658001F2383604FF080420023C0E90433C0E9A0
:10266800072383614FF48073436203F05FFD08B171
:10267800FFF7E2FF0C4803F085FE08B1FFF7DCFF27
:102688004FF0005300220793074808924FF48073D5
:1026980001A9029206920B9303F0A8FD08B1FFF777
:1026A800CBFF0DB05DF804FBE802002000280040D5
:1026B80010B5044690B03822002102A80EF0EAFABC
:1026C8002268194B9A422CD14FF48033029302A806
:1026D8004FF480730F9303F0A3FB08B1FFF7ACFF2F
:1026E8004FF0B0430220D3F8902042F40042C3F8E0
:1026F80090209A6D42F480629A659B6D002203F4E3
:10270800806311460193019B02F026F9022002F032
:1027180055F900222A20114602F01EF92A2002F05B
:102728004DF910B010BD00BF0028004070470000F0
:1027380008B501F09FFC044B0120C3F88800BDE8F0
:10274800084002F08FBE00BF0004005801F099BC99
:1027580008B501F096FC00F059FCFFF729FEFFF7D9
:1027680052FCBDE80840FFF767BE08B501F082FCDF
:10277800BDE808400121002002F024BE70477047E0
:10278800FEE7FEE7FEE7FEE7FEE7704770477047A3
:1027980070470000014803F01BBE00BFE80200209C
:1027A800012002F05FBD022002F05CBD7047704757
:1027B800014802F0DDBA00BFD4010020014802F050
:1027C800D7BA00BFC0030020014802F0D1BA00BF49
:1027D80060030020FFF7F2BF7047202002F042BDDF
:1027E80070470000014804F0B7B900BF200400207A
:1027F800014803F01FBC00BFE8020020014804F0B4
:1028080012B800BF4C0300202DE9F04389B0804680
:102818000020109E0790894615461F46FDF700FDCB
:10282800F0B9104CCDE90090CDE9020407AB0E4891
:102838000593142304933A46434629460068FDF756
:10284800B9FD2346324604F1140153F8044B42F80B
:10285800044B8B42F9D1079B337509B0BDE8F0836F
:102868000120FAE720030020BC0E01081FB50E4C1A
:1028780000233C2202A8CDE902336275237500F0DB
:10288800B9F8042303AA009412210848FFF7BCFFF3
:102898000749142220460EF0EDF9B0FA80F35B09DF
:1028A800637504B010BD00BF34030020E40E0108B6
:1028B800D2060020054808B50823036003F0CEFDC2
:1028C80018B1BDE80840FFF7B7BE08BD4C030020AB
:1028D8004FF0B04307B55A6E42F001025A665B6E7C
:1028E800002203F00103019311463220019B02F0FC
:1028F80033F8322003B05DF804EB02F05FB8000053
:102908000CB407B5054A05AB102101930EF094F8F5
:1029180003B05DF804EB02B0704700BFF60E010883
:1029280030B585B0044602A80D460DF0B1FEBDF9DC
:102938000C30064A00931021029B2046FFF7E0FF67
:102948002046FEF739FD288005B030BDF60E010897
:102958004FF0B04210B5936823F4004393600DF034
:102968001FFF0E4B01241C7000F0B6F80DF0E8FBB9
:102978000B480DF0FFFB0B4B4FF400421A61204649
:102988000DF0FEFBFFF7C0FA00F012F90DF0F4FCB1
:1029980021462046BDE810400DF00EBD580300202A
:1029A80029290008004000580DF01CBD08B5FFF7A4
:1029B800B3FA40F6B83398420CD8B0F5E16F0BD3B0
:1029C800FE23A0F5E16058434FF49663B0FBF3F0A3
:1029D800C0B208BDFE20FCE70020FAE77FB56846D4
:1029E80000F0CAF80198FFF769F800B207B05DF87F
:1029F80004FB0000194A38B5D2F88035591C044642
:102A080019D101F045FB054601F04EFB054401F0E4
:102A180045FB2B0EE3712B0CA3712B0A6371030E7C
:102A2800E370C0F30742C0F307232571C0B2A27058
:102A38006370207038BD190AC3718171190C1B0E9F
:102A480041710371D2F88435C370D2F88405C0F39C
:102A58000722C0F30743000EE9E700BF0070FF1F1D
:102A680038B5094BD3F8803503600133054609D1E1
:102A780001F00EFB044601F011FB444001F014FB89
:102A880044402C6038BD00BF0070FF1F01210220A8
:102A98000DF07CBC002102200DF078BC00207047AE
:102AA800024B187808B100F0BBB8704758030020F3
:102AB80082B00190019802B000F04EB94FF0B043D7
:102AC80082B0DA6C42F00202DA64DB6C03F00203D3
:102AD8000193019B02B070472DE9F043254C87B064
:102AE80001F0E8FA01F0EEFA01F0F4FA012300250A
:102AF80002934FF48059032301A9204604934FF40D
:102B0800005803950595FFF7D9FFFFF7D7FFFFF7A3
:102B1800D5FFFFF7D3FFCDF8049002F077FA01A9AB
:102B280020464FF40067CDF8048002F06FFA01A93F
:102B380020464FF40046019702F068FA01A92046A2
:102B4800019602F063FA2A464946204602F084FBC1
:102B58002A464146204602F07FFB2A46394620464F
:102B680002F07AFB2A463146204602F075FB07B090
:102B7800BDE8F0830004004810B50446FFF7E6F905
:102B8800074BA36040F30F20FEF744FF054B064AAE
:102B98002360064B6060C4E90323002010BD00BF1A
:102BA8000000484200007A440D093E00AB030500CE
:102BB80000207047014B1868704700BF5C03002075
:102BC8000320704708B501464FF47A72002380024B
:102BD800890DFEF799FF08BD4FF47A73A0FB030334
:102BE800800A40EA83507047034B98689A6890427D
:102BF800FBD1C043704700BF0028004008B5FFF76D
:102C0800F3FF014B186008BD5C03002008B5FFF70F
:102C1800EBFF024B1B68C01A08BD00BF5C03002015
:102C2800024B187808B1FFF7DFBF7047590300203F
:102C380010B5074B074C0122DA654FF48071204626
:102C480003F0BEF94FF0FF332363002010BD00BF2F
:102C580000280040E802002002460021014803F055
:102C6800C8BB00BFE802002002460121014803F06A
:102C7800C0BB00BFE802002010B58CB02C22002198
:102C8800044601A80EF006F8FFF7D2FF0C4B0D48DA
:102C98001B681C440023089306934FF00053E44339
:102CA800079301224FF4807301A902940B9303F058
:102CB8009DFA08B1FFF7C0FC00200CB010BD00BFA2
:102CC8005C030020E802002038B50546FFF78CFFBA
:102CD80002210446074803F093FBC4F309024FF4AA
:102CE8007A71A2FB0121920AA30A2A8043EA805042
:102CF80038BD00BFE80200200148002103F080BB76
:102D0800E80200200148012103F07ABBE802002014
:102D1800F8B50F4D2E78CEB90E4C4FF0FF3727631C
:102D2800FFF78CFCFFF784FF4FF48071204603F017
:102D380047F92046276303F007FB32462046022165
:102D480003F057FBFFF75AFF01232B700020F8BD53
:102D580059030020E8020020014610B54FF47A72AA
:102D680000238002890DFEF7CFFE0146FFF73CFFE6
:102D78000446FFF739FF031B8B4200D310BD00BF89
:102D8800F7E70DF015BE000010B5064C02212046ED
:102D980003F036FB0221421C2046BDE8104003F038
:102DA80028BB00BFE80200201648174A08B54FF4B0
:102DB800E133C0E9002300230C22C0E90233C0E953
:102DC8000523C0E90733C0E90933036104F0A5FC12
:102DD80008B1FFF731FC0B48002104F01AFE08B1D6
:102DE800FFF72AFC0748002104F033FE08B1FFF77B
:102DF80023FC044804F0EDFD18B1BDE80840FFF7D6
:102E08001BBC08BD200400200044004070B596B0EB
:102E180005461422002103A80DF03CFF38220021AA
:102E280008A80DF037FF2A68334B9A4261D1022374
:102E3800089308A8314B0A9302F0F2FF08B1FFF794
:102E4800FBFB4FF0B0430C219A6D2D4C42F400323D
:102E58009A659A6D02F400320292029ADA6C42F094
:102E68000102DA64DB6C03F001030193019B022386
:102E78000026CDE903130323CDE905634FF0904005
:102E8800072303A9079302F0C1F81E4826621423FA
:102E9800C4E900031023C4E9023620468023C4E9AC
:102EA8000436C4E9066601F0E9FD08B1FFF7C4FB82
:102EB800154AEC67A562154C1323C4E90023204684
:102EC80000238022C4E90233C4E90423C4E9063399
:102ED800236201F0D3FD08B1FFF7AEFB2520C5F84A
:102EE800804000220221A56201F036FD252001F074
:102EF80065FD16B070BD00BF0044004004000C0022
:102F0800C0030020800002406C00024060030020E3
:102F180002680E4B9A4210B5044616D14FF0B042E3
:102F28000C21936D23F4003393654FF0904002F029
:102F380019F9E06F01F016FED4F8800001F012FED6
:102F4800BDE81040252001F047BD10BD00440040F9
:102F580008B50A460146024803F062FD002008BD94
:102F68002004002013B5114B114C18604FF40013C6
:102F7800009302AB13E90600204604F0CEFC236858
:102F8800DA69D103FCD4DA695202FCD59A68084898
:102F980042F480029A6004F006FD064904480122C2
:102FA80004F074FC002002B010BD00BFB40400207F
:102FB80020040020BC04002008B5074B1860FFF768
:102FC80022F8FFF7F1FE054AD2F8803043F000639B
:102FD800C2F88030002008BDB8040020000800585E
:102FE80008B54FF0B04308489A6B42F400329A6330
:102FF8009A6B22F400329A63FFF78AFF0F2001F0E0
:10300800EBFC002008BD00BF2004002008B50748DD
:1030180004F083FB08B1FFF70FFB054801F02EFD14
:1030280018B1BDE80840FFF707BB08BD2004002021
:10303800C00300200268044B9A4203D1034B0020CE
:103048001B681847704700BF00440040B8040020C0
:1030580002680B4B9A4210B504460FD1094B1B6806
:103068002BB1D0F8902012B9074801219847204683
:103078000549BDE81040012204F008BC10BD00BF9E
:1030880000440040B4040020BC04002010B50A4CE1
:1030980023780BB9E37C6BB1FFF7E8FB0038074BEB
:1030A80018BF0120400018701B78022B02BF0023B4
:1030B8002370E37410BD00BFD2060020C5040020B1
:1030C80038B5114C2378EBB9E37CDBB90F4D2B688D
:1030D800012B07D92B68042B04D80D4A04210120A1
:1030E80000F0F4F92B68042B0CD9FFF7BFFB00386C
:1030F800084B18BF0120400018701B78022B04BF32
:103108000023237038BD00BFD2060020C004002071
:10311800500F0108C504002070477047022808B501
:103128000ED801221021074802F096F83220FFF746
:10313800BFFCBDE8084003480022102102F08CB80B
:1031480008BD00BF000400487047000010B5012109
:1031580004464FF0904002F079F8054AB0FA80F33F
:103168005B0913701378A370024B01221A7010BD0B
:10317800C4040020D106002008B5FFF7E9FBBDE82C
:10318800084000F043BB4FF0FF300DF08FB9704797
:1031980070470000014BD870704700BF5C000020EA
:1031A800014B1874704700BF5C00002020B1037801
:1031B80013B102480DF0AABB704700BF08060020F3
:1031C80008B5022000210DF039F9BDE80840014892
:1031D8000DF09CBB20060020002101200DF02EB927
:1031E80010B5094C60B1206008480DF041FB21681A
:1031F80006480DF0C5FBBDE8104004480DF086BB3D
:1032080042F210732360EFE77400002020060020CC
:1032180010B5094C206023680BB9084B2360084897
:103228000DF026FB216806480DF0AAFBBDE810400A
:1032380003480DF06BBB00BF0C000020A086010006
:103248003806002038B504460D4607484FF400619B
:10325800FFF788F830B92A4621460348BDE83840C8
:10326800FEF782BF38BD00BF00F003080A460149D7
:10327800FFF758B800F0030838B50C480DF0F8FA15
:1032880005F04CF860B90A4C0A480125257004F08D
:10329800D7FE2078294604F029FC04480DF036FBB7
:1032A800BDE8384004480DF031BB00BF20060020BF
:1032B800000000205C000020F005002005F0CAB8DE
:1032C80030B585B0FFF772FB044604F005FD0546EE
:1032D80080B1002434480DF0CBFA344B32481968D9
:1032E800A14238BF21460DF04BFB2F480DF00EFBD5
:1032F80005B030BD01A8FFF729FF2D4A2D49042349
:10330800137053680878187053685D7053681821F3
:10331800997053680121D970516823B203EB4303B4
:1033280003EB4313FE24B3FBF4F30B71224B197820
:1033380011B31D70536860F07F0018700523137077
:103348001E491F4C0978012988BF00235370637AEE
:1033580033B104F0ADFC012802D120460DF088FA03
:10336800184B1348D978002204F0CCFCA8B9164BA6
:103378001870164B1870ACE7144B1B7813B9124B26
:103388001B7843B153680121597153689DF80610A1
:1033980099710723D4E70523D2E7063099D104F0C1
:1033A80081FC044696E700BF200600207400002038
:1033B80004000020B805002050060020C5040020A5
:1033C800BC0500205C000020D1060020E706002094
:1033D80008B5104B0122002102201A700DF02EF8BA
:1033E8000D480DF093FA0D4B1B788BB10C4B1A78E6
:1033F80072B9DB7C63B90B4B1A68042A9EBF1A6842
:1034080001321A600021BDE8084010200DF016B8FE
:1034180008BD00BF5006002038060020EC0500203B
:10342800D2060020C0040020044B1B78022B03D1D5
:10343800002108200DF002B8704700BF00000020EE
:1034480008B504F074FF80B904F032FC01280CD1EF
:10345800BFF34F8F0549064BCA6802F4E062134375
:10346800CB60BFF34F8F00BFFDE708BD00ED00E064
:103478000400FA0510B5044640B190F906302BB99E
:1034880003480DF0F5F9034BE2791A7010BD00BF3F
:10349800BC050020EC050020704770477047704756
:1034A8007047012808B5014602D002280AD008BD95
:1034B8004FF0904001F0CAFE00210220BDE808400C
:1034C8000CF0BCBF00210820F8E7000070B50546E5
:1034D8000C46164604F000FC0346002834D00024AD
:1034E8001A480DF0C5F91A4B18481968A14238BF97
:1034F80021460DF045FABDE8704014480DF006BAB3
:103508004A68F05CD0540133DAB29442F8D8114BCF
:103518000D701B78012B88BF00244C700E4C637A09
:1035280033B104F0C5FB012802D120460DF0A0F903
:103538000A4B0B48D978002204F0E4FB0630CED1C0
:1035480004F0B0FB0446CBE70549DDE72006002080
:1035580074000020C5040020BC0500205C00002089
:1035680004000020044B1B7823B9044A05210120DC
:10357800FFF7ACBF704700BFC5040020550F010816
:1035880010B5002490B03C22214601A800940DF00B
:1035980081FB2C4B2022DA7219788DF800105978AB
:1035A8008DF8011099788DF80210D9788DF80310EC
:1035B80019798DF8041059798DF8051099798DF8D5
:1035C8000610D9798DF80710197A8DF80810597AEC
:1035D8008DF80910997A8DF80A108DF80B2021467C
:1035E8000DF10B0258180131007B02F8010F1C295C
:1035F800F8D193F828208DF8282093F829208DF801
:10360800292093F82A208DF82A2093F82B208DF86A
:103618002B200DF12B0100229818013290F82C0074
:1036280001F8010F142AF7D107484FF40061FEF79B
:1036380099FE20B9044840226946FEF795FD10B06E
:1036480010BD00BF7800002000F80308014940229F
:103658000CF0E8BE00F8030870B52A4D28796B799C
:103668004D2BC0B233D1C0EB001080000A2838BF00
:103678000A204FF47A735843234BAC791860EB79DE
:103688004D2BE4B22BD1C4EB0414A40095F82C30D4
:103698001E4E63BB95F83F304BBB42F21070FFF7EC
:1036A8009FFD3068FFF7B4FD2B7A194A1949DBB240
:1036B80013706B7A184ADBB213700023EA1892F879
:1036C8002C20D2B2CA540133142BF7D170BD6B79B8
:1036D800482B0ABF4FF461636B795843C6E7EB790F
:1036E800482B0ABF4FF46163EB795C43CEE7FFF7E1
:1036F80077FD012C38BF01244FF47A735C433460A2
:10370800CFE700BF78000020740000200C000020E4
:10371800E6060020D2060020C504002010B590B0AF
:1037280000213C2201A800910DF0B4FA402234494E
:1037380068460CF077FE9DF800203AB99DF8010024
:10374800182803D19DF8021001290ED0FFF718FFA1
:103758002C48142200210CF06FFE4FF47A70FFF70A
:10376800A7F9FFF779FF10B010BD274B1A705870F2
:1037780099709DF80310D9709DF8041019719DF87F
:10378800051059719DF8061099719DF80710D971A7
:103798009DF8081019729DF8091059729DF80A10C1
:1037A80099729DF80B1001F03F01D972D87AD1B205
:1037B80088421BD89DF8282083F828209DF82920C6
:1037C80083F829209DF82A2083F82A209DF82B20A9
:1037D80083F82B200DF12B0100229818013211F8E3
:1037E800014F80F82C40142AF7D1BAE701F14000C4
:1037F8006844194410F8340C08730132D6E700BF46
:1038080000F80308D2060020780000201FB5002425
:1038180003A92046039404F06DFD03A9012004F0D8
:1038280069FD354B3548009422464FF4FA710CF087
:10383800C1FF334B3348009422464FF4FA710CF021
:10384800B9FF314B3148009401224FF4FA710CF062
:10385800B1FF2046FEF782FC08B1FEF7EDFE2C4BC7
:10386800009400224FF4FA612A480CF0A3FF2A4A78
:10387800002101200CF09EFE284A002102200CF0B5
:1038880099FE274A002104200CF094FE254A0021C5
:1038980008200CF08FFE00F02DFB2349234804F08C
:1038A800DFFC234804F0CCFB18480DF02FF8214B1F
:1038B8000021187804F01AF91F4900941F4B096871
:1038C8001F4800220CF076FF1D480DF01FF8FFF787
:1038D80025FF1C4A002110200CF06CFE1A4B1B48D7
:1038E80019681B4B009400220CF064FF17480DF078
:1038F8000DF804B010BD00BFA5340008080600206C
:10390800A7340008D4050020A1340008BC05002015
:1039180031340008F0050020417E0008C932000853
:10392800C5320008813200080000030110000020A1
:103938005C0000200000002074000020C93100084D
:1039480020060020C93000080C000020380600209E
:10395800D933000810B50024A2B07C22214603A860
:1039680002940DF097F953238DF808304FF48C73B7
:10397800ADF80A3001238DF80C30ADF80440FFF79C
:1039880015F8FE23B0FBF3F000EB400000EB40100D
:103998008DF80D0001A800F052FBA0B958238DF84E
:1039A8000E3007243022802108480DF073F9224692
:1039B80002A906480DF09FF9044A21460120FFF7A5
:1039C80085FD22B010BD0624ECE700BF510600209B
:1039D80070B50378592B90B0044640F0C081052992
:1039E80059D84378443B162B55D8DFE813F011011A
:1039F80054000101540009015400540054005400BB
:103A080073005400EC005400540054007701540033
:103A180054008F0054005400540017008578482D36
:103A280011D1A64A14210120FFF750FD41F2883038
:103A3800FFF73EF840F6B830FFF73AF810B0BDE8A7
:103A48007040FFF7FDBC532D0ED1302280219C48D9
:103A58000DF020F9FFF77EFF41F28830FFF728F8D4
:103A6800974A1521012066E0432D16D100246846A7
:103A78008DF8004004F05CFA914A4C231370182327
:103A880093709DF80030547001204133D070137149
:103A98000521FFF71BFD10B070BD442DFBD1884CEC
:103AA8002C228021201D0DF0F5F80023257063706D
:103AB80001251823A370E5702571FEF777FFFE2313
:103AC800B0FBF3F000EB400000EB401060712246C1
:103AD8000621C7E78378303BDBB2092BDBD879496D
:103AE800794A0B700B78DBB25372754A59231370FD
:103AF8004D2353700B783033937003210120FFF767
:103B0800E5FC10B0BDE87040FFF73ABD8578482D58
:103B180016D16B4A562313700023537018239370E1
:103B280003231371172353710B230120937112235D
:103B3800D070D371082110B0BDE87040FFF7C6BC43
:103B4800432DA8D15E4C00213C2201A800910DF024
:103B5800A1F86846FFF77AFD2422802104F10C00C1
:103B68000DF098F89DF8003063709DF80130A3704F
:103B78009DF80230E3709DF8033023719DF80430FE
:103B880063719DF80530A3719DF80630E3719DF8C7
:103B9800073023729DF80830257063729DF80B502A
:103BA8009DF80930A3729DF80A30E3722A4603A9EA
:103BB800257304F10D000DF09EF805F10D01224664
:103BC800C9B2012065E7807839280CD83038C0B2EE
:103BD800FFF7A2FA3A4A2378137063785370A378F0
:103BE800937003213EE710B0BDE87040FFF7BABC00
:103BF80080783928F7D83038C0B2FFF78EFAE9E76D
:103C080080783928EFD83038C0B2FFF787FAE1E773
:103C18008378303BDAB2092AE5D8C0783038C2B2A6
:103C2800092AE0D82179A1F14802D2B20B2ADAD8C0
:103C3800264D45FA02F2D207D5D40A224D2902FBB5
:103C4800030036D13C2358434FF47A735843204B32
:103C58001860204B1860FFF7C3FA194A23781370CD
:103C680063785370A3789370E378D37023791371D2
:103C780005210120FFF72AFC134B00221A70182295
:103C88005A7001229A70DA70A278303A02EB8201F7
:103C9800E278303A02EB4102D2B21A7122795A71B3
:103CA8000D4A1278D2B21A72064A1278D2B25A72F1
:103CB80027E74829C8D14FF46163C4E75B0F0108BF
:103CC80051060020C504002078000020DEF7FFFF21
:103CD800740000200C000020E60600208678A6F17B
:103CE8003003092B3FF67FAFC078A0F13003092BD2
:103CF8003FF679AF2179A1F14802D2B20B2A3FF6FB
:103D080072AF5A4B134113F001057FF46CAF584A58
:103D18005923137053235370D07011719670052175
:103D28000120FFF7D3FB534918230D704B70012373
:103D38008B70CB70A378303B03EB8302E378303B86
:103D480003EB4203DBB28B712379CB714A4B1B78AF
:103D5800DBB20B72494B1B78DBB24B72D1E6502BAE
:103D680048D102297FF697AE4378303B012B3FF6C6
:103D780092AE8378312B7FF48EAE0B2904D8FFF7EF
:103D8800F1FB00213A4A6DE63A4D0234002214F85C
:103D9800013FA918303B0132DBB20C2A0B73F6D174
:103DA800FFF7D2F9324B502218211A70997000226D
:103DB80001215A70D97003F8041FA9180132097B30
:103DC8000C2A01F1300103F8011FF6D100232B70F2
:103DD80018236B700123AB70EB70274B1B78DBB299
:103DE8002B72264B1B78DBB26B72EA72FFF7C8FBAB
:103DF8001121C7E7412B7FF44EAE4378432B7FF464
:103E08004AAE16297FF447AE1D4D421C002312F816
:103E1800011FE9540133142BF9D1FFF737F9194B76
:103E28005B7D012B19D113490023EA5CC8180133C3
:103E3800D2B2142B80F82C20F7D1104B00221A7024
:103E48001B78DBB24B72FFF79BFB094A631E1534E4
:103E5800A34206D1064A162104E6084B02221A702C
:103E6800F3E713F8011F02F8011BF1E7DEF7FFFF84
:103E78005106002078000020E6060020C504002036
:103E8800D20600203403002038B504460D4661B33D
:103E980016480CF03BFD2B783BB334B360682378AD
:103EA80018B3032B0CD0042B17D0022B1DD161782B
:103EB80001291AD00B0618D4BDE83840FFF788BD91
:103EC8006378012B11D10078012802D0022800D094
:103ED80058B9BDE8384003F0E1BF6378012B04D13D
:103EE8000378034A03F00103137038BDD40500209A
:103EF800B8050020034B0022C3E902220122C3E9CE
:103F080000227047E806002000487047E8060020B5
:103F18004FF0B04382B0DA6C0243DA64DB6C0340E2
:103F28000193019B02B070472DE9F04186B000244F
:103F38000220154D0594FFF7EBFF0420FFF7E8FF7B
:103F4800124F03944FF4807601230DEB0001CDE965
:103F580001632846032304934FF4005801F056F8F0
:103F680001A93846CDF8048001F050F822464146B0
:103F7800384601F071F928462246314601F06CF9BD
:103F8800204606B0BDE8F08100040048000800485B
:103F9800032810B50ED8012810D868B902460B4876
:103FA8004FF4807101F058F9002209484FF400518C
:103FB80001F052F9002010BD0122F0E70022034869
:103FC8004FF4807101F048F90122EEE7000400483F
:103FD8000008004802207047002070470120704701
:103FE80000280CBF0F201620704700000D4885469A
:103FF80000F029F80C480D490D4A002302E0D45876
:10400800C4500433C4188C42F9D30A4A0A4C00231A
:1040180001E013600432A242FBD30CF043FEFEF72A
:10402800F7FAFEE700000120000000204C01002004
:10403800541A01084C01002084240020FEE7AA231A
:10404800437000207047704710B5032000F072FCE1
:1040580001F018FB064B18600F20FEF71FFD044601
:1040680018B9FEF78CFB204610BD0124FBE700BF02
:10407800B80000204FF0E022136923F00203136117
:1040880070474FF0E022136943F002031361704751
:10409800014BD3F8900570470070FF1F014BD3F810
:1040A800940570470070FF1F014BD3F898057047BF
:1040B8000070FF1F024A536823F0010353607047E2
:1040C800002004E0024A536823F00203536070475B
:1040D800002004E0024A536823F004035360704749
:1040E800002004E08068C0F380007047F7B5002323
:1040F80001930446002800F0E980856D25B9FDF795
:10410800ADFEE56584F8545023689A68D00040F104
:10411800A1809A68D10000F1B480A26D42F010022B
:10412800A265E26D42F00102E26501251846FFF73B
:10413800D9FFA26D02F01002024340F0C980A26DBF
:10414800206922F4817242F00202A2659A68D207BD
:104158005DD4226BA67E94F82CC0003A18BF0122C9
:104168001703D4E902120A43217E42EA8132617EB2
:1041780042EAC13242EA4632002842EA4C02B4BF5F
:1041880020F000414FF400113A430A4394F82010FC
:10419800012903D1002E76D142F48032616A21B11F
:1041A800A66A01F4E07131430A43D968E66C21F448
:1041B800FE3121F4FF711143D96094F83C20616805
:1041C800012A01F0404C4CEA060609D1D4E910272F
:1041D8003A433243A66C324342EA0C0242F00106EB
:1041E8001F693E4A3A4032431A6121F00042B2F157
:1041F800804F0CD0B1F1004F09D0394ED6F80827BE
:1042080001F4701122F470120A43C6F808275A699B
:10421800666BA16B22F0070232435A615A6922F099
:10422800700242EA01125A61002835D19A6A62F096
:104238000F029A625B6903F007039E423CD1002398
:10424800E365A36D23F0030343F00103A365284648
:1042580003B0F0BD9A68234922F0104222F01702F9
:1042680042F080529A60204A1268B2FBF1F20132A1
:1042780052000192019A002A3FF44BAF019A013A89
:10428800F7E7002552E7A16D41F02001A165E16D36
:1042980041F00101E16581E7B0F5001FCAD19A6AD2
:1042A800E269013A92006FF00F0102F01C0201FA74
:1042B80002F2216E0A43BCE7A36D23F0120343F018
:1042C8001003A365E36D43F00103E3650125BEE731
:1042D800A36D43F01003A365F8E700BF02FCFF1FBE
:1042E80000200140400D0300B8000020F8B54569E2
:1042F800082D04460E460AD00368DB68D80705D5A2
:10430800A36D43F02003A3650120F8BD0425FEF743
:10431800C7FB074623681A682A4221D0A26D42F4D7
:104328000072A265DA6812F4406F14D1A27E92B9C5
:104338001A6812070FD51846FFF7D4FE28BB5A682B
:1043480022F00C025A60A26D22F4807222F001025F
:1043580042F00102A265207E00BB0C221A60D4E75D
:10436800711CD8D0FEF79CFBC01BB04201D8002EB0
:10437800D0D123681B682B40CCD1A26D84F854306F
:1043880042F00402A2650320BFE7A26D42F02002BA
:10439800A265E26D42F00102E265DCE70020B4E7C5
:1043A8000368186C70470000F7B50023019390F874
:1043B8005430012B044600F0C580056806690123C6
:1043C80080F854302846FFF78DFE002840F0B4806E
:1043D800D1E90020022826F0040300F08280B3F11E
:1043E800004FC2F3110E13D1AB6A43EA0E03AB625E
:1043F8008B68686903EA022323F07C4323F0FF03F8
:1044080020EA02210B43002A6B6126DB002055E0DD
:10441800236E00F01F074FF00F0C0CFA07FC6FEA31
:104428000C0623EA0C0CBEF1000F11D1C2F3846311
:10443800BB4043EA0C0323668008E36901309842D5
:10444800D6D8A86AC2F38363BB4006403343CEE79D
:1044580092FAA2F3B3FA83F3EAE73B493B48D1F86F
:104468000837824203F0E07519D11B02CED4D1F887
:10447800083723F0E0732B4343F40003C1F80837EF
:10448800334B1A68334BB2FBF3F20C2302FB0333B2
:104498000193019B002BB9D0019B013BF8E72E4803
:1044A800824210D113F08070B0D1D1F8083723F0D0
:1044B800E0732B4343F08073C1F80837002384F876
:1044C800543003B0F0BD254882429FD113F48000D8
:1044D8009CD1D1F8083723F0E0732B4343F48003D1
:1044E800EAE7B3F1004F01BFAB6AC2F311018B4396
:1044F800AB62002A8ADA154813498242D1F8083794
:1045080009D1D1F8082703F0A07322F0E072134311
:10451800C1F808377AE71048824204D1D1F8082751
:1045280003F44003F1E70D4882427FF46FAFD1F8FE
:10453800082703F0C073E8E7A26D42F02002A265E5
:104548001846BBE70220BCE700200140001000B07D
:10455800B8000020400D0300004000B8002000B45F
:10456800026838B504461046FFF7BCFD08B90020BC
:1045780038BD9368990707D4936823F0004323F064
:10458800170343F010039360FEF78AFA0546236881
:104598009B685B07EBD5FEF783FA401B0228F6D928
:1045A80023689B685A07F2D5A36D43F01003A365EF
:1045B800E36D43F00103E3650120D9E773B50023F8
:1045C800026801939368DD07044602D5002002B013
:1045D80070BD9168214B194209D0A36D43F01003B7
:1045E800A365E36D43F00103E3650120EFE79368FA
:1045F80023F0004323F0170343F001039360184BA3
:10460800D3F8083718021CD4637E012BDED0FEF7DE
:1046180047FA144E054622681368DB07D6D4936818
:10462800D9075FBF9368334043F001039360FEF7F7
:1046380037FA401B0228EED923681B68DA07EAD448
:10464800CBE7094B094A1B68B3FBF2F3013301932B
:10465800019B002BD8D0019B013BF8E71700008095
:1046680000200140E8FFFF7FB8000020400D030054
:1046780038B504460068FFF735FD054620BB94F8B9
:104688005430012B20D0012384F854302046FFF702
:1046980095FFB0B9A36D226823F4706323F001037A
:1046A80043F48073A3651C23E065136084F8540009
:1046B800936823F0004323F0170343F00403936047
:1046C80038BD84F85450FBE70220F9E7026838B592
:1046D800936891680446C80701D4002038BD99073B
:1046E800FBD4936803F00503012B19D1936823F0D9
:1046F800004323F0170343F002039360032313607E
:10470800FEF7CEF9054623689B68DB07E5D5FEF77B
:10471800C7F9401B0228F6D923689B68DA07F2D547
:10472800A36D43F01003A365E36D43F00103E36554
:104738000120D3E770B5044600284BD0836D43F0C1
:1047480002038365FFF70CFF054668B92046FFF7AB
:10475800BDFF054608B90123A3652268936823F0C5
:10476800104323F01703936023685A6822F4677292
:1047780022F003025A6040F29F321A60D968164A42
:104788000A40DA601A6922F040421A615A6922F036
:1047980007025A611A6A02F0F0221A625A6A02F093
:1047A800F0225A62DA6A02F0F022DA629A6A0B4A56
:1047B80000269E62D2F8083723F0FE73C2F8083745
:1047C8002046FDF75FFBE6652666A66584F854601B
:1047D800284670BD0125FBE700023E83002001400A
:1047E80010B590F85430012B044615D0012380F8F9
:1047F8005430FFF7B5FE58B92046FFF767FF38B9C0
:10480800A36D23F4807323F0010343F00103A36530
:10481800002384F8543010BD0220FCE7F7B50023CC
:10482800019390F85430012B04467FD0012380F87F
:104838005430FFF74BFF23689A6812F001020546CF
:1048480007D0A36D43F01003A365002384F8543008
:104858002DE0A16D364F21F4817141F00201A1656F
:10486800DE68D96826F4FF4626F07C0621F400416C
:10487800360421F00301360CD960082099683940C4
:1048880041F0004199609968002913DA01990131D2
:1048980001910199B1F52E3FF5D3A36D23F01203D1
:1048A80043F01003A365002384F8543001252846FB
:1048B80003B0F0BDD3F8B410013801F07F010A4409
:1048C800DCD199681A48014041F001019960D3F898
:1048D800B41021F07F0141EAD202C3F8B4209A68EB
:1048E800024042F002029A60FEF7DAF807462368AF
:1048F8009A68D20708D4DA683243DA60A36D23F0E5
:10490800030343F001039FE7FEF7CAF8C01B022820
:10491800EDD923689B68D907E9D5A36D43F0100347
:10492800A365E36D43F00103E365BFE70225BEE736
:10493800E8FFFF7F0749CA6822F4E0620302120415
:1049480003F4E063120C134343F0BF6343F40033F2
:10495800CB60704700ED00E0164B30B5DC68C4F35F
:104968000224C4F10703251D042B28BF0423062DA8
:104978004FF0FF358CBF033C002405FA03F321EA0E
:104988000303A54022EA0502A340002843EA0203E4
:10499800ACBF00F16040084A4FEA0313B8BF00F00B
:1049A8000F00DBB2AABF00F56140135480F8003352
:1049B80030BD00BF00ED00E014ED00E0002807DB8B
:1049C800044A4109012300F01F00834042F82130C6
:1049D800704700BF00E100E000280CDB43090649EE
:1049E80000F01F0020330122824041F82320BFF34A
:1049F8004F8FBFF36F8F704700E100E070B5D0E9CB
:104A080013456560446D14B1D0E916456560D0E979
:104A1800105404F01C060124B4406C600468636000
:104A28008368102B0BBFA260A160E160E26070BDDB
:104A38000268416CD3B210B5083B1424B3FBF4F3FD
:104A48000B4CA24288BF0B4A21F0030199BF01F128
:104A5800804202F50232521807338264064AC26461
:104A680003F01F03012202FA03F3036510BD00BF20
:104A7800070402401C0802408008024038B500289C
:104A88005ED002682F4B9A424FF014014CD82E4B3F
:104A98001344B3FBF1F32D499B00C0E91013022323
:104AA80080F825301368056923F4FF4323F0700369
:104AB8001360D0E9024323432B43456911682B4314
:104AC80085692B43C5692B43056A2B430B43136048
:104AD800FFF7AEFFB4F5804F04BF00234360426880
:104AE800816C02F07F030B60D0E91314013A032AAA
:104AF8004C6020D8164A174981651A44013B920038
:104B0800012103F0030301FA03F300214265C365A1
:104B18001160114A536400230122C36380F82430D2
:104B280080F82520184638BD0C4B1344B3FBF1F32D
:104B38000B499B00B1E70023C0E91533C365EAE7D9
:104B48000120F0E707040240F8FFFDBF0000024023
:104B58003F8200104009024000090240F8FBFDBFF7
:104B68000004024038B5002841D00268136823F0D9
:104B7800010313601F4B9A424FF0140130D81E4BAB
:104B88001344B3FBF1F31D499B00C0E91013012442
:104B980003F01C0304FA03F3002515604B60FFF7CC
:104BA80047FF836C41681D60D0E913325A604A1E82
:104BB800032A06D8124B0B449B0094401D60114BEE
:104BC8005C640023C363C0E91533C0E90B33C0E953
:104BD8000D33C36580F8253080F82430184638BD79
:104BE800094B1344B3FBF1F308499B00CDE70120BF
:104BF800F5E700BF07040240F8FFFDBF00000240D0
:104C08003F82001000090240F8FBFDBF000402408B
:104C180070B590F82450012D04463BD090F82560DB
:104C28000125AE4280F824504FF000062CD1022511
:104C380080F825500568C6632E6826F001062E60A8
:104C4800FFF7DCFE036BBBB12B6843F00E032B6050
:104C5800A36C1A68D20342BF1A6842F480721A60C1
:104C6800636D1BB11A6842F480721A602B6843F0B6
:104C780001032B60002070BD2B6823F004032B6018
:104C88002B6843F00A03E2E78023C36380F82460BB
:104C98002846F0E70220EEE7034640B190F82520C9
:104CA800022A06D00422C263002280F824200120B0
:104CB80070470268806C116821F00E01116001686C
:104CC80021F480710160116821F001011160D3E9BC
:104CD800100202F01C0101228A404260D3E913212C
:104CE80051605A6D32B1116821F480711160D3E9B5
:104CF800162151600122002083F8252083F8240022
:104D0800704710B590F82530022B03D00423C363F5
:104D1800012010BD03681A6822F00E021A601A6892
:104D280022F001021A60826C136823F48073136006
:104D3800D0E9101303F01C02012393404B60D0E923
:104D480013325A60436D33B11A6822F480721A60C4
:104D5800D0E916325A60012380F82530836B00248D
:104D680080F8244013B198472046D2E71846D0E788
:104D780070B4426C046C036826681D6802F01C025B
:104D88000421914031420FD015F0040F0CD01A685D
:104D980092065EBF1A6822F004021A60036B616013
:104DA800002B33D070BC184702219140314217D0F4
:104DB80015F0020F14D01A68940606D41A6822F067
:104DC8000A021A60012280F82520114A93428CBFFA
:104DD800104B114B5960002380F82430C36ADFE779
:104DE80008219140314211D029070FD5196821F0C7
:104DF8000E011960012303FA02F26260C36380F8AE
:104E08002530002380F82430436BC9E770BC704715
:104E18008000024000040240000002400A4A536930
:104E280043F4802330B55361EFF3108472B6002346
:104E3800CD58C5500433B3F5807FF9D11369DB032E
:104E4800FCD484F3108830BD00400058064B5A69E2
:104E5800002ABFBF054A9A6002F188329A60BABF39
:104E68005869C00F0020704700400058230167456B
:104E7800044B5A6942F000425A615869C043C00F56
:104E8800704700BF0040005870B50546FDF708FEA2
:104E9800124E04463369D90313D43369DA0744BF81
:104EA800012232614CF2FA32134011D10B4E3069B3
:104EB80010F480200BD0FDF7F3FD001BA842F6D3B9
:104EC80004E0FDF7EDFD001BA842E3D3032070BD0D
:104ED800024A1361024A01205360F8E70040005873
:104EE800F80600202DE9F041184D98462B78012B43
:104EF80006460C46174626D001232B704FF47A70CD
:104F080000236B60FFF7C0FFA0B9012E16D1104A2D
:104F1800536943F0010353612760BFF36F8FC4F8EF
:104F280004804FF47A70FFF7AFFF094A536923EA08
:104F38000603536100232B70BDE8F08139462046F3
:104F4800FFF76CFFEDE70220F6E700BFF806002048
:104F580000400058054A536923F47E7343EAC000B1
:104F680040F4803040F00200506170470040005823
:104F78002DE9F041234F3B78012B054688463FD069
:104F880001233B704FF47A7000237B60FFF77CFFAE
:104F9800044688B92B68042B13D11B4A536943F480
:104FA800803343F0040353614FF47A70FFF76CFFCA
:104FB8000446154B1A681B6800233B702046BDE861
:104FC800F0814FF0FF33C8F800306E68D5E9013240
:104FD8001344B3420AD93046FFF7BCFF4FF47A7046
:104FE800FFF752FF50B1C8F800600446064A5369FB
:104FF80023F47E7323F002035361DAE70136E5E711
:105008000224DBE7F8060020004000582DE9F04FA5
:10501800524C00234FF00F090A6832FA03F501D108
:10502800BDE8F08F012505FA03F818EA020200F03E
:105038008E804E68032706F003054FEA430E07FAF1
:105048000EFC6F1E012F6FEA0C0C32D8876807EA36
:105058000C0ACF6807FA0EF747EA0A07876047681D
:1050680027EA0808C6F300179F4047EA0807476081
:10507800C76807EA0C088F6807FA0EF747EA0807B7
:10508800022DC76017D14FEAD30800EB880803F058
:10509800070AD8F820704FEA8A0A09FA0AFB27EAB1
:1050A8000B0B0F6907FA0AF747EA0B07C8F82070D5
:1050B80001E0032DDCD1076805FA0EF507EA0C07B5
:1050C8003D4316F4403F056041D023F0030707F144
:1050D800804707F5803703F0030CBD684FEA8C0C56
:1050E8004FF0070E0EFA0CFEB0F1904F25EA0E0EA7
:1050F8002FD01B4DA8422ED005F58065A8420CBFC5
:105108000225072505FA0CF545EA0E05BD60256858
:10511800D74316F4801F0CBF3D40154325606568D2
:1051280016F4001F0CBF3D4015436560D4F880504D
:1051380016F4803F0CBF3D401543C4F88050D4F8A6
:105148008450B60354BF3D401543C4F8845001331E
:1051580062E70025D6E70125D4E700BF000800581C
:1051680000040048374A2DE9F04F00234FF0010AA8
:105178004FF0070B4FF00F0931FA03F401D1BDE8E6
:10518800F08F0AFA03FC1CEA010654D023F003044A
:1051980004F1804404F5803403F00307A568BF00D8
:1051A8000BFA07F8B0F1904F08EA050E45D0264DE6
:1051B800A84244D005F58065A8420CBF0225072502
:1051C800BD40754517D1D2F8805025EA0605C2F8CA
:1051D8008050D2F8845025EA0605C2F88450156834
:1051E80025EA06051560556825EA06055560A5688F
:1051F80025EA0805A560056803265C0006FA04F49C
:1052080023FA06F6254300EB8606056003F007053A
:10521800376AAD0009FA05F527EA05073762856898
:1052280025EA04058560456825EA0C054560C568DA
:1052380025EA0404C46001339EE70025C0E7012580
:10524800BEE700BF0008005800040048036919427F
:1052580014BF0120002070470AB181617047816244
:1052680070470000044AD168014208B502D0D060F6
:10527800FEF717F908BD00BF0008005810B504462E
:1052880000284AD090F8413003F0FF021BB980F89B
:105298004020FDF7FDF8242384F8413023681A687C
:1052A80022F001021A60626822F070621A619A683C
:1052B80022F400429A60D4E90221012924D142F45F
:1052C80000429A605A6842F0007242F400425A6002
:1052D800DA6822F40042DA60D4E904210A43A169B9
:1052E80042EA0122DA60D4E907210A431A601A68FF
:1052F80042F001021A6000202023606484F84130E3
:10530800206384F8420010BD42F4044202299A60E6
:1053180004BF4FF400625A60D4E70120F3E710B5E8
:1053280090F84120202A0346D4B21CD190F840209E
:10533800012A18D0242280F841200268106820F041
:1053480001001060106820F480501060106801435C
:1053580011601168002041F00101116083F841409B
:1053680083F8400010BD0220FCE710B590F84120FA
:10537800202A0346D4B21BD190F84020012A17D026
:10538800242280F841200268106820F00100106093
:10539800106820F4706040EA012111601168002053
:1053A80041F00101116083F8414083F8400010BDCD
:1053B8000220FCE7024A136843F4807313607047C5
:1053C800000400580D4B10B55B690C4628B99A05C6
:1053D80007D500F027F820B110BD9B0501D400F0D7
:1053E80019F8074A1369012C23F00403136101D14A
:1053F80030BFF1E740BF20BF20BFEDE700040058F1
:1054080000ED00E0024B186800F4C060704700BF70
:1054180000040058024A136843F48043136070473D
:10542800000400580C4A136823F4804313600B4BA4
:105438001B6832214B430A49B3FBF1F351698905D3
:1054480000D533B9536913F4007F14BF032000203B
:105458007047013BF2E700BF00040058B800002085
:1054680040420F000B4A136823F0070343F002037E
:105478001360094B1A69012842F004021A6105D128
:1054880030BF1A6922F004021A61704740BF20BF7A
:1054980020BFF6E70004005800ED00E04FF0B043ED
:1054A8001868C0F3404070474FF0B0431868C0F325
:1054B800400070474FF0B042536823F47F4343EAFB
:1054C8000023536070474FF0B0431868C0F3406042
:1054D800704700007FB54FF0B0432C4AD3F808312D
:1054E800C0F3031003F00F0352F82040284A52F883
:1054F8002330B4FBF3F4FFF785FF264B054693E80A
:105508000700B5F5007F04AB03E9070010D0224B74
:105518009C4218D303F5B70303F67F539C4229D95D
:1055280003F5741303F510639C4225D802230BE09E
:105538001A4B9C4207D91A4B9C421BD903F53703D7
:1055480003F5D853F0E7002304AA02EB830353F8CA
:105558000C4C144D2B6823F0070323432B60FDF7F5
:105568009FFA06462B6803F007039C4206D10020E9
:1055780004B070BD0123E7E70024EAE7FDF790FADD
:10558800801B0228EED90320F2E700BFD00F0108E4
:10559800700F0108400E0108C0CF6A00BFEA210160
:1055A8003F933402004000584FF0B04310B59A685A
:1055B800D96812F00C0205D00C2A4AD101F0030375
:1055C800012B50D14FF0B0412B480B6813F0080362
:1055D80006D00B6813F0080337D1D1F8941007E010
:1055E8000C68240756BFD1F894300968C3F3032325
:1055F80050F82330002A0CBF184600204FF0B04165
:105608008A6802F00C020C2A1ED1CA6802F0030252
:10561800022A2ED0032A06D10B68184A13F4801FD9
:10562800174B18BF13464FF0B042D068D168D26804
:10563800C0F306205843C1F302130133B0FBF3F063
:10564800530F0133B0FBF3F010BD0B68C3F3031322
:10565800CEE7042A0AD0082A05D11B6813F4801360
:1056680004D10748CAE700231846C7E703480023C0
:10567800C4E7024BD7E700BFD00F01080024F400AD
:105688000048E80108B5FFF78FFF4FF0B043044A20
:105698009B68C3F3031352F82330B0FBF3F008BD43
:1056A800700F01082DE9F0410446002853D04FF04F
:1056B800B0439D68DE6803689B0605F00C0506F09C
:1056C800030668D5026A1DB10C2D46D1012E44D1BE
:1056D800002A40D04FF0B043A16A1A68170756BF96
:1056E800D3F894301B681B0903F0F00399421FD9C3
:1056F8000846FFF7EFFE00282DD14FF0B04213689F
:1057080043F0080313601368A16A23F0F0030B4306
:105718001360606AFFF7CEFEFFF7B4FFAB4B18606B
:10572800AB4B1868FDF7BAF9002834D0BDE8F08112
:105738004FF0B042136843F008031360136823F076
:10574800F0030B431360606AFFF7B4FE0846FFF7E7
:10575800C1FE0028E0D00120E8E74FF0B043002A5E
:1057680054D01A6842F001021A60FDF799F9074609
:10577800FFF79AFE002842D04FF0B042136843F07A
:10578800080313601368A16A23F0F0030B43136046
:10579800606AFFF78FFE2368D80748D42368990703
:1057A80000F18C8023681E0740F1FA80A3694FF04E
:1057B800B046002B00F0E180D6F89430E16903F0A0
:1057C8001002914200F0C48003F00302022AC2D002
:1057D800D80740F1B380D6F8943023F00103C6F817
:1057E8009430FDF75DF90746D6F89430990740F1F3
:1057F800A580FDF755F9C31B112BF5D904E0FDF77A
:105808004FF9C01B0228B3D903208FE71A6822F08A
:1058180001021A60FDF744F90746FFF745FE002824
:10582800B9D0FDF73DF9C01B0228F6D9ECE7082DE1
:1058380003D00C2D05D1032E03D16368002BADD105
:1058480089E74FF0B043A1681A6822F480120A432E
:105858001A606268B2F5803F10D11A6842F480324B
:105868001A60FDF71DF90746FFF718FE002895D1C5
:10587800FDF716F9C01B6428F6D9C5E7B2F5041F71
:1058880004D11A6842F400121A60E6E7196821F494
:1058980080311960196821F400111960002AE0D1DB
:1058A800FDF7FEF80746FFF7F9FD00283FF476AF4D
:1058B800FDF7F6F8C01B6428F5D9A5E7042D236980
:1058C80003D00C2D0ED1022E0CD1002B3FF443AF88
:1058D8004FF0B0426169536823F0FE4343EA016325
:1058E80053605FE74FF0B046BBB1336843F4807351
:1058F8003360FDF7D5F8074633685A0507D573684E
:10590800626923F0FE4343EA026373604AE7FDF7E6
:10591800C7F8C31B022BEFD976E7336823F48073EB
:105928003360FDF7BDF8074633685B057FF53AAF8E
:10593800FDF7B6F8C31B022BF6D965E74FF0B04266
:10594800E169D2F8943023F010030B43C2F8943085
:105958004FF0B047D7F8943043F00103C7F89430BC
:10596800FDF79EF80646D7F894309A0718D4FDF745
:1059780097F8831B112BF6D946E7D6F8943023F015
:105988000103C6F89430FDF78BF80746D6F8943033
:105998009B0705D5FDF784F8C31B112BF6D933E710
:1059A8002368580754D50B4F3B68D90514D4FFF723
:1059B80001FDFDF775F806463B68DA050CD4FDF7DE
:1059C8006FF8831B022BF7D91EE700BFB800002031
:1059D800BC00002000040058E3684FF0B046002BDC
:1059E80058D023F08003052B02BFD6F8903043F03F
:1059F8000403C6F890304FF0B046FDF751F8D6F8DA
:105A0800903043F001030746C6F8903041F28838D9
:105A1800D6F890309B0705D4FDF742F8C31B4345E1
:105A2800F6D9F1E6E36823F00403812B1BD1FDF7D7
:105A380037F8D6F8903043F08003C6F89030074620
:105A48004FF0B04641F28838D6F89030180504D5A2
:105A5800E06A00284AD1002068E6FDF721F8C01B5B
:105A68004045F1D9D0E6FDF71BF8D6F8903023F081
:105A78008003C6F8903007464FF0B04641F28838A8
:105A8800D6F890301905E3D5FDF70AF8C01B404554
:105A9800F6D9B9E6FDF704F8D6F8903023F080037C
:105AA8000746C6F8903041F28838D6F890301A0583
:105AB80016D4FCF7F5FFD6F8903023F00103C6F8AA
:105AC800903007464FF0B04841F28836D8F8903009
:105AD8009B07BDD5FCF7E4FFC31BB342F6D993E699
:105AE800FCF7DEFFC01B4045DFD98DE60C2D4ED0FC
:105AF8004FF0B04302281A6822F080721A6033D13E
:105B0800FCF7CEFF0546FFF7DEFC38BBD4E90C31C5
:105B18004FF0B0420B43D0682D4901400B43E16B75
:105B28000B43216C0B43616C0B43A16B43EA0123CC
:105B3800D360136843F080731360D36843F08053D5
:105B4800D360FCF7ADFF0446FFF7BDFC002882D107
:105B5800FCF7A6FF001B0A28F6D955E6FCF7A0FFBC
:105B6800401B0A28CFD94FE6FCF79AFF0446FFF7F7
:105B7800AAFC30B94FF0B042164BD1680B40D36045
:105B8800D4E5FCF78DFF001B0A28F0D93CE6012874
:105B98003FF4CCAD4FF0B043226BDB6803F0030158
:105BA80091427FF4D8AD616B03F070028A427FF4B2
:105BB800D2ADA16B03F4FE42B2EB012F7FF4CBAD63
:105BC800626C03F0604393423FF445AFC3E500BF06
:105BD8008C80C111FCFFFEEE2DE9F0410D46044614
:105BE80010B90120BDE8F081684E336803F007035F
:105BF8008B4216D323689A0727D54FF0B047A2687F
:105C0800BB6823F0F0031343BB60FCF749FF06466B
:105C1800BB68DB0319D4FCF743FF831B022BF7D9BE
:105C280011E0336823F007030B433360FCF738FFB8
:105C38000746336803F00703AB42DBD0FCF730FFBD
:105C4800C01B0228F5D90320CCE72368580617D5CE
:105C58004FF0B0476269D7F8083123F00F0343EAE1
:105C68001213C7F80831FCF71BFF0646D7F80831AE
:105C7800D90305D4FCF714FF831B022BF6D9E2E7FE
:105C880023685A0713D54FF0B047E268BB6823F47E
:105C9800E0631343BB60FCF703FF0646BB689B0346
:105CA80005D4FCF7FDFE831B022BF7D9CBE723684D
:105CB800180714D54FF0B0472269BB6823F4605326
:105CC80043EAC203BB60FCF7EBFE0646BB68590318
:105CD80005D4FCF7E5FE831B022BF7D9B3E723684D
:105CE800DA070FD4294C236803F00703AB4239D8ED
:105CF800FFF7C8FC264B1860264BBDE8F041186832
:105D0800FCF7CCBE6268022A1DD1FFF7C7FB00284A
:105D18003FF467AF4FF0B04641F28838B36823F0DC
:105D280003031343B360FCF7BBFE0746B36862681E
:105D380003F00C03B3EB820FD4D0FCF7B1FEC01B09
:105D48004045F3D97FE7032A02D1FFF7BCFBDEE722
:105D580012B9FFF7A9FBDAE74FF0B0431B685B0500
:105D6800D8D43EE7236823F007032B432360FCF7CE
:105D780097FE0646236803F00703AB42B8D0FCF74A
:105D88008FFE801B0228F5D95DE700BF0040005850
:105D9800B8000020BC00002008B5FFF773FC4FF0E6
:105DA800B043044A9B68C3F3022352F82330D84017
:105DB80008BD00BFB00F010808B5FFF763FC4FF03E
:105DC800B043044A9B68C3F3C22352F82330D84037
:105DD80008BD00BFB00F01084FF0B043D3F89000E2
:105DE800C0F3400070474FF0B0410209D1F8883045
:105DF80002F47F22000123EA020300F47F20034318
:105E0800C1F8883070474FF0B041020CD1F88830A3
:105E1800120423EA020343EA0040C1F888007047ED
:105E280070B5066816F48036044638D0FFF7C2FA13
:105E3800FCF736FE614E05463368DB0529D54FF081
:105E4800B043616BD3F8902002F44072914214D0B1
:105E5800D3F89010D3F8902042F48032C3F8902001
:105E6800D3F8902021F4407022F480328D07C3F8D3
:105E78009020C3F8900000F190804FF0B042616B21
:105E8800D2F8903023F440730B43C2F890300026C8
:105E980005E0FCF705FE401B0228CDD9032625683E
:105EA800E8070AD54FF0B0416268D1F8883023EA94
:105EB800124392B21343C1F88830A9070AD54FF0AC
:105EC800B041A268D1F8883023EA124392B2134352
:105ED800C1F88830AA0609D54FF0B0422169D2F836
:105EE800883023F440630B43C2F88830AB0502D5F1
:105EF800206AFFF788FF680502D5606AFFF783FF0D
:105F0800290502D5A06AFFF77EFF6A0602D56069F7
:105F1800FFF769FF2B0602D5A069FFF764FFE805C4
:105F280002D5E069FFF75FFFE90610D54FF0B042F0
:105F3800E168D2F8883023F440730B43C2F8883004
:105F4800B1F5807F02BFD36843F08073D3602A0421
:105F58000ED54FF0B042216BD2F8883023F0404381
:105F68000B43C2F8883019B9D36843F08073D36003
:105F78006B0410D54FF0B042E16AD2F8883023F0B4
:105F880040530B43B1F1005FC2F8883003D1D368A6
:105F980043F48033D360304670BDFCF781FD41F295
:105FA80088360546FFF718FF01283FF466AFFCF76F
:105FB80077FD401BB042F5D970E700BF00040058D8
:105FC80030B590F82C30012B02464FF0020022D059
:105FD800174B82F82D00CA24012582F82C505C62E8
:105FE80053245C62B1F5807F146B996914D121F454
:105FF80088519961596C24F0010421F000415964D9
:106008001463DD650A4BFF2159620020012382F8E1
:106018002D3082F82C0030BD21F408519961D96CDB
:1060280024F0020421F00041D9641463D865E9E73B
:106038000028004070B50B4E036B756D1D40EA07D4
:10604800044603D50123F365FCF79BFEAB0704D593
:106058000223F365204600F0CBF9012384F82D30A4
:1060680070BD00BF0028004038B50A4CE36823F033
:106078002003E360FCF714FD0546E3689B0601D5A1
:10608800002038BDFCF70CFD401BB0F57A7FF4D931
:106098000320F6E7002800402DE9F041114DEC6897
:1060A80014F0400407461AD1EB6843F08003EB6014
:1060B800FCF7F6FC4FF003080646EB685B0601D4D4
:1060C800032C02D12046BDE8F081FCF7E9FC801BD7
:1060D800B0F57A7F84BF87F82D800324EDE700248C
:1060E800F0E700BF0028004038B50F4CE36823F004
:1060F8008003E360A3699B06054606D4FFF7B4FF57
:1061080010B1032085F82D0038BDA36923F02003C2
:10611800A361FFF7A9FF10B1032085F82D00A3693B
:1061280043F02003A361EFE70028004038B5044698
:1061380000284BD090F82D3003F0FF021BB980F8EF
:106148002C20FCF7B5FA0223214D84F82D30EB689A
:10615800DB0632D4CA236B6253236B622046FFF7F7
:106168009BFF78BBAB6923F08E6323F04003AB61E0
:1061780021696368AA690B431343A2691343AB619E
:10618800D4E9022343EA02432B61D4E90931EA68DE
:106198000B4322F4F8521343EB602046FFF7A4FFA9
:1061A80080B9D4E90713AA690B4322F0604213436C
:1061B80062691343AB61FF236B62012384F82D30BE
:1061C800002002E0024BFF225A6238BD0120FCE7A2
:1061D800002800400023092803D840EA0310C0B271
:1061E80070470A380133C0B2F5E700002DE9F047DF
:1061F80090F82C30012B05464FF0020069D001239E
:1062080085F82C304E4B85F82D00DE6806F4407674
:10621800B6F5807F78D04C69087891F8019091F8AC
:1062280002A091F82470002A55D19B6913F040030D
:1062380008BFCB70FFF7CEFF80464846FFF7CAFF7E
:1062480002465046FFF7C6FF81463846FFF7C2FFB1
:106258000B6ACF78234343EA875343EA090343EAA7
:10626800084343EA022343EA0063354ACA205062DE
:10627800532050628C6A8869B4F5807F946945D14F
:1062880024F4885494610124D465B6F5807F09BF4D
:10629800CB6913640343536418BF5064284B4A689E
:1062A8001A672A6B42F001022A639A6942F48852FB
:1062B8009A61244AD2F8803043F40033C2F880301F
:1062C8001F4BFF225A620020012385F82D3085F8E4
:1062D8002C00BDE8F087B4F1803F07D0B4F5000F7B
:1062E80004D09B6913F0400308BFCB700B6ACA78CF
:1062F8001C4344EA0A0444EA004343EA092343EA04
:10630800825343EA0763B0E70023AEE724F4085456
:1063180094610224D465B6F5807F09BFCB69936484
:106328000343D36418BFD064054B4A685A672A6B85
:1063380042F002022A639A6942F40852B8E700BFA1
:10634800002800400008005890F82C20012A034635
:106358004FF0020012D00A4A83F82D00CA21516278
:1063680053215162916941F020019161FF215162ED
:106378000020012283F82D2083F82C00704700BFED
:106388000028004090F82C20012A03464FF0020014
:1063980019D00D4A83F82D00CA2151625321516248
:1063A80091690A4841F080019161D0F8801041F468
:1063B8008021C0F88010FF2151620020012283F85B
:1063C8002D2083F82C007047002800400008005852
:1063D800064B5A6D520610B5044603D54022DA65BD
:1063E800FCF7D2FC012384F82D3010BD00280040B2
:1063F8007047890001F1804101F531410A60704719
:10640800890001F1804101F53141086870470000B9
:10641800034AD2F8903043F40043C2F890307047F2
:1064280000040058034AD2F8903023F40043C2F81D
:106438009030704700040058074B1A6822F0400259
:106448001A6040F441704FF4B85218605A601A68E4
:1064580042F040021A6070470000015837B50546FF
:1064680000284ED0837903F0FF046BB1032C0BD0C6
:10647800254B4FF400629A612868FFF7DDFF00247E
:1064880001232B71AC602FE000236B712846FCF7C9
:106498001FFA1E4AD2F8903043F48053C2F8903065
:1064A800002CE5D102234FF0B042AB71D2F8943002
:1064B80023F40043C2F89430154B1B681C214B434E
:1064C800DB0C64214B430193019B93B90124AC601D
:1064D800FFF79EFF0C4B9A6842F400629A604FF4F3
:1064E80000629A61002CC7D00123AB71204603B02B
:1064F80030BD019B013B0193D2F894305B04E3D497
:10650800E6E70124F2E700BF00040058000800583D
:10651800B800002037B5174D2B6802461C204343AE
:10652800DB0C6420434314480193019B93B9012079
:106538009060114C21732B681C214B43DB0C6421A8
:106548004B430193019B6BB9012090600A4BDB68B8
:1065580003B030BD019B013B019383689C07E4D5E0
:106568000020E6E7019B013B0193A368DB07E9D51F
:10657800ECE700BFB80000200000015837B5184DFF
:106588002B6802461C204343DB0C64204343154818
:106598000193019BA3B901209060124CFF23237340
:1065A8002B681C256B43DB0C64256B430193019B13
:1065B80073B9012090600B4BDB680B7003B030BDE2
:1065C800019B013B019383689C07E2D50020E4E727
:1065D800019B013B0193A368DB07E8D5EBE700BF0C
:1065E800B8000020000001580F4B13B51B680F4C72
:1065F800182253431B0D64225343014601936269D9
:10660800019B02F0040223B902238B60012002B02F
:1066180010BD019B013B0193606910F00200F6D0A8
:10662800002AECD11046F2E7B80000200004005818
:1066380007B50379012B0FD10A4B1B681822534366
:106648001B0C0193FFF7EEFE019B013B0193019B9D
:10665800002BF9D1FFF7DCFE03B05DF804EBFFF780
:10666800C3BF00BFB8000020F8B51E468379012BD0
:10667800154604460F46DAB22DD14379012B2AD0AC
:10668800022342718371FFF7D3FF0D212046FFF7E4
:10669800C9FEFFF73FFF390A2046FFF73BFFF9B273
:1066A8002046FFF737FF2E44B5420ED12046FFF7AC
:1066B800AFFEFFF799FFA06801230038A3714FF0E0
:1066C800000318BF01206371F8BD15F8011B2046AF
:1066D800FFF720FFE8E70220F6E7F8B51E468379C2
:1066E800012B154604460F46DAB22FD14379012B08
:1066F8002CD04271FFF79CFF1D212046FFF792FE28
:10670800FFF708FF390A2046FFF704FFF9B22046D1
:10671800FFF700FF00212046FFF7FCFE2E44B5429C
:106728000ED12046FFF774FEFFF75EFFA068012335
:106738000038A3714FF0000318BF01206371F8BD42
:1067480029462046FFF71AFF0135E8E70220F6E759
:10675800F8B51F468379012B154604460E46DAB272
:106768002CD14379012B29D04271FFF761FF06F044
:10677800EF03A3F18402534253412371314620466B
:10678800FFF750FEFFF7C6FE2F44AF4210D1FFF7C8
:106798003FFE842E02D02046FFF726FFA068012383
:1067A8000038A3714FF0000318BF01206371F8BDD2
:1067B80015F8011B2046FFF7ADFEE6E70220F6E7D5
:1067C800F8B51E468379012B154604460F46DAB202
:1067D80027D14379012B24D04271FFF729FF39468D
:1067E8002046FFF71FFEFFF795FE00212046FFF722
:1067F80091FE2E44B5420ED12046FFF709FEFFF761
:10680800F3FEA06801230038A3714FF0000318BFFE
:1068180001206371F8BD29462046FFF7AFFE013518
:10682800E8E70220F6E737B50023ADF8043001AAFF
:10683800022312210546FFF7C3FFBDF804400223D7
:1068480064BA01AAA4B219462846FFF781FFE207F5
:1068580002D5284609F076FBA30702D5284609F099
:1068680077FB600702D5284609F09CFB210702D573
:10687800284609F09DFBE20602D5284609F09EFB52
:10688800A30602D5284609F087FB600602D52846EC
:1068980009F064FB210606D514F4807118BF0121A4
:1068A800284609F061FBA20502D5284609F06CFBD1
:1068B800630402D5284609F087FB03B030BDF8B55C
:1068C8001E468379012B154604460F46DAB227D1B6
:1068D8004379012B24D04271FFF7AAFE0E212046EE
:1068E800FFF7A0FDFFF716FE39462046FFF712FE18
:1068F8002E44B5420ED12046FFF78AFDFFF774FEFD
:10690800A06801230038A3714FF0000318BF0120CD
:106918006371F8BD15F8011B2046FFF7FBFDE8E79A
:106928000220F6E7F8B51E468379012B1546044682
:106938000F46DAB22BD14379012B28D04271FFF7E9
:1069480077FE1E212046FFF76DFDFFF7E3FD394670
:106958002046FFF7DFFD00212046FFF7DBFD2E4430
:10696800B5420ED12046FFF753FDFFF73DFEA06864
:1069780001230038A3714FF0000318BF0120637191
:10698800F8BD29462046FFF7F9FD0135E8E7022062
:10699800F6E7026852E8003F23F0C00342E80031FE
:1069A80002680029F5D102F1080353E8003F23F4F7
:1069B800000302F1080C4CE800310029F3D1202330
:1069C800C0F888307047000010B5026852E8003FF0
:1069D80023F4907342E8003102680029F5D10F4C86
:1069E80002F1080353E8003F234002F1080C4CE889
:1069F80000310029F4D1C36E012B07D152E8003FC2
:106A080023F0100342E800310029F7D12023C0F811
:106A18008C300023C366436710BD00BFFEFFFFEF45
:106A2800F8B504461346D4F88850202D32D1F1B178
:106A3800EAB1E06FA4F85620A4F8542000262122D9
:106A4800C4F890602165C4F88820226888B1124F84
:106A5800C762124F0763124F2832C0E90D76FEF75E
:106A6800D7F830B11023C4F89030C4F8885001200A
:106A78000FE0236840221A62226802F1080353E8F3
:106A8800003F43F0800302F1080141E8003000288C
:106A9800F3D1F8BD0220FCE7AD6A0008F56A0008EA
:106AA800016B000808B50346806A1B681B6813F071
:106AB800200317D1A0F85630026802F1080353E802
:106AC800003F23F08003083242E8003102680029C1
:106AD800F2D152E8003F43F0400342E80031002978
:106AE800F7D108BDFCF7A6FAFBE7704708B5806A3E
:106AF800FFF7FBFF08BD7047806A38B50468D0F817
:106B08008830D0F88C50A268120606D5212B04D103
:106B18000023A0F85630FFF73CFFA3685B0606D5B4
:106B2800222D04D10023A0F85E30FFF74DFFD0F8E6
:106B3800903043F01003C0F89030FFF7DCFF38BD09
:106B480008B5806A0023A0F85E30A0F85630FFF739
:106B5800D2FF08BD704700000368D9691A682DE99B
:106B6800F04140F60F0631429D68044610D18E066A
:106B780040F1978002F0200605F080573E4300F070
:106B88009080436F002B00F08580BDE8F0411847E6
:106B9800AB4EAC482E401040304300F08280CF0707
:106BA80009D5D00507D501201862D4F8900040F027
:106BB8000100C4F890008F0709D5E80707D502201F
:106BC8001862D4F8900040F00400C4F890004F0711
:106BD80009D5E80707D504201862D4F8900040F0DA
:106BE8000200C4F890000F070BD502F020003043D4
:106BF80007D008201862D4F8900040F00800C4F8C4
:106C080090000E050AD5500108D54FF400601862AF
:106C1800D4F8903043F02003C4F89030D4F8903082
:106C2800002B37D08B0609D502F0200205F08055DD
:106C38002A4303D0636F0BB1204698472668D4F8DF
:106C48009020B36802F0280203F0400353EA0205DB
:106C5800204621D0FFF7B8FEB3685F0617D5226833
:106C680002F1080353E8003F23F04003083242E8EA
:106C780000310029F3D1D4F8800040B1724B83630E
:106C8800FEF73FF830B1D4F88000836B7DE72046EB
:106C9800FFF731FFBDE8F081FFF72DFFC4F89050F2
:106CA800F8E7E06E012840F08980CE0640F1868042
:106CB800D00640F1838010221A629A6851064BD59B
:106CC800D4F8802011684A6892B2002AE2D0B4F859
:106CD8005C009042DED9A4F85E200A6892062FD4A0
:106CE80053E8002F22F4807243E800210029F7D1ED
:106CF80003F1080252E8002F22F0010203F1080014
:106D080040E800210029F3D103F1080252E8002FDE
:106D180022F0400203F1080040E800210029F3D1E5
:106D28002022C4F88C20E16653E8002F22F01002DC
:106D380043E800210029F7D1D4F88000FDF7ACFF23
:106D480002232367B4F85E30B4F85C10C91A89B21C
:106D58002046FFF7FFFE9DE7B4F85E20B4F85E001A
:106D6800B4F85C1080B292B2002893D0891A89B224
:106D780000298FD053E8002F22F4907243E80020B6
:106D88000028F7D1314D03F1080252E8002F2A40BC
:106D980003F1080646E800200028F4D12022C4F8B0
:106DA8008C206067E06653E8002F22F0100243E869
:106DB80000200028F7D102232367C9E7CF0209D5AD
:106DC8006E0207D54FF4801220461A62BDE8F041E2
:106DD80000F0A0BD08060BD502F0800005F4000500
:106DE800284305D0A36F002B3FF454AF2046CCE6D0
:106DF8004F0611D556060FD553E8002F22F0400252
:106E080043E800210029F7D12023C4F88830A1677E
:106E18002046FCF70FF93DE70D0206D5500004D5D2
:106E28002046BDE8F04100F077BDCB017FF532AFD9
:106E3800002ABFF62FAF2046BDE8F04100F06BBD39
:106E48000100001020010004496B0008FEFFFFEF5D
:106E5800D0F88C20B0F86010222A08B5036855D104
:106E68005B6A826D0B401370836D01338365B0F8E4
:106E78005E30013B9BB2A0F85E30B0F85E309BB24A
:106E8800002B42D1026852E8003F23F4907342E895
:106E9800003103680029F5D103F1080252E8002FF8
:106EA80022F0010203F1080C4CE800210029F3D17B
:106EB8002022C0F88C20184A41679342016705D107
:106EC800C26E012A0ED0FCF7C3F81EE05A68110200
:106ED800F6D553E8002F22F0806243E8002100290C
:106EE800F7D1EDE70022C26653E8002F22F0100226
:106EF80043E800210029F7D1DA69B0F85C10D2061E
:106F080044BF10221A62FFF725FE08BD9A6942F0B5
:106F180008029A61F9E700BF00800040D0F88C2091
:106F2800B0F86010222A08B5036852D15A6A114095
:106F3800826D22F8021B8265B0F85E20013A92B297
:106F4800A0F85E20B0F85E2092B2002A40D153E843
:106F5800002F22F4907243E800210029F7D103F1B1
:106F6800080252E8002F22F0010203F1080C4CE855
:106F780000210029F3D12022C0F88C20174A41674C
:106F88009342016705D1C26E012A0ED0FCF760F862
:106F98001EE05A681102F6D553E8002F22F08062ED
:106FA80043E800210029F7D1EDE70022C26653E843
:106FB800002F22F0100243E800210029F7D1DA69F6
:106FC800B0F85C10D20644BF10221A62FFF7C2FD67
:106FD80008BD9A6942F008029A61F9E7008000400A
:106FE8002DE9F74F0368B0F86080DF691A689D687B
:106FF800D0F88C1001922229044640F0B480B0F8F1
:107008006890DFF86CA1DFF86CB10026B9F1000FC9
:1070180001D0BB0621D4B4F85E309BB2D3B1B4F82A
:1070280068209A4216D9226802F1080353E8003F03
:1070380023F08053083242E8003122680029F2D157
:107048004D4B636752E8003F43F0200342E80031AC
:107058000029F7D103B0BDE8F08F2368A26D5B6A01
:1070680003EA08031370A36D0133A365B4F85E3017
:10707800013B9BB2A4F85E302368DF6978072CD007
:10708800F9070AD5019AD20507D501211962D4F862
:10709800901041F00101C4F89010B80709D5E9072C
:1070A80007D502211962D4F8901041F00401C4F800
:1070B80090107A0709D5E80707D504211962D4F892
:1070C800903043F00203C4F89030D4F8903023B1E4
:1070D8002046FFF710FDC4F89060B4F85E309BB20C
:1070E800002B93D1216851E8003F23F4807341E8D5
:1070F800003023680028F5D103F1080252E8001F88
:1071080001EA0A0142E800100028F5D120215B4578
:10711800C4F88C10606720670AD05968090207D53F
:1071280053E8001F21F0806143E800100028F7D1E0
:10713800E16E012913D1E66653E8001F21F0100122
:1071480043E800100028F7D1D969CA0644BF1021C6
:1071580019622046B4F85C10FFF7FCFC56E720469D
:10716800FBF776FF52E79A6942F008029A6171E7E5
:10717800FEFFFFEF00800040596E00082DE9F74F31
:107188000368B0F86080DF691A689D68D0F88C10D1
:1071980001922229044640F0B280B0F86890DFF8E6
:1071A80068A1DFF868B10026B9F1000F01D0BB066D
:1071B80021D4B4F85E309BB2D3B1B4F868209A42B7
:1071C80016D9226802F1080353E8003F23F08053E0
:1071D800083242E8003122680029F2D14C4B63673B
:1071E80052E8003F43F0200342E800310029F7D17C
:1071F80003B0BDE8F08F2368A26D596A08EA01015F
:1072080022F8021BA265B4F85E20013A92B2A4F8F3
:107218005E20DF6978072CD0F9070AD5019AD205D4
:1072280007D501211962D4F8901041F00101C4F882
:107238009010B80709D5E90707D502211962D4F8D3
:10724800901041F00401C4F890107A0709D5E807B6
:1072580007D504211962D4F8903043F00203C4F82A
:107268009030D4F8903023B12046FFF744FCC4F89E
:107278009060B4F85E309BB2002B95D1216851E83C
:10728800003F23F4807341E8003023680028F5D1DB
:1072980003F1080252E8001F01EA0A0142E800105F
:1072A8000028F5D120215B45C4F88C106067206761
:1072B8000AD05968090207D553E8001F21F08061F8
:1072C80043E800100028F7D1E16E012913D1E666E2
:1072D80053E8001F21F0100143E800100028F7D1FF
:1072E800D969CA0644BF102119622046B4F85C1057
:1072F800FFF730FC58E72046FBF7AAFE54E79A69E7
:1073080042F008029A6173E7FEFFFFEF0080004039
:10731800256F000838B5044603682169A2681D680E
:10732800C0690A4361690A437D49024329400A4307
:107338001A605A68E16822F440520A435A60794A4E
:10734800A16993421CBF226A11439A6822F06E42D7
:1073580022F430620A439A60DA6A616A22F00F0204
:107368000A43DA62704A93421CD14FF0B043D3F813
:10737800883003F0030343F44033A3F54033013B63
:10738800022B00F2C780694A9B5CB0F5004F40F0C1
:107398008980082B24D8DFE803F061C08323802389
:1073A80023236500624A934209D14FF0B043614AF2
:1073B800D3F8883003F00C0343F44023E4E7594A38
:1073C80093420DD14FF0B043D3F8883003F44063B3
:1073D800B3F5006F1AD005D853B1B3F5806F12D04A
:1073E800012009E0B3F5406FFAD14FF400400EE0F8
:1073F800FEF7D2FC58B900204FF00113A366002312
:10740800C4E91D3338BDFEF7CFF8F3E74A4865688D
:107418004A4B626A05EB450133F81220B0FBF2F3E0
:107428009942DDD8B3EB053FDAD800231946FAF7BD
:107438006BFB090241EA10616B080002C0182A467A
:107448004FF0000341F10001FAF75EFB3C4BA0F559
:1074580040729A42C4D82368D860CCE7FEF79CFCF7
:107468000028C8D06168354B626A33F81220B0FB37
:10747800F2F24B0803EB42034FF6EF72B3FBF1F362
:10748800A3F110019142ABD823F00F02216892B208
:10749800C3F342031343CB60ADE7FEF785F8DFE79C
:1074A8002548DFE7082B9BD801A252F823F000BF3C
:1074B800017500080D75000819750008E9730008C2
:1074C80013750008E9730008E9730008E9730008F8
:1074D800DD7400084FF400406368616A174A32F8A7
:1074E8001120B0FBF2F000EB5300B0FBF3F04FF6C5
:1074F800EF73A0F11002ACE7FEF74EFC00283FF452
:107508007AAFE9E7FEF758FCF8E7FEF74DF8F5E73C
:107518000948E1E7B0F5004FF4D1FEF74DFC9FE7CD
:10752800F369FFCF008000400038014010100108C7
:10753800004400401310F5070024F400201001084F
:10754800FFFC0F00836ADA0710B506D50168C46A24
:107558004A6822F4003222434A609C0706D5016833
:10756800046B4A6822F4803222434A60590706D5E0
:107578000168446B4A6822F4802222434A601A0751
:1075880006D50168846B4A6822F4004222434A60A7
:10759800DC0606D50168C46B8A6822F4805222434F
:1075A8008A60990606D50168046C8A6822F400523C
:1075B80022438A605A060FD50168446C4A6822F44F
:1075C80080122243B4F5801F4A6005D14A68846C52
:1075D80022F4C00222434A601B0606D50268C16C29
:1075E800536823F400230B43536010BD2DE9F04189
:1075F800DDF8188004460E4615461F462268D369F2
:1076080036EA03030CBF01230023AB4201D000205C
:1076180027E0B8F1FF3FF2D0FBF742FAC01B404524
:10762800206802D8B8F1000F1DD150E8003F23F4BC
:10763800D07340E80032002AF7D100F1080353E87C
:10764800003F23F0010300F1080141E80032002A5D
:10765800F3D12023C4F88830C4F88C3084F884200F
:107668000320BDE8F08103685A07C7D5C3691B0525
:10767800C4D54FF40063036250E8003F23F4D0738D
:1076880040E80032002AF7D100F1080353E8003F30
:1076980023F0010300F1080141E80032002AF3D188
:1076A8002023C4F88830C4F88C30C4F89030D5E76B
:1076B80073B504460026C0F89060FBF7F1F923681B
:1076C8001B681A07054619D423681B685B070AD587
:1076D8006FF07E43009300222B464FF48001204632
:1076E800FFF784FFB0B900202023C4F8883084F85D
:1076F8008400C4F88C30E06620670CE06FF07E43AD
:107708000093324603464FF400112046FFF76EFF00
:107718000028D9D0032002B070BD10B5044650B37C
:10772800D0F888301BB980F88430FBF76FFB2268EB
:107738002423C4F88830136823F00103136020461B
:10774800FFF7E8FD012816D0A36A13B12046FFF71A
:10775800F9FE23685A6822F490425A609A6822F027
:107768002A029A601A6842F0010220461A60BDE8AF
:107778001040FFF79DBF012010BD000030B58165A6
:107788008168A0F85C200023B1F5805FA0F85E2036
:10779800436735D10369002B40F2FF1318BFFF235D
:1077A800A0F860300023C0F890302223C0F88C3055
:1077B800016801F1080353E8003F43F00103083171
:1077C80041E800340368002CF2D1456E84680169F1
:1077D800B5F1005F34D1B0F86850954230D8B4F5AF
:1077E800805F1DD1254A264C002918BF22464267D2
:1077F800C1B153E8002F42F4807243E80021F7E753
:1078080029B90369002B14BF7F23FF23C8E7B1F10F
:10781800805FC5D10369002B0CBF7F233F23BFE7DF
:10782800174AE4E703F1080252E8002F42F08052B9
:1078380003F1080040E800210029F3D1002030BD01
:10784800B4F5805F0FD10F4A0F4C002918BF2246AC
:10785800426751B153E8002F42F4907243E8002187
:107868000029F7D1EAE7084AF2E753E8002F42F087
:10787800200243E800210029F7D1DFE785710008DD
:10788800E96F0008256F0008596E0008D0F88C30A1
:10789800202B30B415D1B9B1B2B100230468C36646
:1078A8000A4B9C420AD063681B0207D554E8003F84
:1078B80043F0806344E80035002DF7D130BCFFF772
:1078C8005DBF022030BC70470120FBE7008000400C
:1078D800436E30B52BB90123A0F86A30A0F86830A0
:1078E80030BD0368094D9A689968094C490FC2F37D
:1078F80042626B5C615CDB00B3FBF1F3A0F86A30B9
:10790800AB5CA25CDB00B3FBF2F3E7E740100108D5
:10791800381001087047704770471FB504AB03E97A
:10792800060090F88430012B04463AD0012380F8F1
:1079380084302423C0F8883003681A6822F00102D2
:107948001A609A6822F440120A439A6071B95A6818
:10795800BDF80C009DF80E1022F0100202435A6088
:107968005A6822F07F4242EA01625A601A6842F07D
:1079780001021A60FBF794F86FF07E42034600920A
:107988004FF4800100222046FFF730FE38B920234B
:10799800C4F88830002384F8843004B010BD032074
:1079A800F8E70220F9E790F88430012B0FD0012383
:1079B80080F88430016851E8002F42F0020241E863
:1079C8000023002BF6D180F8843018467047022037
:1079D800704710B590F88430012B044617D0242343
:1079E800C0F8883003681A68196821F00101196025
:1079F80042F000524FF0005141661A60FFF768FFED
:107A08002023C0F88830002084F8840010BD0220AC
:107A1800FCE770B590F88430012B044617D0056850
:107A28002423C0F888302E682B6823F001032B60CC
:107A3800AB6823F060431943A960FFF749FF20238F
:107A48002E60C0F88830002084F8840070BD0220C1
:107A5800FCE770B590F88430012B044617D0056810
:107A68002423C0F888302E682B6823F001032B608C
:107A7800AB6823F060631943A960FFF729FF20234F
:107A88002E60C0F88830002084F8840070BD022081
:107A9800FCE7000038B5084D052455F8043B2BB920
:107AA800013C14F0FF04F8D1204638BDDB68984744
:107AB8000028F5D0F9E700BF2C080020034BD87048
:107AC800034B1B681B6C03B1184770474008002024
:107AD80028080020034B1874034B1B685B6C03B128
:107AE800184770474008002028080020F0B5314D9D
:107AF800314B95F90420314E91B00C46012795F988
:107B080005108DF8047002288DF809208DF80A10E8
:107B180010D18DF80800D8711C7202F09FFD3378DF
:107B280003B114B101A803F003FA254B059A1A60B2
:107B380011B0F0BD59714FF480711A71D9801C725F
:107B480033788DF8087053BB1F2306A88DF81C20C6
:107B58008DF8183002F064FF20238DF8183006A83D
:107B68002B798DF81C3002F05BFF22238DF818303A
:107B780006A86B798DF81C3002F052FF21238DF88E
:107B8800183006A86B798DF81C3002F049FF2923BC
:107B98008DF8183006A80B4B079302F041FF02F04E
:107BA8005DFD012306A88DF818308DF81C3002F011
:107BB80037FFB4E740080020C00000201C08002060
:107BC80020080020000400017FB5092301A88DF8D2
:107BD800043003F0ADF90038044B059A1A6018BF59
:107BE8000120404207B05DF804FB00BF20080020D8
:107BF80070B504460B46134962784A700020A27893
:107C08000A7208701A884A729A788A72DB780B743A
:107C18006368CB600C4B1B68DA6A2AB1237803F0DF
:107C2800FB030A2B00D09047084E052556F8043B65
:107C38001BB15B6A0BB120469847013D15F0FF0563
:107C4800F4D170BDCC000020280800202C080020AA
:107C580070B5044610480123037063784370A37815
:107C68008372E368C360E3780376236943762379F4
:107C780043720A4B1B689B6A03B19847084E052557
:107C880056F8043B1BB19B690BB120469847013D50
:107C980015F0FF05F4D170BDE00000202808002091
:107CA8002C080020014B1868704700BF20080020EE
:107CB80000B58BB0012368468DF8003002F088FDCE
:107CC80038B99DF80400003818BF01200BB05DF8E2
:107CD80004FB0020FAE7000008B501F073FE48B97C
:107CE800FFF7E6FF012806D0054BD879197AFFF788
:107CF800FDFE012008BDBDE80840FFF7CBBE00BF70
:107D0800C00000202DE9F04186B005460E46174612
:107D180001F058FE00287FD101F06CFE044640B9FE
:107D2800FFF7C6FF012807D03D4B197AD879FFF72E
:107D3800DDFE6FF0020462E0DFF8E88088F8086092
:107D4800003E18BF01268DF80460374E68783379F5
:107D58008DF81230694602F0D9FC00283ED08DF823
:107D680004400394ADF810406FF0060495E8030052
:107D78002E4B83E80300337988F80A30394601A886
:107D880003F0DAF92A4B059A1A60112841D801A3A1
:107D980053F820F0FB7D0008217E00081B7E0008B8
:107DA8001B7E00081B7E00081B7E00081B7E000847
:107DB8003B7D00081B7E00081B7E00081B7E000818
:107DC800157E00081B7E00081B7E0008217E000827
:107DD800217E0008217E00080F7E00082B788DF890
:107DE80008306B78ADF810306B6803934FF0FF34B0
:107DF800BCE7104B00221A70E31D18BF144620463A
:107E080006B0BDE8F0816FF00404F8E76FF00504F0
:107E1800F5E74FF0FF34F2E76FF00104EFE700BF3A
:107E2800C0000020E000002040080020F0000020F2
:107E3800200800202408002037B501F0E5FD144D86
:107E4800052455F8043B5BB11B694BB155F8043C5C
:107E58009B682BB1984718B155F8043C1B699847A3
:107E6800013C14F0FF04ECD1FFF714FE68B9094D8A
:107E78002B7853B1084BADF80040D97801942246CD
:107E88006846FFF73FFF00B92C7003B030BD00BF54
:107E98002C080020240800204008002030B58BB0B2
:107EA800054601F08FFD0446002839D1FFF700FF91
:107EB800012838D168468DF8004002F089FC10B1DD
:107EC8004FF0FF3004E09DF80430AB4202D10020AF
:107ED8000BB030BD012DF3D0022D11D0002DF7D1FC
:107EE800002BF4D068468DF8045002F099FD002864
:107EF800E6D10E4B1B681B6B002BE8D09847E6E7D2
:107F0800002BDDD168468DF8045002F089FD002869
:107F1800D6D1064B1B681B6B002BD8D02846EDE743
:107F28006FF00100D4E76FF00200D1E728080020C5
:107F380010B504468AB018B94FF0FF300AB010BD2A
:107F4800002368468DF8003002F042FC0028F3D187
:107F58009DF804302370F1E77FB500220B462049D5
:107F68008DF8072001220A7042784A700446002AD8
:107F780033D102790A721A884A729A788A72DB783F
:107F88000B740369CB60C378164D8DF80830037BFA
:107F98008DF80930836803932B68DB6A0BB102A85C
:107FA80098472B689B6B13B1227E02B198470E4EFF
:107FB800052556F8043B1BB1DB690BB120469847F1
:107FC800013D15F0FF05F4D10DF10700FFF7B0FFF3
:107FD800637913B1054B01221A7004B070BD00BF5C
:107FE800CC000020280800202C08002024080020AD
:107FF80010B504468AB018B94FF0FF300AB010BD6A
:10800800202368468DF8003002F0E2FB0028F3D107
:10801800024A9DF9043023701371EFE740080020ED
:1080280000B58BB02323019068468DF8003002F02C
:10803800F7FC003818BF012040420BB05DF804FB84
:1080480070B5654C01468EB01822204606F0ECF853
:10805800624B00221A70FBF757FF23784068012211
:1080680002FA03F1014004D15D4B084608F0D2F84A
:10807800FEE75C495C481A4602F032F918B14FF045
:10808800FF300EB070BD272304A88DF8103002F021
:10809800C7FC564E564D002870D1012333702B680B
:1080A800DB690BB100209847272304A88DF810300E
:1080B80002F08EFB059B93F84820227093F8182154
:1080C80093F81A316270A370464BD3E9020105F0A8
:1080D8009DFF05460028D2D1464E062304A88DF8F8
:1080E800103002F075FB059B736104A802F098FC40
:1080F800022304A88DF81030059602F069FB0836B3
:10810800032304A88DF81030059602F061FB0F26B2
:1081180006F040F8012304A88DF814308DF810609B
:1081280002F07EFC10230DEB03008DF810308DF863
:10813800145002F075FC04238DF8103004A8A378BD
:108148008DF8143002F06CFC3A238DF8103004A836
:108158006369059302F064FC02A920788DF8086031
:1081680004F0E4F8003818BF0120E0711420FFF78C
:1081780057FFE07903F0A4F9284682E728238DF811
:1081880010302B681B6943B104A802F021FB2B684F
:1081980005981B6940F2C4519847272304A88DF815
:1081A800103002F03DFC50B9012304A88DF81030BE
:1081B80002F00EFB9DF81430002B7FF46EAF33787D
:1081C800002B7FF46CAF052204A88DF810200593CE
:1081D80002F026FC78E700BF4008002024080020B1
:1081E8004810010868080020800800201C080020AA
:1081F800280800200408002037B500230D46019305
:108208000446D0B900F0A8FB0190019BD3B10F4AF6
:1082180042F824300E4A9A620E4A1268916B19632A
:10822800916C596392690C49D9625A6128465B6816
:108238000A49F2229847002006E001A900F092FBC3
:108248000028E2D04FF0FF3003B030BD2C080020EA
:10825800F57A000828080020D17B000810070020C4
:10826800194B07B51860194B194A1A60194A5A6010
:10827800194A9A60194ADA60194B02681A6042680A
:108288005A6082689A60C268DA60164A1A6182691E
:108298005A61154BC26B5A60144A019119609A6071
:1082A8001946134ADA600020FFF7A6FF48B901A86B
:1082B80000F056FB003818BF0120404203B05DF8BB
:1082C80004FB4FF0FF30F9E7280800208008002061
:1082D800597C0008617F000879830008F97B000851
:1082E80068080020E5C2000858080020C57A000880
:1082F800DD7A000851B118B1012804D00020704778
:10830800044B0B607047044B0B60F7E74FF0FF30EE
:10831800704700BF000400010100010208B503F026
:10832800EBF8002814BF6FF00100002008BD08B565
:1083380002F0BCF9002814BF6FF00100002008BD4E
:1083480010B504468AB018B94FF0FF300AB010BD16
:10835800212368468DF8003002F03AFA0028F3D15C
:10836800024A9DF9043023705371EFE7400800205A
:108378002DE9F0412E4D2F4F00232B7043786B7061
:108388003B689B6A8AB004460BB128469847DFF8D9
:10839800A880052658F8043B1BB11B6A0BB1204680
:1083A8009847013E16F0FF06F4D12378052B2FD00D
:1083B8000B2B35D0012B25D1204C062368468DF890
:1083C800003002F005FA0199E07905F065FE10B970
:1083D8001B4B019A5A611B48FFF70AFE1A48FFF720
:1083E800AFFF6B788BB9A371184B5878FFF756FD20
:1083F8003B685B6A0BB1114898476B7813B9E07911
:1084080005F0DAFE0AB0BDE8F081FF23A371EFE7BB
:108418000F4B01225A74227A9A74627ADA74F1E75D
:108428006378002BEED00AB0BDE8F041FFF7CCBB73
:10843800E0000020280800202C080020C0000020B0
:1084480004080020C4000020C500002040080020C7
:10845800CC00002030B58BB0FFF769FF0446F0B9B7
:1084680003F044FF831C1DD0F8B9134D2B685B69DA
:10847800DBB1272368468DF8003002F0A9F92B6894
:1084880001985B694FF4B961984703F041FF78B9E7
:108498002CB9094B1B68DB690BB1012098472046B2
:1084A8000BB030BD6FF00704EFE74FF0FF34ECE797
:1084B8004FF0FF34F3E700BF28080020014B18787D
:1084C800704700BF94080020014B5878704700BFE0
:1084D8009408002070470000044B9A7A0AB10122E0
:1084E8005A70034B5B6903B1184770479408002022
:1084F800FC00002073B5224C6378002B33D008F0C1
:1085080073F966680546FFF7CDFB0644AE4214D200
:10851800A37A93B1E0228DF800208DF80130217AFA
:10852800E368019301226846FFF7ECFB08B10730C6
:1085380010D100236370A372656094F83430EBB1F6
:10854800002384F834300F4B5B6BBBB102B0BDE83D
:108558007040184740F2DC510B4808F011FA0A48FD
:1085680008F0D4F9E8E794F83520002AE5D094F823
:10857800360084F83530FFF791FCDEE702B070BDB5
:1085880094080020FC000020CC08002037B5104DCE
:10859800104CC8B1C1B10123627200222860E160A9
:1085A80023700D480D4B00924FF0FF3108F002F98F
:1085B80000250B4825822022294605F049FE6570D2
:1085C800A574A58603B030BD00232B602370EFE7A8
:1085D8009008002094080020CC080020E1840008BE
:1085E800A80800202DE9F0478E4C23788CB0002B8A
:1085F80056D0C2780AB9837B13B1238A0133238208
:10860800437B002B4CD0E02A4AD10023A372876811
:1086180097F80080B8F1220F27D8B8F1220F30D888
:10862800DFE818F04100FB0052005A0061006E00BC
:1086380075008E009D00B400C7002F002F002F008A
:108648002F002F002F002F002F002F002F002F00AA
:108658002F002F002F002F002F002F002F002F009A
:108668002F002F00C900D000D400B8F17E0F00F011
:10867800CC80B8F17F0F00F0DF80B8F17D0F00F0FB
:10868800AB80A57A002D00F05B81674C637A3BB91B
:108698004FF47A71204608F073F9204608F036F94D
:1086A8000CB0BDE8F087E36801220021A2721970BE
:1086B800A37AE1689818A0720620C854A37AE168E2
:1086C8009818A072CA54DCE7584B9B6A002BD8D084
:1086D800012102209847D4E77B7884F836300123BB
:1086E80084F83530CDE704238DF804307B78003BDF
:1086F80018BF012301A88DF8083002F091F9C0E7EE
:108708007878003818BF012002F0DAFEB9E7484E41
:108718000FCE01AD0FC50FCE0FC596E8070085E84F
:1087280007007B780A2BACD8424A12685268002AA4
:10873800A7D00CA901EB830353F82C0C9047A0E7B2
:108748007878431E012B9CD83A4B01381B6818BF18
:10875800012020729B68002B93D0984791E7E2682C
:1087680001230821A3721170627A057BA17AAA42BB
:1087780028BF2A46934284D285685A1CEB5CE56878
:1087880001334E1CA6726B54D3B2EDE7E3680122A5
:10879800A27209221A70A37AE268218A581CA07270
:1087A800D154A27A238AE1681B0A501CA0728B5408
:1087B80067E7238265E705238DF8043001A802F0F6
:1087C800B7FB5EE7194BDB6A98475AE7194B78788D
:1087D8001B686075DB68BEE7037B072B7FF451AF2E
:1087E80006238DF80430B7F80130ADF808307B79EE
:1087F8003A791B0443EA0223FA7813436422534369
:108808000393BB798DF81030D8E73B2201A88DF887
:1088180004208DF8083002F003F9012384F834307D
:108828002FE700BF94080020CC080020FC0000209F
:108838004C0E0108900800202A2301A88DF8043066
:1088480001F0C6FF94F80A90E6689DF808009DF8C4
:1088580009509DF80A709DF80BC09DF80D309DF8E1
:108868000E209DF80F109DF80CE009F1010A84F81C
:108878000AA006F80980354E94F80A903668D4F8AC
:108888000C8009F1010A84F80AA096F803A008F8F8
:1088980009A094F80A90D4F80C8009F1010A84F828
:1088A8000AA096F802A008F809A094F80A90D4F84B
:1088B8000C8009F1010A84F80AA096F801A008F8CA
:1088C80009A094F80A9009F1010A84F80AA096F818
:1088D8000080E66806F8098094F80A80E66808F1DE
:1088E800010984F80A9006F808C094F80AC0E668F6
:1088F8000CF1010884F80A8006F80C70A77AE6687B
:1089080007F1010C84F80AC0F555A57AE6686F1CD2
:10891800A7727055A07AE568461CA6722954A17AF8
:10892800E0684D1CA5724254A27AE168501CA072FE
:108938008B54A37AE268591CA17202F803E0A0E6FE
:10894800034807F095FF6570AAE600BF900800206D
:10895800CC0800207047000000487047FC00002049
:10896800002070474FF0FF3070470000044B054A65
:1089780093F81831022B18BF062382F890347047F9
:10898800A80E002070140020034BD3F8483313B10D
:108998005B6903B11847704770140020034A1378C5
:1089A80043F004031370FFF7EFBF00BF6C140020FF
:1089B8001FB50A4B8DF8090093F87C208DF80A2022
:1089C80093F88C2093F848000D3202A98DF80820FE
:1089D80003F0ACFCC0B205B05DF804FBA80E0020A3
:1089E80010B5074C04F5806007F042FF94F81A347C
:1089F80013B1012384F81934BDE81040FFF7C4BF50
:108A08007014002010B50C4CD4F8403343F08003A8
:108A1800C4F8403394F81A3413B10020FFF7E0FF8C
:108A280094F8913423F0120343F0120384F891343C
:108A3800BDE81040FFF79ABF701400202DE9F041FF
:108A4800DFF8AC8098F81831022B06460D4602D0A4
:108A5800284BDB6A984702F0E9FD044628B102205A
:108A680002F0DAFD002002F0DCFD98F81831012B45
:108A780017D102F0DDFD074630B1002002F0CDFD30
:108A8800002002F0CFFD3C4602F0D4FD48B10020A2
:108A980002F0C4FD002002F0C6FDBDE8F041FFF77A
:108AA80065BF002CF9D1144C94F8902494F81A342A
:108AB800BAB90BB184F84164304602F065FFD8F8C2
:108AC8002C0007F09BFED4F8B4339842E5D30B484A
:108AD80007F0CEFE94F8913443F0100384F89134F3
:108AE800DBE70BB184F84154284602F04DFFF1E76B
:108AF800A80E0020CC1701087014002008180020C8
:108B080073B5164C164D04F57A76EB6C95F8502033
:108B180095F9781095F84800009603F02DFC95F823
:108B2800303184F8FC3395F8480040F2012304F210
:108B380024423146A4F8FA3303F02AFC58B194F8D9
:108B4800243484F86A34074B00205B6B984794F808
:108B5800FB3384F8903402B070BD00BF701400205D
:108B6800A80E0020CC170108074A10B5137843F067
:108B780002031370FFF708FFBDE81040034B012202
:108B88000021022007F046BB6C1400209110010858
:108B9800074A10B5137843F008031370FFF7F4FE83
:108BA800BDE81040034B01220021022007F032BB30
:108BB8006C140020A11001082DE9F0410F4616465B
:108BC8001D46804607F010FE0B4A0C4C137827818F
:108BD80023F0110343F011031370C4E90008668100
:108BE8002573FFF7D1FEBDE8F041054B01220021B6
:108BF800022007F00FBB00BF6C1400201C1A0020D5
:108C0800B110010813B507F0EFFD0D4B6C46186065
:108C1800204607F03DFD94E803000A4A0A4B83E822
:108C28000300137843F020031370FFF7ADFE074BE2
:108C380001220021022002B0BDE8104007F0EABA84
:108C48002C1A00206C140020A8170020BE10010860
:108C5800F8B5334D95F81841012C06464BD0022C37
:108C680051D064B938B9D5E91B0105F1740383E81B
:108C780003002046F8BD01283DD0022801D0032476
:108C8800F7E7284F85F8180107F5747EBEE80F004E
:108C980007F57A7CACE80F009EE8030095F8E93008
:108CA8008CE8030087F8FB63E3B195F80031022BE9
:108CB80018D1D5F804316B67C7F8EC3395F87D30D7
:108CC80095F8082187F8F83395F88C3085F87820DE
:108CD80087F8F93397F81B2487F8E82340F2013323
:108CE800A7F8FA33002387F81A340F4BDB6A984742
:108CF800FFF706FFBDE702F0A4FC04460028B8D140
:108D080085F81861B5E70028B9D1064B85F8180130
:108D1800062283F89024044BDB6A98473446A8E778
:108D2800A80E002070140020CC1701082DE9F0418E
:108D380092B0064602F07AFC002840F05981AD4D09
:108D480095F81831012B09D02B6BAB4C93B194F8E3
:108D58000431BBB1042B6FD0032003E002F068FCA0
:108D680018B10F2012B0BDE8F08102F063FC0028B2
:108D7800EAD0F6E7B5F82031D4F81C24013B534378
:108D88002B63E4E79D4803F008FA002840F02C81A3
:108D980094F80C3123802B6B0C930DF1180895F87F
:108DA80039308DF83830404695F81C318DF83A3016
:108DB80007F094FCD5F82831009302AF98E8060034
:108DC800D5F82431384607F020FC97E803000FABAC
:108DD80083E80300EB6A0D9300238DF84430238861
:108DE800ADF8463095F8303101228DF839201BB99D
:108DF8008DF844208DF83930814B0093814B95F8DC
:108E08004800A3F179020CA903F005FBC0B10B28B7
:108E1800A8D1D4F8941499B1002EA3D0D4F8403333
:108E2800794843F02003C4F8403307F0A9FD764899
:108E380007F06CFD002095E7704803F0E2F9A4E71D
:108E480095F8487095F9693095F9392095F87D10AD
:108E58006E4E384603F0ECFA009641B2EB6C95F88A
:108E680050203846183603F087FA0096EB6C95F8D0
:108E7800502095F9701095F8480003F07DFAD4F861
:108E8800C413AB6DD4F8DC230B44C4F8B033EB6DDA
:108E98001344C4F8B43394F80431042B07D02B6E70
:108EA8000B44C4F8B0336B6E1344C4F8B4330023D6
:108EB800089395F8303183B108A802F095FC002892
:108EC8004ED195F9390094F837629DF82070FFF774
:108ED8006FFD3E4480B2B04240D300238DF813307A
:108EE80095F839308DF8213095F838308DF82230E2
:108EF800D5F880300993D5F884300A932388ADF8E3
:108F08002C3095F8303194F81B648DF82E3095F894
:108F180048003F4B8DF820600DF1130208A903F0BB
:108F28003FFA012384F8413495F8393084F8423403
:108F38009DF8133084F84334D4F81C34C4F85064D2
:108F4800C4F84834C4F8583402F076FB50B1D4F869
:108F58001C0402F083FB28B1102003E7082001E776
:108F68001320FFE695F81831012B01D102F078FBA8
:108F780002F065FB0023059394F8043195F9395004
:108F880094F81B649BB1042B7FF4E6AE05A802F0AD
:108F980067FE58BB94F8183413B1059B013B059341
:108FA800164B05983246E9B202F0BCFE02E01348BF
:108FB80002F090FEC0B9D4F8403394F80C11218027
:108FC80043F00203C4F8403394F8183411480133CD
:108FD800DBB284F8183484F845340F4B00259B6ABB
:108FE800C4F89854984725E71120BBE61220B9E643
:108FF8000E20B7E6A80E0020701400207815002077
:10900800D80E002004190020D817002028180020A6
:109018008C18002072140020CC170108F0B5504CB1
:10902800504EB4F8DC202287D4E92D0194F8B12001
:1090380084F8692004F16C0282E80300D4E92F0166
:1090480004F1740282E80300B4F8C420A4F87C2078
:1090580091B0D4F8CC20D4F8C810C4F884200025E6
:10906800D4F8D020C4F888200123A4F82031C4F80B
:10907800801084F83051A56284F81B5184F83A5066
:1090880084F81D5184F81E51C4F83451C6F8985418
:10909800A6F8185486F81A54A4F838518DF81830E0
:1090A80004F50973039304F50A7394F84800A4F8C7
:1090B8004651049303A92C4B84F84551C4E94F55F4
:1090C800059303F041F9E36EC6F8D43394F87D3084
:1090D80086F8E03394F88C3086F8E1334FF48073E7
:1090E800A6F8E23386F8D05394F8303186F8E433A2
:1090F80006F574770FCF06F57A740FC497E8030066
:1091080040F2012384E80300A6F8FA33D6F848337E
:1091180086F81B54CDE901551BB15A685B69019269
:109128000293124B0793A3F148020892A3F1140289
:1091380009920F4A0B9229330A93A2F19C030C93CC
:10914800A2F198030D93131D0E9301A902F14C038C
:1091580007A802F599620F9302F05DFA11B0F0BD0D
:10916800A80E0020701400208C190020D8180020A8
:109178008C0F0020F8B50D4F0D4C0E4E0D4607F024
:1091880077FB3B6B984796F8480004F2244229463F
:1091980003F0FEF848B194F8243484F86A34706D0A
:1091A8007B6B9847EB7C84F89034F8BDCC170108AA
:1091B80070140020A80E00200F4890F81B3480F887
:1091C800B8330E4B93F8692080F8BB2393F87D20C1
:1091D80080F8C82393F88C2080F8C92393F830319D
:1091E80080F8CC330022A0F8CA2300F56E7100F590
:1091F8006070FFF7BFBF00BF70140020A80E0020EA
:10920800114890F89034EBB190F81B3480F8D033C3
:109218000E4BDA6EC0F8D42393F87D2080F8E02353
:1092280093F88C2080F8E12393F8303180F8E43308
:109238004FF48072A0F8E22300F5747100F56670AF
:10924800FFF798BF704700BF70140020A80E0020D9
:1092580070B5344C2421204604F0FCFF636A984220
:1092680018BF60624FF01C012F4814BF012500256C
:1092780004F0F0FF636C984218BF60644FF480718B
:109288002A4818BF45F0020504F0E4FFD4F8483135
:10929800984218BFC4F848014FF0D401244818BFB9
:1092A80045F0040504F0D6FFD4F82032984218BFE0
:1092B800C4F820024FF000011E4818BF45F0080509
:1092C80004F0C8FFD4F82432984218BFC4F8240226
:1092D8004FF46071184818BF45F0100504F0BAFF44
:1092E800D4F8A835984218BFC4F8A8054FF014015F
:1092F800124818BF45F0200504F0ACFFD4F8C0357B
:1093080098420F4B18BFC4F8C005D3F8483318BFAC
:1093180045F040052BB11B691BB12846BDE87040DC
:10932800184770BDA80E0020D00E0020F00E0020B7
:10933800F40F0020CC100020D0100020541400207E
:10934800701400202DE9F04F91B04FF00008012B68
:1093580005460F4602928DF81580ADF8188003D89F
:10936800C84EC146B94502D311B0BDE8F08F15F813
:10937800090002F077FA4844B842F5DC15F80930DC
:1093880009F10104023BE4B2112BEDD801A252F815
:1093980023F000BFE593000817940008179500080C
:1093A80041950008C9950008F195000863960008E2
:1093B80095960008119700087193000871930008AA
:1093C8006F97000871930008719300082D980008A2
:1093D8005598000899980008D7980008052002F0C9
:1093E800EDFA90B10521002002F0ACFA2A5DA64BF7
:1093F80009F1030409F102095FFA89F983F85C2489
:1094080015F8092083F85D24E4B2A146AAE70023F1
:109418008DF816308DF817308DF81C308DF8203007
:10942800B8F1000F6CD14FF0050896F87C208DF844
:109438003920631E96F839208DF83B202B4496F886
:1094480038200D938DF83C2096F81A3196F868204C
:109458008DF83D20D6F82C218DF83A300C9273B354
:109468007B1C1B1BDBB28DF8383008AB019307ABB4
:10947800009396F848000DF117030DF116020CA998
:1094880002F09AFF8DF8150000F00700072813D1A5
:1094980096F939209DF9163086F839309A429DF8A8
:1094A800173086F83830B8BF01229DF81C30B8BF95
:1094B80086F81D2186F868304FF0000909E0052379
:1094C800D1E701220DF11501032002F0DBF809F1C3
:1094D80001095FFA89F29DF82030B3FBF8F1914257
:1094E800EFD82344DCB2631EDBB29F420DD9EA5C9D
:1094F800032A9AD0A74288BF1C464FF0010884E788
:1095080009F105095FFA89F4F7E71C46F5E72B5DD1
:10951800012203F00F0309F1020986F81B3102FA50
:1095280003F35FFA89F9A6F82031002206A904207E
:1095380002F0A8F84C4668E707238DF815302B5D34
:1095480096F84800C3F3021203F00F038DF8303089
:1095580009F10303DBB28DF83120EA5C09F1040359
:10956800DBB209F10504EB5C09F102095FFA89F93C
:109578001B0443EA022315F80920134364225343CA
:109588000CA90D9302F027FF00F00703072BE4B2A4
:109598008DF815000CD19DF8303086F8703086F8BB
:1095A80078300D9BF36673679DF8313086F8693023
:1095B8008DF81800012206A9052002F063F824E7B7
:1095C800314BD3F848336BB11B685BB19847029BAA
:1095D8008DF8180003F03F038DF81930022206A910
:1095E8000620EAE7FF20F2E703238DF815302B5D0C
:1095F8008DF824300CAB089309F10303DBB209F1B1
:109608000604EA5C96F8480009F10403DBB208A9ED
:10961800EB5C1B0443EA022309F10202D2B209F10E
:109628000509AA5C1343642253435FFA89F90C9332
:1096380000230D9315F809308DF8383002F0D1FE6B
:10964800C3B20028E4B28DF81530FFF6DEAE8DF80F
:109658001830012206A90720AFE72B5D03F00F039E
:10966800012B4FF47A7238BF0123534309F10209E1
:10967800B36513445FFA89F9F365002206A9082047
:1096880056E700BFA80E0020701400202B5D96F846
:109698004800C3F340128DF81D2007A9C3F3001238
:1096A80003F00F038DF81C208DF81E3002F09FFE8A
:1096B80009F1020901305FFA89F93FF43BAFBDF8BF
:1096C8001C30914AA6F87C309DF81E309DF81C404D
:1096D800D05CF8F79BF90223C6F880000CA996F82D
:1096E80048008DF830308DF8324002F01FFE96F9B0
:1096F8003930089040B29842B8BF184686F8390009
:10970800002206A9092013E703238DF815302B5DE5
:109718008DF8303009F10303DBB209F10504EA5C86
:1097280096F8480009F10403DBB209F10209EB5C81
:109738005FFA89F91B0443EA022315F80920134349
:10974800642253430CA90D9302F057FEC3B20028BC
:10975800E4B28DF81530FFF658AE8DF818300122B6
:1097680006A90A2029E7092002F028F9DFF89CA1B8
:10977800002854D00921002002F0E4F80023ADF8B5
:10978800263009F10203DBB24FF47A71EA5C09F181
:109798000303DBB20DF1300BEB5C1B0443EA02233D
:1097A8002A5D134309F10402D2B209F1060409F152
:1097B8000509AA5C5FFA89F943EA026315F80920EA
:1097C80003934A4312125846ADF8242006F060FF6E
:1097D800039B03F1965303F5A91303F5EC53089380
:1097E800DAF83C3300930DF1200999E80600DAF81D
:1097F80038330AA806F009FF0B9B00939BE8060084
:109808000A9B484606F0E6FE99E8030006F018FFB2
:1098180001F021FF0123E4B28AF83834F5E58AF82B
:109828003804F2E50C2002F0C9F800283FF4EDAD49
:109838000C21002002F086F8344B93F89034043B56
:10984800012B7FF6E2AD01F002FFDEE509F102032C
:10985800DBB22A5DE95C09F10303DBB209F1050417
:10986800EB5C09F104095FFA89F91B0415F8090092
:1098780043EA012313436421594300F00F0001F028
:10988800E7FEE4B28DF81800012206A9112094E63B
:109898000D2002F093F800283FF4B7AD0D21002009
:1098A80002F050F809F10203DBB2194AE85C2B5DBB
:1098B800126809F1040409F103095FFA89F943EA16
:1098C800002015F80910E4B201F0C4FE9DE52A5DF8
:1098D80009F1020309F1040409F10309DBB25FFA93
:1098E80089F9E95C15F809301B0443EA012313439D
:1098F8006420584301F0B0FEE4B28DF8180001224C
:1099080006A9132059E600BFCB10010870140020E7
:109918001C1A00200E4B93F89124920703D593F854
:109928008F24012A08D90B4991F81A2122B18A6A91
:10993800501C18BF01328A620022A3F8182483F849
:109948001A24D3F8402322F00202C3F840237047B8
:1099580070140020A80E002070B5184C184D04F59E
:109968005A7006F085FFD4F84033D4F89804D5F837
:10997800906023F02003C4F8403338B106F03EFF6E
:10998800864203D2002385F83A3070BD0120FFF7E4
:10999800CDF90028F9D00B28F7D095F8393084F89C
:1099A8004234092094F8183484F8453484F8410482
:1099B80001F0EAFFBDE87040FFF7ACBF701400206B
:1099C800A80E0020094BD3F84023012A0AD00849E1
:1099D8000978C90708D43AB993F89204013818BF2E
:1099E8000120704700207047012070477014002044
:1099F8006C140020034BD3F84003431E58425841CF
:109A0800704700BF701400202DE9F04FA9B0EFF3A4
:109A1800108272B6DFF8F4820021D8F80030C8F856
:109A2800001082F31088BA4C002B00F0E480DAB200
:109A38009B06039264D5B74D95F81831022B02D0D6
:109A4800B54BDB6A9847EFF3108972B6B34F06F04F
:109A5800CBFE3E68D4F8B013361A3144B04806F04D
:109A68008FFFAF4806F052FFD4F8B413AD48314425
:109A780006F086FFAB4806F049FF89F3108894F892
:109A88001A34002B00F06D81152312A995F84800AF
:109A98008DF8483002F04AFCD4F8B4130F90014412
:109AA800A14806F06DFFA04806F030FF3B6894F827
:109AB8001B24EB620DAF38468DF870201D9306F01D
:109AC8000DFED5F82831009306AE97E80600D5F8C4
:109AD8002431304606F099FD96E803001FAB83E871
:109AE8000300D4F81C341E9395F8303195F84800DB
:109AF800003B18BF01231CA98DF8713002F01FFC30
:109B0800039BDF064BD5834DDFF820A2D5F8E42070
:109B1800BAF90A30059298F800200493002363F3F9
:109B280000020A9388F8002084F84434049AA4F8C0
:109B3800223484F82534C4F82834A4F82C3484F862
:109B48002E34C4F8303484F82034C4F8343484F81B
:109B58003834C4F83C34704B9AF90C90A4F88C242F
:109B680094F89024DB6A84F88E9484F88F24DAF8C9
:109B78000470BAF80860984794F88F3413B96948A4
:109B880006F076FE3146384601F04EFD8346002841
:109B980000F0EA80049BA4F87E3484F88094039B48
:109BA80019071AD55B4B93F81831022B02D05A4B80
:109BB800DB6A98470220FEF7D9FE84F8410401F0D9
:109BC800E3FE94F81A3413B1012384F8193494F895
:109BD800913443F0100384F89134039B5A0703D55A
:109BE80006210520FEF72AFF039B9B0703D50421C6
:109BF8000320FEF723FF01F035FD94F89124D706E2
:109C08005FD5002384F89234D4F840331E0644BF4D
:109C180023F08203C4F8403312F0050F00F0FC82F1
:109C28000B2001F0CBFE002800F0F68294F8913466
:109C3800DD0700F1F182580740F10883D4F840337A
:109C480023F00203C4F84033D4F8402382BB94F8CD
:109C5800915415F001011EBF2B4662F3000384F8EE
:109C6800913494F891345E0744BF6FF3820384F80B
:109C78009134012384F8923421B1D4F844332C4828
:109C88001B6898476D070BD52A4801F0A3FE01F021
:109C9800D1FE28B194F8913443F0040384F8913448
:109CA80001F0CEFC94F891346FF3041384F89134E6
:109CB800012384F8923494F8913443F0200384F813
:109CC800913494F8913418070AD56FF3C3031A49ED
:109CD80084F89134D4F84433A1F12400DB68984720
:109CE80094F8913499070AD56FF34103124984F81F
:109CF8009134D4F84433A1F16C005B68984794F828
:109D08009034022B1AD1FEF7FBFE17E06C140020EA
:109D180070140020A80E0020CC1701082C1A00206F
:109D2800F017002008180020701800201C1A0020C6
:109D3800B0180020C4180020FC18002094F89134B2
:109D48009A0640F1C6826FF3451384F89134D4F82B
:109D58004033002B40F0BD8229B0BDE8F04FFFF73B
:109D680077BA84F84134A1E695F81821012A0CD174
:109D780001F05EFC804668B1584601F04EFC58463A
:109D880001F050FC042384F88F347EB9012384F851
:109D9800213450E101F04EFC0028F6D0404601F095
:109DA8003DFC404601F03FFC0523ECE73B7804937B
:109DB8005B09013B062B00F21882DFE813F007006D
:109DC800160295001602920016020702102EDDD91F
:109DD80095F830311297F6B28DF84C60002BD5D13A
:109DE8001CA804F04BF912AA1CA9FF2002F0AEF837
:109DF8009DF85830C3F3030307468DF82C3095F8C7
:109E0800480095F87D308DF82D3007220BA902F017
:109E1800A0FA002F5DD100285BD09DF853309DF843
:109E280052201599C5F8E4101B0443EA02239DF853
:109E3800512002201343C5F8E03004F02DF99DF8B5
:109E4800583095F8480085F82E71C3F30212C3F311
:109E5800030385F8703085F878309DF8593085F817
:109E68006920012B38BF01234FF47A725343AB6545
:109E78001344EB650DF15A034FF001081093113E9E
:109E880094F81B348DF83C300FA985F868808DF85C
:109E9800446002F066FA0223404685F8303101F04A
:109EA8008DFD18B14146384601F04CFD94F88F34C9
:109EB800012B00F2A88194F81A34002B40F09B8102
:109EC80094F8913443F0100384F89134FEF74EFD72
:109ED80065E6012001F072FD0028E7D00121072086
:109EE800E2E7012384F8203495F87D308DF82E3090
:109EF80094F824348DF82D3095F88C3095F8480076
:109F08000D330BA98DF82C3002F010FAA6F10D03D1
:109F18001BB2099023EAE37300B283423FF736AFDE
:109F28000B2E7FF633AFBB4B25931CA8FF231C9742
:109F38008DF874608DF8983002F0D4F80746002840
:109F48007FF424AF95F81831012B13D101F070FB81
:109F5800002873D0384601F060FB384601F062FBF8
:109F680004239DF87C101E9884F88F34C1F30011E7
:109F780001F077FB9DF87C301E99C4F8341413F077
:109F88000F0203D09DF89000002863D19DF8980037
:109F9800002862D0002A7FF4F9AE9DF89020002AAC
:109FA8000CBF4FF002084FF0030800220A92D5F8C0
:109FB800EC20914254D195F8E910002950D0D5F8F9
:109FC8000C1195F8EAB009680A9195F81811022958
:109FD80002D1032184F88F14B8F1030F7FF4D6AEB1
:109FE80013F0600F7FF4D2AE0592012795F82E3159
:109FF800BBF1000F37D0BBF1010F38D1012B34D1A1
:10A008006FF0090646FA08F606F00106C6F10206E0
:10A01800F6B2BDF87E100AAA304601F02DFE40B314
:10A0280007280CBF0823012384F821340A9BC4F8AD
:10A038003034C4F86C34FEF7E5FCB0E501F0FAFA08
:10A04800002897D0384601F0E9FA384601F0EBFAD3
:10A05800052386E74FF00008A7E74FF00108A4E7BB
:10A068004FF0010BC2E70426D3E70326D1E701230B
:10A07800DAE71CAB009305990A9B3246584601F073
:10A08800B7FE20B102280CBF0A230B237FE60A9BE8
:10A09800C4F83034C4F86C349DF87C3084F821045A
:10A0A800C3F3401384F82E3484F8443494F88F347E
:10A0B80084F82274012B9EBF0122A86285F81E2114
:10A0C800012FC4F8280484F82C0484F8410438D1FA
:10A0D800022284F8202495F83A20002A4AD19DF8D3
:10A0E8007C20D60646D4012B94F840149DF87C2099
:10A0F80005D8012901D1900601D501F05FFBB8F11F
:10A10800020F94F88F3443D0B8F1030F0AD09DF8AA
:10A118007C10B8F1010F4A4601F00F0120A83BD08E
:10A12800FFF710F99DF8903084F82334259BC4F884
:10A1380028349DF8983084F82C34012384F82D3481
:10A1480030E0049A02F0E002A02A1BD195F82E1103
:10A15800012285F83A2009B927996963012B84F807
:10A16800202407D9D5F89020C4F83C24DAF8002038
:10A17800C4F8982495F81821002AB4D1012284F84B
:10A188002524B0E7002285F83A2084F82024A6E7A1
:10A198009DF8981025984A46FFF7D4F89DF8903016
:10A1A80084F823349DF89020E02A08D195F81F31CF
:10A1B8002BB984F82324C4F82834A4F82C3494F850
:10A1C800913443F0020384F891346FE6114D013E57
:10A1D800B2B2791C284604F027F80323A4F82034E7
:10A1E800C4F8285484F82C64E9E7012384F821345E
:10A1F800FEF708FC5AE694F84434002B3FF460AEAE
:10A208000020FEF7EDFB94F88F34022B3FF45EAE8E
:10A2180056E600BFA816002094F89134590715D5C2
:10A22800012001F0CBFB60B1012001F09DFB08B9D2
:10A2380084F81804D4F8403323F00203C4F84033F8
:10A2480004E0062001F0BAFB0028F3D194F8913419
:10A25800DA077FF5F9AC94F840240AB1032A18D13B
:10A268001D4A94F8181492F86820914205D29B0769
:10A2780023D594F88F34012B1FD8184806F0F8FA24
:10A28800D4F8403323F02003C4F84033FFF742FBEF
:10A29800DAE4012A11D194F81924002A3FF4D4AC45
:10A2A8000D4A94F8181492F868209142E5D29F0755
:10A2B80003D594F84434002BDFD194F8913400206E
:10A2C8006FF3041384F8913484F81904FFF744FBFE
:10A2D800BAE429B0BDE8F08FA80E0020D8170020F6
:10A2E8002DE9F04F89468DB090460746002800F0CA
:10A2F8008F81002900F08C810368002B00F0888191
:10A308004368002B00F084818368002B00F0808173
:10A31800C368002B00F07C81104602F003F8002887
:10A3280000F07881BD4CBE4D384601F0C1FA40F2CC
:10A33800C4520021204603F08BFF40F21C5200213A
:10A34800284603F085FFB74BC4F82C3104F5097390
:10A35800089304F50A7300264046099308A9B24BEE
:10A3680084F848800A9384F8186184F88C608DF822
:10A378002C6001F0E9FF0F2306A994F848008DF836
:10A38800183001F0D3FF801B18BF01204FF00A0BD3
:10A3980084F81C0106A994F848008DF818B001F05B
:10A3A800C5FF4FF0060A84F8DC0006A994F84800B7
:10A3B8008DF818A001F0BAFF102384F8DD0006A973
:10A3C80094F848008DF8183001F0B0FF1123C4F854
:10A3D8009C0006A994F848008DF8183001F0A6FFF3
:10A3E8001223C4F8A00006A994F848008DF8183084
:10A3F80001F09CFF1323C4F8A40006A994F84800B0
:10A408008DF8183001F092FF1423C4F8A80006A9AB
:10A4180094F848008DF8183001F088FF1623C4F826
:10A42800AC0006A994F848008DF8183001F07EFFBA
:10A43800172384F8B10006A994F848008DF818305D
:10A4480001F074FF18230DEB0301C4F8B400C4F83D
:10A45800BC0094F848008DF8183001F067FFC0B2CE
:10A468001D2384F8B80084F8C00006A994F84800B1
:10A478008DF8183001F05AFF1E2384F8C40006A98D
:10A4880094F848008DF8183001F050FF1F2384F825
:10A49800C50006A994F848008DF8183001F046FF69
:10A4A8002023C4F8C80006A994F848008DF818308D
:10A4B80001F03CFF0B23C4F8CC0006A994F848002F
:10A4C8008DF8183001F032FF0C2306A9A4F8D0004B
:10A4D80094F848008DF8183001F028FFD4F89C3023
:10A4E8006365D4F8A030A365D4F8A430E365D4F844
:10A4F800A83023664FF00108D4F8AC300590A4F8D2
:10A50800D200636684F8B080C4F894B084F898A048
:10A51800C4F84CB084F850A084F8688084F81F818F
:10A52800C5F84893FEF77AFD404B009632464FF047
:10A53800FF3105F55A70C5F84473C4E90B6684F811
:10A54800198185F89164C5F8408306F033F9384BD2
:10A55800009632464FF0FF3105F5607006F02AF993
:10A56800344B009632464FF0FF3105F5667006F021
:10A5780021F902AF304B009632464FF0FF3105F516
:10A58800806006F017F9384606F0A8F897E8030047
:10A5980004F5927383E80300284B294F1E60294B6A
:10A5A800C5F84C33284BC5F85433284BC5F85C33F1
:10A5B800274BC5F85033274BC5F8583305F553706A
:10A5C8003B68984704F5A67003F084FB20B1112678
:10A5D80030460DB0BDE8F08F204601F01DFB002885
:10A5E800F5D101F041F8B8B91B4801F067FB064600
:10A5F8000028ECD17B69984703F0F4FDBB6D94F813
:10A6080019019847FB6A9847012385F89234DFE7D8
:10A618000326DDE70926DBE71326D9E7A80E002085
:10A6280070140020000400018C19002061990008B2
:10A63800C191000809920008E98900086C140020FB
:10A64800CC1701080D8C0008C18B0008A5890008EB
:10A65800998B0008718B0008900F002008B5034BF8
:10A668000020C3F84003FEF781F908BD70140020EC
:10A6780010B5FFF7A7F90A4C60B90A4B93F81831DF
:10A68800022B02D1084BDB6A98470123C4F84033F8
:10A69800002010BDD4F84003013818BF0120F8E7A6
:10A6A80070140020A80E0020CC17010838B5134CF0
:10A6B80004F55A7006F0DCF804F5607006F0D8F876
:10A6C80004F5667006F0D4F804F5806006F0D0F85A
:10A6D80000F0B5FF0A4B0025DB6A9847C4F84053E1
:10A6E800FEF7B6FD0749084840F2C45203F09CFD46
:10A6F8000123C4F84033284638BD00BF7014002039
:10A70800CC170108A80E0020E408002070B52E4BD5
:10A718008AB0054693F8DD008DF8090093F8DC004F
:10A728008DF80A0029489A6A90F8180403920026BE
:10A738008DF80B0004960C46002940D00692D3F8F9
:10A74800882007921A8F93F81A118DF8151052BAAB
:10A75800ADF8202093F87C2093F848308DF8243009
:10A7680003AB8DF822008DF8232000930DF10A0227
:10A778000DF10B030DF1090105A88DF8146000F027
:10A78800DDFE9DF90900FEF713F9607004A801F0D9
:10A798002BF8B0B9049A0F2A0DD863789A420AD8D0
:10A7A8001544AB42A3EB02012CBF0020012021700D
:10A7B800C0000AB070BD002323700820F9E7032009
:10A7C800F7E71320F5E700BFA80E0020701400205B
:10A7D8001FB50446002800F012810078412800F2D5
:10A7E8000881DFE810F0420048004D005200560092
:10A7F8005A005F000601060106010601060106016E
:10A808000601060166006A006E0079008000830078
:10A8180086008B0089008D009100940097009A00B3
:10A828009D00A000AF00B300BB00B700BF00C2008E
:10A83800C600CF00CB00CD000601D30006010601FB
:10A8480006010601060106010601060106010601C8
:10A8580006010601060106010601DB00DF00E30030
:10A86800E800EC00F000F400FD00674B93F81831A5
:10A87800237104B010BD644B93F83031237102E0AA
:10A88800606803F0B5FB0020F3E7606803F0F6FBAF
:10A89800F9E75D4B93F81A31F0E75B4BD3F8E030FA
:10A8A8006360F0E7584B211D93F8300103F0FEFB7D
:10A8B800E9E7554B93F81931E0E7534B93F88C309F
:10A8C800DCE71C238DF808304F4B02A993F84800A9
:10A8D80001F02CFD6060D6E74C4B043493E803008C
:10A8E80084E80300CFE74A4B0434F7E7494B0434C4
:10A8F800F4E7494B0434F1E71A23E3E71923E1E7C6
:10A90800414B93F86830B9E73F4B5B6DC8E73E4B66
:10A918009B6DC5E73C4BDB6DC2E73B4B1B6EBFE74E
:10A92800394B5B6EBCE702238DF80830364B02A921
:10A9380093F87C2093F848008DF80A2001F0F6FC83
:10A948002071A0E7304B93F8DD3097E72E4B93F852
:10A95800393093E72C4B93F8DC308FE72A4B93F888
:10A9680038308BE7284BDB6C9AE7274B93F850304D
:10A9780084E7254BD3F88430636084E7224B8FE764
:10A98800264B8DE7204BD3F8CC30F5E71E4BD3F898
:10A998002C31636001F058FDA06074E71A4BD3F8BE
:10A9A80090307DE7184B93F81F3167E7164BB3F8E3
:10A9B8008830A38067E7144BB3F88A30F9E7124B65
:10A9C800B3F8D030F5E7104BB3F8D230F1E70E4BBF
:10A9D80093F848200AB1062A13D1B3F8A035E8E75E
:10A9E800094B93F848200AB1062A0AD1D3F8A435AE
:10A9F80056E7204604B0BDE8104000F024BE03200E
:10AA080037E7182035E700BFA80E0020140F0020F4
:10AA18005C0F00201C0F0020640F0020E4080020B9
:10AA28007FB5044610B9032004B070BDA44DD5F815
:10AA380040339A0700F171820278412A00F26A8253
:10AA4800DFE812F04200480056005C006000650034
:10AA58006A007700820088008E0094009A00A000A7
:10AA6800A600AC00B6006802BB00DD00F0001701CC
:10AA780039012A0144014D015101550159015D0176
:10AA88006802610173019B018901AD01B301BA013B
:10AA9800BF01C40168022A026802680268026802EB
:10AAA800680268026802680268026802680268024E
:10AAB800680268026802680236023B0240024502E8
:10AAC8004A024F0254025E020079FEF7C1F80028DC
:10AAD800AAD105E00379022BA5D07A4A82F8303151
:10AAE80095F8913443F0200385F8913400209BE7D2
:10AAF800406803F06FFA0028F2D094E7406803F04A
:10AB0800ADFAF8E76F4B027983F81A21E8E76D4B45
:10AB18004268C3F8E020E3E76A4E416896F83001DE
:10AB280003F0BAFA00287FF47EAF6368C6F8E43011
:10AB3800D6E7416800293FF476AF002001F0EAF932
:10AB48000028CDD011206FE7416800293FF46BAF92
:10AB58000120F3E7416800293FF465AF0820EDE7DD
:10AB6800416800293FF45FAF0920E7E74168002901
:10AB78003FF459AF0C20E1E7416800293FF453AF97
:10AB88000D20DBE7416800293FF44DAF0E20D5E7E3
:10AB9800416800293FF447AF0F20CFE74A4C494BA3
:10ABA800007983F81901A36D9847E36A984797E7F6
:10ABB800444B027983F88C2092E7424E037A8DF851
:10ABC800043096F8480096F87D308DF80530072255
:10ABD80001A901F0BEFB00283FF425AF636896F891
:10ABE80048000193002201A901F0B3FB00283FF4BB
:10ABF8001AAF6C36D4E9010186E8030070E7314EDC
:10AC0800037A8DF8043096F8480096F87D308DF870
:10AC18000530072201A901F09CFB00283FF403AF8F
:10AC2800B436E7E7274E037A8DF8043096F84800E3
:10AC380096F87D308DF80530072201A901F089FBCF
:10AC480000283FF4F0AED4E9010106F1740383E86B
:10AC5800030096F81831022B7FF442AF96F8303192
:10AC6800002B3FF43DAF184BDB6A9847FDF748FFD0
:10AC780036E7144E037A8DF8043096F8480096F8B3
:10AC88007D308DF80530072201A901F062FB00280C
:10AC98003FF4C9AEBC36ADE74368029301238DF893
:10ACA8000C30084B02A993F8480001F05FFB00281C
:10ACB8007FF416AFB7E6436802930023EFE700BFBF
:10ACC80070140020A80E0020CC17010803795A1E22
:10ACD8000E2A3FF6A8AE934A82F8683000E7914BF7
:10ACE80042685A65FCE68F4B42689A65F8E68D4BD8
:10ACF8004268DA65F4E68B4B42681A66F0E6894BDF
:10AD080042685A66ECE6874C037994F848008DF857
:10AD18000430062201A901F01CFB00283FF483AE91
:10AD28009DF8043084F8DD30DAE67E4C03798DF83E
:10AD3800043094F8480094F87C308DF806300522E9
:10AD480001A901F006FB00283FF46DAE9DF8043020
:10AD580084F83930C4E6734C037994F848008DF8C8
:10AD680004300A2201A901F0F4FA00283FF45BAE8E
:10AD78009DF8043084F8DC30B2E66A4C037994F824
:10AD880048008DF80430092201A901F0E2FA0028F0
:10AD98003FF449AE9DF8043084F83830A0E6614BA2
:10ADA8004268C3F89420DA649AE65E4B027983F825
:10ADB800982083F8502093E65A4B4268C3F88420C1
:10ADC8008EE6584B4268C3F8CC2089E6012B40F048
:10ADD800A480554C2421204603F03CFA636A98422B
:10ADE80001D0172020E61C2104F1280003F032FAD4
:10ADF800636C9842F5D14FF4807104F1480003F078
:10AE080029FAD4F848319842EBD1D42104F5A67038
:10AE180003F020FAD4F820329842E2D1002104F558
:10AE2800097003F017FAD4F824329842D9D14FF4B4
:10AE3800607104F50A7003F00DFAD4F8A835984249
:10AE4800CFD1142104F2AC5003F004FAD4F8C03581
:10AE58009842C6D1334E2146304640F2C45203F0E0
:10AE6800E3F9204640F2C452002103F0F1F995F8C5
:10AE78001B3485F8E833736FC5F8EC3396F87D30EA
:10AE880085F8F83340F20123A5F8FA33274B96F8F2
:10AE980019019B6D984723E68379012B3FF6C3ADD3
:10AEA800204B42684068C3F82C2100F0D1FE47E6E9
:10AEB8001C4B4268C3F8902012E61A4B027983F8BB
:10AEC8001F210DE6174B8288A3F8882008E6154B4A
:10AED8008288A3F88A2003E6124B8288A3F8D02040
:10AEE800FEE5104B8288A3F8D220F9E50D4B93F8C4
:10AEF80048200AB1062A12D1A288A3F8A025EFE5B6
:10AF0800084B93F848200AB1062A08D16268C3F8AA
:10AF1800A425E5E500F099FBD9E5012084E5182092
:10AF280082E500BFA80E0020E4080020CC17010825
:10AF38002DE9F04387B00023ADF80030064600281D
:10AF480000F0ED800361FEF73DFD20B101242046AD
:10AF580007B0BDE8F08300F073FD0028F6D100F0DB
:10AF680069FD014618B96F48142203F071F96E4D56
:10AF780095F89134012243F0040385F8552485F8A7
:10AF8800913433788DF804300021013B8DF8052089
:10AF9800ADF806100C2B00F2BA80DFE803F007B812
:10AFA800B8B87881B8B88FB8AC99A800D5F840730C
:10AFB80017F02007CAD196F80480B8F1020F45D1DE
:10AFC800DFF868815A4CFEF729F896F9051098F8C9
:10AFD80048003A4601F017FA88F83900B37988F83A
:10AFE8003830384607238DF80530FDF731FEFF234A
:10AFF80004F58670A5F80C31C5F8084185F8047188
:10B0080003F03CF804F58A7002F0F2FF3846FDF7C9
:10B018008DFE044640B196F9051098F848000122C3
:10B0280001F0F1F988F83900D5F894343361002C2F
:10B0380071D000F0FFFC002889D195F8913485F88B
:10B048001A0460F3820385F8913480E7B8F1010FA0
:10B058004FF00204E8D1DFF8D4908DF8144099F845
:10B06800480089F81D7102A901F06EF9337989F851
:10B0780030318DF805708DF80680FDF785FC95F860
:10B08800913443F0100385F891340024CCE7002272
:10B098006946022000F0F6FA0028F6D01324C3E728
:10B0A800244BB288DB6B96F90C10B0689847D5F83A
:10B0B800403343F00203C5F84033E6E702A90D2008
:10B0C80000F060FB0028E0D0002269460D20E1E78F
:10B0D800164B93F81831D3B9347904F0070000F00F
:10B0E800ADFA8DF80040012269461020D2E700220F
:10B0F80069461220CEE78DF8072000F090FA044642
:10B1080038B900F089FA204600F08BFA8CE702245F
:10B118008AE7012488E701A800F0DEFB17E703248B
:10B1280015E700BFC418002070140020A80E0020E6
:10B1380072140020CC1701082DE9F04F99B0804611
:10B14800059118B9032019B0BDE8F08F00230361F9
:10B15800FEF738FC0646002840F0AB8045460FCD88
:10B168000EAC0FC45A4C98F800A0B8F80C7098F9B7
:10B178000EB0142204F58860314603F069F8012204
:10B1880084F84124534C94F83021022A35460BD1D7
:10B1980094F81821022A07D194F81E2122B9BAF18D
:10B1A800010F38BF4FF0010ABAF1010F2DD0BAF1E3
:10B1B800030F2CD0BAF1000F35D102229DF83C3094
:10B1C800DDF84090029362F34715012694F87C104D
:10B1D8008DF8321002220CA994F848008DF830201E
:10B1E80001F0A4F894F81A3194F830C194F81D11BC
:10B1F80040B20222002B6FD0BCF1010F65D10029AB
:10B2080063D1002E6DD1104627E00422D6E7002333
:10B21800DDF83C90BDF840709DF942B0029365F0AE
:10B228001F050126D2E74FF0000BD946CDF808B02C
:10B23800CCE74FF0010084F81A04DDE005F29A42E9
:10B248000BA900F0DDFA002800F020811320049BF0
:10B2580033871F4B002283F81A241D4BD3F89434EC
:10B26800C8F810306FE705F29A452A460BA900F096
:10B27800C7FA0028EAD10B9B84F82801C4F82C519E
:10B2880084F8303102E1B9F1000F00F0FF80002AA4
:10B2980000F0FC804946E01C02F0C6FF94F8373203
:10B2A80001332380F2E01220D1E70220CFE7072004
:10B2B800CFE7012047E7064B93F8912483F840A491
:10B2C80042F0010283F89124C7E7EEB90220C4E7EF
:10B2D80070140020A80E0020002E94D05845B8BF46
:10B2E800584694F87C308DF82000052294F84800E0
:10B2F8008DF8223008A901F02CF800283FF422AF7D
:10B308009DF8203084F83930694A6A4BD2F898049D
:10B31800D3F8904038B105F071FA664B84423CBFCF
:10B32800002283F83A20198F1A8F93F8300104917C
:10B33800996A099152BA0028B9D093F81B0100B94B
:10B34800186393F81801ADF85820013893F87C2059
:10B3580093F81A411491D0F1000BD3F888108DF8A6
:10B368005B204BEB000B93F8482093F83A0093F8D6
:10B3780068308DF85A3009AB00934F4B03904FF06B
:10B3880001008DF84C0015918DF85C20A3F12F0178
:10B39800A3F1300213A88DF84D4000F0CFF8039BBD
:10B3A8004FEA0B1B4BEA431B00264BEA801B4BEA78
:10B3B800C413B1453E4C039308BF37463A46494645
:10B3C80004F59C70CDE90A669B46268084F81A64C9
:10B3D80002F02AFFE9B2A570C5F34215FAB2042DAE
:10B3E800344E039B84F837223FF423AF072D3FF4F4
:10B3F8004AAF022D7FF459AF304D84F80D11042067
:10B40800029984F80401FF2084F80C0184F82811BB
:10B4180084F81431D6F8E410C4F8085105F59B7384
:10B428000AA8C4F8101184F83021C4F82C3100F0AF
:10B4380017FC00287FF437AF0A9BA4F844040BA834
:10B44800A4F81631C4F84C3400F0CEF900287FF483
:10B45800FDAE0B9BD3B196F93900FDF7A9FA94F824
:10B468003732002B3FF4FFAE0B9B0F2B3FF6E6AEB7
:10B4780005F58B720BA90F2000F0C2F900287FF4A4
:10B48800E5AE0B9B63F3030B84F814B10598FDF745
:10B498004DFC00287FF4DBAE099B86F83A00B362C6
:10B4A80000F07EF900283FF406AF1320D1E600BF74
:10B4B80070140020A80E0020100F00207214002025
:10B4C80037B50B4D8DF8040004460F2295F8480057
:10B4D80001A900F03EFF40B1064A85F81C4192F8E8
:10B4E800913443F0200382F8913403B030BD00BF9B
:10B4F800A80E00207014002010B5FFF7B9F8044614
:10B5080088B90A4805F0B4F9094805F0B1F90948BD
:10B5180005F0AEF900F093F8FDF780FD064BDB6A05
:10B528009847204610BD0124FBE700BFD81700202C
:10B53800F017002008180020CC1701082DE9F04F5B
:10B548008BB047780093149B90F90C8090F90D60AC
:10B5580090F80E908B464168196004469246002F79
:10B5680057D002238DF8103004A9C37B007C8DF8D6
:10B57800123000F0DBFEB4F808C0618943B260689D
:10B58800984545466144B8BF1D46604534BF00270D
:10B598000127884209D30A218DF81010207C0193D5
:10B5A80004A900F0C3FE019B46B2B4F808C0608944
:10B5B80061680CEB400E714520D3A1EB0C01B1FB87
:10B5C800F0FC00FB1C11C9B998450ADC237833B19B
:10B5D8000223207C8DF8243006A900F0B5FE4FF038
:10B5E800010921238DF81030207CE37B8DF8115060
:10B5F80004A98DF8123000F099FE45B2009B8BF833
:10B60800005038468AF8006083F800900BB0BDE817
:10B61800F08F4546F2E77047704770477047002043
:10B628007047704770477047002070470020704788
:10B63800002070470020704700207047704770470F
:10B6480070470220704702207047022070477047F9
:10B6580000207047704770470020704700207047EF
:10B66800704770477047000010B5054C4FF40372DF
:10B678002046002102F0ECFD0020C4E9000010BDC6
:10B68800301A00202DE9F8438146174600293FD09B
:10B69800244B002503F1010C1A462801103312F837
:10B6A800018FB8F1000F36D19A42F8D11E4E336897
:10B6B8000BB9C6F800C073680BB1C3F800C03318E3
:10B6C800002401359C6083F80C900D302B01BAB230
:10B6D80006EB05153044F750C6F804C002F0A4FD87
:10B6E800B9F1110F4FF0000398BF104C6B71D6F8E9
:10B6F800083298BF24FA09F403F1010398BF04F053
:10B7080001043B442C71C6F808324046BDE8F88372
:10B718004FF00108F9E70135202DBBD14FF00208A1
:10B72800F3E700BF371A0020301A00202007020074
:10B7380010B510B3124A1368984204D10368136015
:10B74800002304E00B4613B119688842FAD1516806
:10B75800884208BF53600BB101681960D2F80832FB
:10B768008168013B00245B1A04602146C2F8083254
:10B77800102202F06DFD204610BD0120FCE700BF3D
:10B78800301A0020054B1B6813B11A798242FAD18E
:10B79800002B0B600CBF032000207047301A0020DC
:10B7A80010B5054B186800B910BD037B04680BB9C8
:10B7B800FFF7BEFF2046F6E7301A002038B5084BE1
:10B7C800084C186800B938BD03790568112B05D8ED
:10B7D80024FA03F3DB0701D5FFF7AAFF2846F1E7B0
:10B7E800301A00202007020028B1044BD3F8083291
:10B7F8000360002070470120704700BF301A002006
:10B808002DE9F04107460E4615463AB331B3144BBD
:10B818001C6800232CB93046FFF7E6FF0020BDE87E
:10B82800F081A268F91A0132914210D32279EA54C0
:10B83800581C22895FFA80F8611D55FA80F002F0E1
:10B84800F3FCA368246898445FFA88F3E2E720468B
:10B858002468FFF76DFF002CF9D1DCE70120DEE753
:10B86800301A00200238C0B211289ABF014B185C68
:10B8780000207047DB10010830B50B4B93F82020EF
:10B888000446084672B100211C330578A54208D049
:10B8980001319842CDB20CBF04480430AA42F4D812
:10B8A800002030BD1046FCE73C1C0020481C00204E
:10B8B80010B5084C00232060142204F10C00FF216D
:10B8C80084F82030C4E9010002F0C2FC012384F8A6
:10B8D800213010BD3C1C002010B50E4A92F82010F3
:10B8E800042915D8936804781C7044785C70C4786F
:10B8F800807898700131DC7082F8201002F11C0108
:10B908008B4214BF043302F10C039360012010BD75
:10B918000020FCE73C1C0020094B93F8200068B18C
:10B928005A6803F11C018A4200F1FF3014BF043247
:10B9380003F10C0283F820005A600120704700BF11
:10B948003C1C002010B5074B93F8202004460846FD
:10B9580032B15968FFF790FF10B10123447083702A
:10B9680010BD00BF3C1C002008B5064B93F82020F2
:10B978002AB15968FFF780FF08B1407808BD012057
:10B98800FCE700BF3C1C002030B50A4A92F82010A2
:10B99800536882F8210061B1916801241C32DD7876
:10B9A800587005B99C7093420CBF034B04339942FD
:10B9B800F5D130BD3C1C0020481C002008B5044BC4
:10B9C8005968FFF759FF003818BF012008BD00BFAC
:10B9D8003C1C00202DE9F3410422154E04460021A9
:10B9E8000DEB020096F8208002F032FC0025EBB245
:10B9F800984502D802B0BDE8F081736819782170C3
:10BA08005A7862709F785FB1336820469B68984780
:10BA1800FFF782FF17B901A8FFF75EFF0135E6E7D8
:10BA2800DB788DF804108DF805208DF80730EFE7E6
:10BA38003C1C0020014B93F8200070473C1C002060
:10BA4800034B93F82000042894BF0020012070477E
:10BA58003C1C00201FB50024CDE90244C41F8DF80A
:10BA680000408DF801100C0AADF80420090C120CE6
:10BA78008DF803108DF806208DF8073002461B0A52
:10BA8800012168468DF802408DF8083002F04BFA23
:10BA9800002818BF0E2004B010BD2DE9F04188B071
:10BAA80017460D460F9A064600284DD0002401215E
:10BAB800CDE904448DF810109DF838108DF8151054
:10BAC800ADF81630190CCDE900441B0ECDE902443F
:10BAD8008DF81930ADF81A20130C120E07948DF852
:10BAE80018108DF81C308DF81D20E3B24FEA0318AA
:10BAF800002D5FFA88F803DC002008B0BDE8F0816B
:10BB0800013310218DF81F303A466B460DEB0100CA
:10BB180002F09FF90346C8B9102DAC46A8BF4FF0F4
:10BB2800100CDAB2624503F1010303DB103D2DB2BC
:10BB38000134DAE708EB020020326A44315C12F87B
:10BB4800202C4A403254ECE70920D6E70E20D4E7EF
:10BB58000138032815D8DFE800F002080C100A4B5A
:10BB68001B681B690B6000207047074B1B685B69EB
:10BB7800F8E7054B1B689B69F4E7034B1B68DB6917
:10BB8800F0E70520704700BF601C00202DE9F04158
:10BB9800C4B00C464A9E17461D468046B8B3B1F558
:10BBA800807F36D84FF488720021684602F050FB37
:10BBB800492300934FF48073ADF804302B0C8DF8B3
:10BBC8000830330CADF80650ADF80A608DF80C302B
:10BBD80022460023414604A82D0E360E8DF80E305D
:10BBE8008DF809508DF80D608DF80F4002F01CFBA0
:10BBF80004F110014B9A3B4689B2684602F013F9EA
:10BC080010B1012818BF0E2044B0BDE8F08109200A
:10BC1800FAE70D20F8E7000010B590B10A4C282289
:10BC28000021206002F014FB2368084A1A600020F3
:10BC38004FF0FF32C3E90302C3E90522C3E9072233
:10BC480010BD0820FCE700BF601C002000010101B6
:10BC5800024B1B6818600020704700BF601C002062
:10BC680030B1044B1B68DB68013303600020704768
:10BC780009207047601C002013B500230C4601936F
:10BC8800D2B101A9FFF764FF18B9019B591C02D171
:10BC9800146002B010BD99B2611A002902DD0B448C
:10BCA8001360F6E702D113600720F2E71B0C1B04B0
:10BCB80003F580332344F3E70920EAE728B1044B6E
:10BCC8001B681C334362002070470920704700BF7F
:10BCD800601C002013B50446D8B1114B1A6893882C
:10BCE80001339BB29380C38200F057FA98B904F1EC
:10BCF8001803009321680123132202F08BF860B91E
:10BD0800204600F04AFA003818BF0120000102B0AE
:10BD180010BD0920FBE71020F9E70E20F7E700BF68
:10BD2800601C0020F0B5054687B01C463BB32F4E7B
:10BD38003368DB68834257D894F82020002A14BF60
:10BD480009220822834205D3204600F05AFA70B12E
:10BD580010200AE0002301900093A36894F82810AB
:10BD6800606AFFF79AFE0028EED007B0F0BD23798D
:10BD78002168B4F808C0A768043B9AB209B9092039
:10BD8800F3E7B2F5807F2DD8ADF80EC08DF81730E7
:10BD98004FEA174C04F12C033F0E8DF811700093F5
:10BDA8002F0C08234FF0490EADF80C008DF81470D5
:10BDB8008DF816002F0E0DEB0300CDF808E08DF876
:10BDC80010C0ADF812508DF8157002F023F808B1C4
:10BDD8000E20CAE7204600F014FA0028B8D13368CC
:10BDE800DD60C2E70D20C0E70620BEE7601C00202A
:10BDF8002DE9FF410A9D80460F4616461C46002D38
:10BE08005AD0002303A910460393FFF7A1FE18B1E7
:10BE1800062004B0BDE8F081039B9C4201D80133A1
:10BE2800F6D1284600F05EF9002847D1264B1A784B
:10BE3800424503D01A79424542D10120AA68BA4244
:10BE480040D103EB8002EB6A92F801802979CDE9B1
:10BE580000430439927828683B4689B2FFF796FE7A
:10BE68000028D6D195F820300194002B4FF001031B
:10BE7800009314BF4246082295F82810686A3B468A
:10BE8800FFF70BFE0028C4D1013E032EC1D8DFE81E
:10BE980006F002070B0F0D4B1B681C611C62B8E70C
:10BEA8000A4B1B685C61F9E7084B1B689C61F5E766
:10BEB800064B1B68DC61ACE70920AAE70F20A8E75E
:10BEC8000B20A6E70220A4E734010020601C002014
:10BED8001FB50A460B2A4FF00001CDE90011CDE944
:10BEE800021107D00C2A13D00A2A0FD00A2005B055
:10BEF8005DF804FB012802D120238DF80030684644
:10BF080002F011F8002818BF0E20F0E73023F4E7FC
:10BF18000B21F4E738B5054602F000F8044678B975
:10BF28007DB9094B1B680B219878FFF7D1FF38B909
:10BF38000C21FFF7CDFF18B90A21FFF7C9FF00B19F
:10BF48000E24204638BD00BF601C00202DE9F043B8
:10BF580080468FB00C461746002A6BD0002969D05E
:10BF6800002529461D2206A8059504F093FE8DF8A4
:10BF78001350344D2B680DF114099E88CDF80490A8
:10BF88000DF1130302933B7900933B683246214637
:10BF9800404601F0E4FF00284ED138683A79494616
:10BFA80002F042F9384600F04FF8002846D13C7AB2
:10BFB800FA79BB79240444EA02241C432B689A6862
:10BFC80094423DD99C609DF813000B21FFF780FF38
:10BFD800034658BB0C21FFF77BFF034630BB0A2101
:10BFE800FFF776FF034608BB7B7ABA7AFF7A3F04ED
:10BFF80047EA02271F433A46334621460920FFF7FE
:10C0080029FD034690B933463A4621460820FFF7F2
:10C0180021FD034650B92A689DF81310917000213C
:10C02800D1604FF0FF31C2E90411916118460FB099
:10C03800BDE8F0830923F9E70E23F7E70F23F5E7B7
:10C048000323F3E7601C002010B50446002845D000
:10C058000168002942D011F8013B437103220630E0
:10C0680002F0E2F82046032250F8091B043102F0DE
:10C07800DBF82168CB79E3600A7A43EA0223E360BC
:10C088004A7A43EA0243E3608A7A43EA0263E36056
:10C09800CB7A23740B7B63742379212B1AD110225A
:10C0A8000D3104F1120002F0BFF81D222168501C66
:10C0B8008B5C6362085C43EA0023901C6362085C43
:10C0C800033243EA004363628A5C43EA02636362C1
:10C0D800002010BD112B03DC0D22E7E70220F8E752
:10C0E8000120F6E710B50446002854D0016800295D
:10C0F80051D00B7843714B7883608A7843EA0223E6
:10C108008360CA7843EA024383600A7943EA026398
:10C1180083604B7903738B79C381CA7943EA02231D
:10C12800027BC38102F00F020831103002F07CF864
:10C13800237B002203F00F0384F8202084F82820B2
:10C14800227903F10800111A04290DDD2168093349
:10C15800043AD21A085C84F82000D2B2606A84F8E3
:10C168002820194402F060F8237922681A44002034
:10C1780012F8043CE36212F8031C43EA0123E36269
:10C1880012F8021C43EA0143E36212F8012C43EA65
:10C198000263E36210BD0220FCE710B5044660B3F9
:10C1A800036853B30279162A29D942791A700146CD
:10C1B800082251F8060B013002F040F82146082207
:10C1C80051F80E0B093002F039F82368E28A5A74E4
:10C1D800E38A22681B0A93742368A269DA74A36944
:10C1E80022681B0A13752368628B5A752368E27EDE
:10C1F8009A7517232371002010BD0120FCE7022047
:10C20800FAE738B50446002863D00168002960D0F1
:10C21800037B90F8282003F00F03002A57D1083336
:10C22800207904321344984255D363790B702368FC
:10C23800A2685A70A36822681B0A937023686289EF
:10C24800DA702368E27A1A712368227B5A712368AC
:10C25800E2899A71E38922681B0A2146D371227BFD
:10C2680051F8100B02F00F02083001F0DDFF237BBC
:10C2780094F8282003F00F0303F108052AB1226877
:10C2880094F82010515503F10905206894F82820E6
:10C29800616A284401F0C8FF94F828302268E16AEE
:10C2A8002B44D1545A1CE16A206892B2090A81547D
:10C2B8009A1C2168E08D92B28854DA1C216894F89F
:10C2C8002F0092B2043388542371002038BD0933FB
:10C2D800A6E70120FAE70220F8E70000024B1A88D7
:10C2E80010431880704700BF641C002008B5074B36
:10C2F8001B883BB1FEF7BCF900280CBF00206FF08B
:10C30800020008BD6FF00100FBE700BF641C0020BD
:10C3180010B5034B00241C80FEF7A0F9204610BD81
:10C32800641C0020B0FA80F04009704782B018B948
:10C33800084602B000F0CAB8002002B0704710B931
:10C34800084600F077B9704710B9084600F08EB972
:10C3580070470346084611460BB900F0E5B90020BE
:10C36800704710B9084600F071BD704710B908460B
:10C3780000F006BA0020704710B40446084611467B
:10C388001A46019B14B910BC00F018BA10BC7047CB
:10C398000346084611460BB900F042BA0020704720
:10C3A80010B40446084611461A4614B910BC00F0E9
:10C3B800AFBA002010BC704730B405460846114695
:10C3C8001A46DDE902341DB9029430BC00F02EBBD8
:10C3D800002030BC704710B9084600F0DFBB0020D1
:10C3E800704710B9084600F06FBD0020704710B9BB
:10C3F800084600F0EEBB0020704710B9084600F070
:10C40800EBBB002070470346084611460BB900F005
:10C4180005BC0020704710B40446084611461A4669
:10C42800019B14B910BC00F0FBBB092010BC70477D
:10C4380010B40446084611461A4614B910BC00F058
:10C4480063BDC8B210BC70470048704701000102C4
:10C45800064B10B51B6A0446984730B10448054B93
:10C46800204498428CBF0020012010BDCC17010841
:10C4780040C220C980B92A00F0B5114B85B00C46DE
:10C4880010491F56054601F049F80F4BE4B25E6AA1
:10C49800072D4FF00103CDE9024301460AD10522D9
:10C4A8000023CDE900234FF47A727A431846B04747
:10C4B80005B0F0BD08220020CDE900203A46F5E796
:10C4C80017110108F0100108CC1701081FB5002347
:10C4D80000930378013B372B21D8DFE803F01C24B5
:10C4E8002020201E202020204143454E2055585B07
:10C4F8005E6164206C1E6E73787A20207D81262010
:10C5080020202020202020202020202083858A20F1
:10C5180020838A208C90C3780BB102230093009863
:10C5280005B05DF804FB8378F6E743788DF80430AE
:10C5380005238DF805308378003B18BF01235B0085
:10C548008DF8063010238DF80730304B1B6801A892
:10C5580003F55872CDE9022300F0C0FF0090DEE732
:10C568004023DBE72023D9E7827890F9013012B91C
:10C57800274AD35CD2E7274AFBE7827890F9013053
:10C58800002AF8D1244AF4E740F6B833C6E74FF456
:10C598007A73C3E74FF4FA63C0E741F28833BDE723
:10C5A80041F27073BAE71D484FF47A7101F020FE2A
:10C5B80000F5FA60D2E71A4BB0E7144B1B6803F595
:10C5C8005873ABE7114B1B6803F55B73A6E71023A1
:10C5D800A4E70E4B1B68A1E74FF0834300939EE747
:10C5E800104BFBE7104B99E740F21113ADF8003000
:10C5F80095E7032392E790F901300C4AB9E70C4913
:10C6080090F9010000F08AFFA8E700BF6C1C002029
:10C618009F110108A7110108AF11010818FCFFFFBD
:10C6280000EA06379A99094040F7093717110108B7
:10C63800F010010837B50B4B02781B680C2101FB81
:10C6480002335B7A03EB4304074B1D6803690093CD
:10C65800C3684278816805EBC40000F0DFFC03B0D2
:10C6680030BD00BF6C1C0020681C002070B586B06F
:10C67800027B6423ADF80030012A4FF00003CDE9B6
:10C688000133CDE903338DF802308DF8143030D002
:10C69800022A39D05ABB03684BB343683BB31F4DDA
:10C6A80080682B601E4B18226946186001F0BCFD9B
:10C6B8001C4B2C6893E807000C3384E8070093E8C8
:10C6C800070004F10C06032386E80700A4F86C337E
:10C6D800012204F55B7104F5587000F090FC2B689A
:10C6E8004FF6B072A3F878230522C3F87C2306B06E
:10C6F80070BD0A4908684360036100F55B7100F585
:10C70800587000F07CFCF2E7044B1B68B3F8602318
:10C71800B3F86C130A43A3F86023E8E76C1C002005
:10C72800681C0020780E010808B503460A2924D899
:10C73800DFE801F006232323230B161B2321210006
:10C74800BDE808400068FFF783BE90F900009978BB
:10C75800052271B900F013FC003818BF012008BD8C
:10C76800052293F900000021F4E790F900005978B8
:10C77800EEE70221EEE70722F3E70020EFE70000EB
:10C7880010B504791CB1012C0BD0002010BD0A4B48
:10C7980001681B68012203F5587000F030FC012085
:10C7A800F4E7054B01681B68224603F55B7000F04F
:10C7B80026FC2046EAE700BF6C1C0020F7B50528D8
:10C7C800144D1C46A8BF052058700E46294617462A
:10C7D80000F0A4FE94F90130A070072B13D1322089
:10C7E80000F09CFD0C4BDB6D0546984704F10C02EC
:10C7F80008340346019200943A463146284600F030
:10C8080092FD03B0F0BD054A55F82310D05C00F046
:10C818007DFDE7E7F0100108CC17010817110108A2
:10C828002DE9F04F344F90F901607B68D0F80490FF
:10C838008BB00446884698470546002859D1E37CC2
:10C8480073B92E4A2378126803EB4303990002EB6D
:10C858008303D3F80490B9F1000F01D152F8019085
:10C86800274B484613F906B0FB689847A37CD7F8CE
:10C8780018A022890993072E28D100230121CDE988
:10C888000223204A0693CDE90431CDE90733052177
:10C89800CDE900214FF47A7202FB0BF24CF25031D1
:10C8A8001846D047637C13B3174B995D7B6D0D31E8
:10C8B800C9B228469847E07C3246494600F040FE17
:10C8C80088F8006001200BB0BDE8F08F0021012539
:10C8D8000823CDE90013CDE90715CDE90511CDE908
:10C8E80003110292A1782B465A462846D9E7074BEE
:10C8F800DBE70020E7E700BFCC1701086C1C00202D
:10C908001711010885450100AF1101089F110108A1
:10C918002DE9F04F8DB090F90130DFF8FCA0DFF879
:10C92800FC90CDE90A123E4A12F903B00278DAF80F
:10C9380000300C2505FB02333A4A5B7A126803EB98
:10C94800430302EBC303044693F9021090F9020073
:10C9580000F0DFFD3449064694F9010000F0DEFDE1
:10C96800A26861688046304600F005FD2178DAF853
:10C978000020D9F80C306943074650589847D9F831
:10C988001C309C4694F901300025072B4FF47A633C
:10C99800CDE90753CDE905552DD10123CDE9035341
:10C9A8000523CDE901534FF47A7303FB0BF300938E
:10C9B8003946434646F2A81228466746B8472378C0
:10C9C800DAF800200C214B4394F90110D05800F0FC
:10C9D800D9FDA18994F90100FFF74EFD0B9B217B3E
:10C9E8001860D9F85430284698470A9B01201E70D1
:10C9F8000DB0BDE8F08F01200823CDE90350CDE943
:10CA080001032A46CDF800B0654643463946A84793
:10CA180001200546D3E700BF6C1C0020CC17010895
:10CA280017110108681C0020F01001082DE9F04FCB
:10CA38008FB0002405468A46914698460494ADF87E
:10CA48001440ADF8024007264FF0010B2B7AA342A1
:10CA580006D9686804A9204400F0F2FB00285ED1DA
:10CA680002238DF8083002A86B7A8DF80A30FFF798
:10CA78002DFDAB7A8DF81D309DF811308DF81E30E4
:10CA88009DF812308DF81F309DF810308DF8203049
:10CA9800EB7A8DF821302B7B8DF822306B7B8DF86B
:10CAA800233010238DF81C608DF824303A4E8DF811
:10CAB8002C000DF102030A9305238DF82D303368FD
:10CAC8000C930723ADF834302B6806930DF112024E
:10CAD80004AB0DF1110106A800F0CCFB07280546B0
:10CAE8000BD130680C22002100F5587001F0B0FB22
:10CAF8003368BDF80220A3F860239DF811308AF846
:10CB080000309DF8123089F800309DF8103088F810
:10CB18000030189B28461C700FB0BDE8F08F9DF8B8
:10CB28001330BDF81470ADF802702044C4B2F3B9E4
:10CB380017B3194A00201168072602464FF00C0C5B
:10CB4800062B1BD10CFB00FE51F80EE0BEF1000FC6
:10CB580004D00BFA00F23A4397B2012201301028B0
:10CB6800EED1002A3FF472AFADF802706EE75A1E9C
:10CB7800042A01D9062BDCD0062667E747FA00FE0F
:10CB88001EF0010FEAD00CFB00FE51F80EE0BEF1DA
:10CB9800000F08BF0626E1E76C1C002038B50546E3
:10CBA8004068FFF755FC0522841D002195F9000017
:10CBB800E4B200F0E4F908B904F0FD0495F90100C5
:10CBC8000722002100F0DBF908B904F0FB04204635
:10CBD80038BD00207047000010B503780F2B0446BD
:10CBE80018D84068FFF734FC22780B4902EB420260
:10CBF8000968831C01EB820051F82220DBB21AB9C4
:10CC080003F0FD0358B210BD032B06BF62684260F3
:10CC18000223F7E70020F6E76C1C0020022070478B
:10CC28002DE9F04FDFF838810446D8F8000099B0B4
:10CC38008946174600211E460122032300F5587035
:10CC4800CDE90611CDE908118DF814108DF81510ED
:10CC5800ADF8163000F0B5F938B9D8F80020B2F8B8
:10CC6800603343F00303A2F86033D8F80020637AF6
:10CC78008DF8283002F55871CDE90B12394A94F92C
:10CC8800083012680D920DF116020F922268109268
:10CC980062681192D4E90301A27A8DF84820012232
:10CCA8008DF8492013AA82E803001025227DE18A25
:10CCB8008DF8293018468DF85420ADF83850FFF714
:10CCC800DBFB0AAB17930DF1150316900093314661
:10CCD800019705AB06AA10A800F0BCFB064698BB56
:10CCE8009DF81410204F013901F082FA1F4B1B697F
:10CCF8000393C4B24FF00C0B04F160036B44D8F8F3
:10CD0800000013F848AC9DF814300BFB0AFC013402
:10CD18003946B4FBF3F203FB1244D0F87C33B0F984
:10CD2800782350F80C00DDF80CC0E4B2E04728B1D5
:10CD380089F800A0304619B0BDE8F08F013D15F024
:10CD4800FF05D9D10D26F5E70C2801BFD8F800203A
:10CD5800B2F8603343F00303A2F86033EAE700BF98
:10CD68006C1C0020681C0020400D0300CC17010833
:10CD7800F8B50679012E054601D80620F8BD0F2E14
:10CD88002BD80368187A40F303000522002140B22B
:10CD980000F0F5F82B680446187A40F303100522D2
:10CDA800002140B200F0EBF8A8B1B4FA84F46409A9
:10CDB80029680B7A086843F3030243F3031352B25A
:10CDC8005BB29A42C8BF0124FFF742FB48B9002C66
:10CDD800D3D10420D2E70124EAE70320CEE70520D7
:10CDE800CCE7002CFBD10C4F29683B6806EB4600CA
:10CDF80003EB80000C2201F017FA3A680C2303FBBE
:10CE0800062320465C72B2F860130123B3400B433B
:10CE1800A2F86033B2E700BF6C1C002010B40178A0
:10CE280001290ED9084B18680C234B43C41800225B
:10CE3800C250C4E9012200F5587010BC102200F05D
:10CE4800A7B8002010BC70476C1C00202DE9F041E9
:10CE580086B050238DF81430037A102B074630D152
:10CE68004368DD7B6DBB0224A8466426062C14D8D3
:10CE78007A68535D03932A44517843EA0123039364
:10CE8800927843EA02437343CDE9033863B96846AD
:10CE98008DF80040FFF7C2FF0DE0CDF80C808DF84B
:10CEA8001480CDF81080F2E703AB01A801938DF848
:10CEB8000840FFF75DFF0134E4B2102C05F10305CB
:10CEC800D4D106B0BDE8F0811FB5026803791168B6
:10CED80051B901A88DF80430FFF7A0FF78B90020F8
:10CEE80040B205B05DF804FB02A802928DF80C3040
:10CEF800FFF73EFF0628F2D8024B185CF0E7032044
:10CF0800EEE700BF10110108C90020B9034B0B441C
:10CF18009856C0B27047024BF9E700BF1F110108CD
:10CF28005F110108F0B59A42069D03DB9DF91430A4
:10CF38009A4220DD0020F0BD03EB430331F814C012
:10CF480005EB830300264CFA06F7FF0707D51F7A7F
:10CF580007F00F0E724502DBB2EB171F0DDD01362D
:10CF6800102E03F10C03EED10134E4B22301DBB23D
:10CF78009842E1D8DEE70024F8E70120DBE78842A1
:10CF880004DB9042CCBF002001207047002070478E
:10CF980010B51409B4EB111F03464FEA11100ED354
:10CFA80091420CD202B201F00F0133F81240012075
:10CFB80000FA01F124EA010123F8121010BD002043
:10CFC800FCE7F0B528B100EB4105012700209142AC
:10CFD80000D3F0BD002435F802CB234607FA04F647
:10CFE80036EA0C0608BF013304F1010408BFDBB2BE
:10CFF800102CF3D118440131C0B2C9B2E7E710B51B
:10D0080000B149B910BD31F8134020F8134001337D
:10D01800DCB2A242F7D8F5E70023F9E782B030B5D1
:10D02800048804936AB9B3F5616F18D349F6AF253C
:10D0380042F21072AB4298BF4FF47A72944238BFF2
:10D048001446012C38BF01246143BDE83040C36851
:10D058008B428CBF5B1A0023C36002B07047642206
:10D06800ECE700002DE9F04F91B01546DDF86C8033
:10D0780004939DF8683009930C46064603F0B4FB08
:10D08800684ADFF8A4B10590A8F5F633303BB3FB46
:10D09800F2F3534303F5F63203F5A83303F5C073EF
:10D0A8000393182313FB0543303206920893002597
:10D0B8004FF0FF3A089BA34207D1002D14BF5046FA
:10D0C8004FF0FF3011B0BDE8F08FBDF97030ADF80A
:10D0D8002C300B99CDF86C804046CDF8288003F0B1
:10D0E80013FBB4F800906EB9B8F5616F5BD349F6DD
:10D0F800AF2242F21073904598BF4FF47A73994566
:10D1080038BF99464B46012B38BF01230793002EA1
:10D1180052D1B9F1640F48D1A0605F46A1680EA84A
:10D1280003F014FB0F9B0093DDE90A120E9B0CA879
:10D1380003F06BFA049B0C9A0BB9099B2BB123697A
:10D14800BB4202D1394B9A420DD9394BE760984519
:10D1580009D90023ADF83430069B0D990C93184675
:10D1680003F0D2FAA060606800B9E760276126B1D1
:10D1780003F044FBE3680344E360D4E903329342D9
:10D18800059B1D996360079B88BFE2604B43E1687C
:10D19800994202D20498A8B9A6B101231D44237567
:10D1A800EDB2183486E76423A9E7B9F57A7F0ABF98
:10D1B800204F214FA060B1E7049B0BB9C4F80CB015
:10D1C8005F46D0E700209342207506D85B1A9A453F
:10D1D80005F1010528BF9A46EDB2002EE1D1B9F15B
:10D1E800640F164AADF8346019D049F6B023B9F582
:10D1F8007A7F18BF1346904584BF039A9B180C93F7
:10D208001C9B00930CAF97E806001B9B384603F065
:10D21800FCF997E8030003F077FA8246C1E74FF478
:10D228006163E8E78051010040771B007F510100EE
:10D238002FEC010080A81201002E930230EC0100AF
:10D248000378032B14D1437803F00F021B098A706B
:10D258004B7083788B80C27843EA02238B800379F2
:10D26800C3F3021203F00F03CA700B700520704756
:10D27800002070472DE9F34798464379057990F9DE
:10D2880007609146044690F906208A4683B190F9D2
:10D29800087075B30F2A12D194F909200F2E1ED1E8
:10D2A80094F90A60072D24D1002F08BF012720E038
:10D2B80090F90B7090F9092090F90A60E9E7A369E1
:10D2C800019394F915300093216994F91430207B67
:10D2D800FFF728FE0028E1D105F0FD05DEE794F907
:10D2E8001D30B3420FDC94F91C30B342DADA05F092
:10D2F800FB0528468AF8002089F8006088F8007045
:10D3080002B0BDE8F0871E46CCE70000024B03FAE6
:10D3180000F0B0FBF1F0704740420F004FF4FA53B1
:10D32800B3FBF0F0704730B54FF47A750C1F6A43C1
:10D3380000FB042252001EBF00F1FF341219B2FB99
:10D34800F0F2914238BF1146039A116082004843B7
:10D358001CBF013040084FF47A71121A01FB1323E5
:10D36800002BCABF03F2E73393FBF1F1B3FBF1F1F2
:10D37800049B196030BD38B5400014460D46F4F7DB
:10D3880045FB01462846F4F78FFA2146F4F78CFA54
:10D39800F4F77EF903F0C4FCF4F75AFA40B238BD4A
:10D3A8002DE9F74F019300231F469C461C01058A6F
:10D3B8005FFA84FE04F0F004A54206D8019B82F8C7
:10D3C80000C01F7003B0BDE8F08F0EEB4E054FEAAA
:10D3D8004309AD000024466836F809602641F6077F
:10D3E80027D5866806EB050A765916B3067836B946
:10D3F800466926B136F809602641F60719D59AF824
:10D40800086090F901B046F303084FFA88F8D84548
:10D418000FDC46F3031676B25E450ADB9AF809601C
:10D4280006EB4608C66806EBC806367D4EB90137D6
:10D43800FFB20134102C05F10C05CCD10133DBB25D
:10D44800B4E70CF101060EEB040801F80C805FFA52
:10D4580086FCEEE72DE9FF4704464068DDE90C67E6
:10D468001D468A46914603F0C9F923681B1A3B609A
:10D478004FF000080123337085F80080636813B10A
:10D488002368834224D8CAF80080D4F81CC0A36952
:10D498009CF800E00393D4E9030101AB83E803009F
:10D4A800237D0093DCF80C10237A627A7046FFF72C
:10D4B800D9FD334638602A46E0694946FFF770FFD0
:10D4C8002B782BB1C7F80080002004B0BDE8F087A6
:10D4D8003378002B14BF0B200C20F6E737B590F9F2
:10D4E800002090F90250954204460FD0013A52B2FA
:10D4F80095420BD0A368019394F9013000936168B9
:10D50800E0782B46FFF70EFD0028EFD0104603B059
:10D5180030BD8842B8BF08467047000051F8200067
:10D52800054B984205D0054BC31A58425841400054
:10D5380070470120704700BF90D0030020A107006A
:10D5480005281FB50ED80C4B53F820300093CDE9B1
:10D5580001120A4B01220021022002F05BFE05B0F5
:10D568005DF804FBCDE90012054B012200210220E1
:10D5780002F050FEF3E700BF24120108B7110108BA
:10D58800D611010807B5054BCDE90001012200219C
:10D59800022002F03FFE03B05DF804FBF21101081F
:10D5A80010B5102204460021F13000F051FE002190
:10D5B800C4F814112046F022BDE8104000F048BE1F
:10D5C80002460846102100F0A5B92DE9F0430446AB
:10D5D800D0F8140185B00E46154604F2011988B337
:10D5E800C0F110089045474628BF1746BAB24844CC
:10D5F80000F01AFED4F814313B440F2BC4F8143150
:10D608002DD9A8452BD204F1F00304F5807113F845
:10D61800012F187C8B4282EA00021A70F7D104F1BC
:10D62800F10810224146684600F0FEFD2246694690
:10D63800684600F0E9F910226946404600F0F4FD1A
:10D648003E44ED1B04F5807804F1F107102D09D84C
:10D65800AAB23146484600F0E7FDC4F8145105B0B7
:10D66800BDE8F08304F1F003711E13F8012F11F8DF
:10D67800010F434582EA00021A70F6D1102239469A
:10D68800684600F0D1FD22466946684600F0BCF9BC
:10D6980010226946384600F0C7FD1036103DD5E720
:10D6A800F0B589B00C46102200210546684600F006
:10D6B800CFFD22466946684600F0A6F99DF900307C
:10D6C800002B6A464FF0000143DA137812F8010F75
:10D6D80001315B0043EAD0130F2902F8013CF4D171
:10D6E8009DF80F305B0083F08703D4F81401DBB298
:10D6F80010288DF80F303BD104F58073694604F586
:10D70800887013F8016F11F8012B984282EA06021B
:10D718001A70F6D104F1F00304F5807113F8012FA3
:10D72800187C8B4282EA00021A70F7D110220DEBA6
:10D73800020004F1F10100F077FD2246294604A811
:10D7480000F062F910220021684600F081FD09B05E
:10D75800F0BD137812F8010F01315B0043EAD013D2
:10D768000F2902F8013CF4D19DF80F305B00BCE7AB
:10D778009DF90030002B6A464FF0000137DA137824
:10D7880012F8016F01315B0043EAD6130F2902F842
:10D79800013CF4D19DF80F305B0083F08703471CF0
:10D7A800DBB28DF80F30102F04EB0003C0F10F0629
:10D7B8004FF0800288BF002600F5817083F80121B0
:10D7C8000021324620443E4403F064FAC4F8146150
:10D7D80004F58073694604F5887013F8016F11F831
:10D7E800012B984282EA06021A70F6D192E7137862
:10D7F80012F8016F01315B0043EAD6130F2902F8D2
:10D80800013CF4D19DF80F305B00C8E70A78037833
:10D81800534003704A784378534043708A7883783A
:10D8280053408370CA78C3785340C3700A79037928
:10D83800534003714A794379534043718A79837914
:10D8480053408371CA79C3795340C3710A7A037A02
:10D85800534003724A7A437A534043728A7A837AEE
:10D8680053408372CA7AC37A5340C3720A7B037BDC
:10D87800534003734A7B437B534043738A7B837BC8
:10D8880053408373CA7BC37B5340C373704710B53F
:10D898000B7814786340037054784B786340437076
:10D8A80094788B7863408370D478CB786340C37066
:10D8B80014790B796340037154794B796340437150
:10D8C80094798B7963408371D479CB796340C37140
:10D8D800147A0B7A63400372547A4B7A634043722A
:10D8E8008B7A947A63408372D47ACB7A6340C3721A
:10D8F800147B0B7B63400373547B4B7B6340437304
:10D90800947B8B7B63408373CB7BD27B5340C37305
:10D9180010BD0000A1F11003DBB2102B2DE9F04778
:10D9280004D8374C24FA03F3DB0705D4002382F824
:10D93800F030FF20BDE8F087531E4418A0424ED1B6
:10D9480001F11C039B005FFA83F9C3F30313013B46
:10D958002C4D82F8F03001240B46D618B3FBF1F0B9
:10D9680001FB103010F0FF0016F804AC16F803ECB9
:10D9780016F802CC16F8017C36D115F80E8015F889
:10D988000CE015F807C015F80A70E00900EB400034
:10D9980084EA080800EBC0006400C0B2E4B2444066
:10D9A800C246581AC0B212F800808AEA080A02F879
:10D9B80003A01044043390F801808EEA080E86F81C
:10D9C80001E090F802E08CEA0E0C86F802C0C078FC
:10D9D800DBB247409945F770BFD80020AAE710F896
:10D9E800015B03F8015FA9E71829DAD9102801BFFC
:10D9F80015F80AA015F80EE015F80CC0EF5DD0E791
:10DA0800010101003C1401082DE9F04FA3B092F880
:10DA1800F0301D911B920193002B00F053810146B9
:10DA28001EA8FFF734FF1B9BA74CA84DA84E103328
:10DA38000293002303939DF87C0004909DF88600D0
:10DA48000590205C06909DF87B000790205C08906C
:10DA580004989DF881C0205C099014F80C000A9085
:10DA68009DF880000B909DF885009DF878809DF8C2
:10DA78007DE09DF882A09DF887900C909DF87A0033
:10DA8800029B1C9314F80A2014F8093014F80810A3
:10DA980014F80E700D90205C0E909DF87F000F908A
:10DAA800205C10900B98205C11900C98205C1290D0
:10DAB8009DF8840013909DF8790014909DF87E00DD
:10DAC8001590205C16909DF883001790205C1890A4
:10DAD8001398205C19901498205C1A9003980130D0
:10DAE80003900298DDF804B0103002909DF80C0005
:10DAF800834536D88DF878108DF87A2009990E9AD2
:10DB08008DF87C108DF882201199069A8DF8801076
:10DB18008DF87E201999169A8DF884108DF8862034
:10DB28000A99189A8DF87D108DF887201299109A05
:10DB38008DF87B301B9B8DF881108DF883201A9906
:10DB4800089A1D988DF885108DF87F201EA903EB83
:10DB58000B128DF87970FFF79AFE002023B0BDE80C
:10DB6800F08F15F808B082EA03008BEA000016F877
:10DB78000EB080EA0B008DF8780015F80E004B40C7
:10DB8800434016F80A0043408DF8793081EA0703CC
:10DB980015F80A10594016F80930594016F8083097
:10DBA8008DF87A107A40534015F8092053408DF8C3
:10DBB8007B30089A069B5340049AAA5C534016F897
:10DBC8000C2053408DF87C30DDE908325A4015F8B6
:10DBD8000C305340059AB25C53408DF87D30DDE936
:10DBE80009325A40059BEB5C5340079AB25C53409C
:10DBF8008DF87E30069B0A9A5340049AB25C5A40CC
:10DC0800079BEB5C5A408DF87F200E9B109A53407F
:10DC18000B9AAA5C53400C9AB25C53408DF8803042
:10DC2800DDE910325A400C9BEB5C53400D9AB25C14
:10DC380053408DF88130DDE911325A400D9BEB5C81
:10DC480053400F9AB25C53408DF88230129A0E9B63
:10DC580053400B9AB25C5A400F9BEB5C1C995A409C
:10DC68008DF88320169B189A5340139AAA5C534048
:10DC7800149AB25C53408DF88430DDE918325A406A
:10DC8800149BEB5C5340159AB25C53408DF8853079
:10DC9800DDE919325A40159BEB5C5340179AB25C88
:10DCA80053408DF886301A9A169B5340139AB25CEB
:10DCB8005340179AAA5C1EA853408DF88730FFF787
:10DCC800A5FDB8E6FF2049E73C1401083C1201080D
:10DCD8003C13010808B538B1044A05491060D82238
:10DCE80000F0A2FA002008BD0220FCE7701C00200A
:10DCF8006C1901080A4B1A6870B5002302F118055F
:10DD080003EB03142E5D864204D1183422440A60C2
:10DD1800002070BD01330B2BF2D10320F9E700BFBF
:10DD2800701C00202DE9F041CCB00646DDF8488192
:10DD380017461C460D4631B3B8F1000F23D006A88C
:10DD4800FFF72EFC204601A9FFF7D4FF0446B0B91F
:10DD5800019906A80131FFF733FC26B1102231469C
:10DD680006A8FFF732FC3A46294606A8FFF72DFC1D
:10DD780006A902A8FFF794FC029BC8F800302046C9
:10DD88004CB0BDE8F0810224F9E7000030B595B049
:10DD980013A90446FFF7AEFF002830D11B490C2316
:10DDA80003FB00F2555CA5422BD1139B187C109005
:10DDB800D87B0F90987B0E90587B0D90187B0C9019
:10DDC800D87A0B90987A0A90587A0990187A08901D
:10DDD800D879079098790690587905901879049021
:10DDE800D8780390987802900A445B7801939368F6
:10DDF80000930022064B1146022002F00BFA15B0E0
:10DE080030BD01300B28CBD1F9E700BFB4160108AB
:10DE18003C1501080B2B10B402D810BCFFF782BFC9
:10DE2800032010BC704730B50D4685B01446014636
:10DE380068B103AA002000922A460390FFF772FFF8
:10DE480018B90398001B18BF012005B030BD022087
:10DE5800FBE72DE9F0430D46BFB0144699468046CE
:10DE680020B31BB311F00F0122D1F02201A800F05A
:10DE7800EFF920466946FFF73DFF044648B9009888
:10DE880001AA10210130FFF745FD2E46AF1BFFB256
:10DE98001EB920463FB0BDE8F08301AA09EB07018F
:10DEA80008EB0700FFF7B0FD103EEFE70224F0E7AC
:10DEB8000524EEE7F0B5184E3468024685B00846EA
:10DEC800002304F1180103EB03154F5D97421ED19F
:10DED8000D2A05F1190513D10023CDE90033CDE949
:10DEE80002330C2210216B46FFF7B3FF044630685B
:10DEF80010226946284400F097F9204605B0F0BD85
:10DF080001461022601900F08FF90024F5E701336B
:10DF18000B2BD8D10324F0E7701C002009B1FFF7C0
:10DF2800C9BF022070471FB51446A0B10C2A01D101
:10DF38000B2912D10023CDE90033CDE902330A467B
:10DF48006B461021FFF785FF18B969462046FFF791
:10DF5800B1FF04B010BD0220FBE70320F9E7F8B5D4
:10DF68001E46DDE907479DF818505BB354B34FB31D
:10DF7800212D29D819462A46204600F055F90122B4
:10DF8800631C691EB018FFF764FFF8B9E37ADB0970
:10DF98003B70EBB96319204613F8012C13F8021CE7
:10DFA800120642EA014213F8041C0A4313F8031C40
:10DFB800012342EA0122291FFFF735FF003818BF65
:10DFC8000120F8BD0220FCE70520FAE70720F8E762
:10DFD8000420F6E708B5014630B1044B082218685A
:10DFE80000F022F9002008BD0220FCE7701C002088
:10DFF80008B530B1044B0822196800F015F9002063
:10E0080008BD0220FCE700BF701C00207FB5124E3F
:10E018000023044602A801930D46FFF7E9FF336881
:10E028005B6901936CB102AA082312F8011B41B97C
:10E03800013B13F0FF03F8D102A8A04702A8FFF79D
:10E04800C9FF35B1019B23B901A8A8473368019AD4
:10E058005A61002004B070BD701C002008B501464C
:10E0680038B1054B18680822104400F0DDF800208C
:10E0780008BD0220FCE700BF701C002008B538B1BD
:10E08800044B19680822114400F0CEF8002008BD9E
:10E098000220FCE7701C0020034B1B6802280CBF01
:10E0A8001961596100207047701C002041B1054B6F
:10E0B8001B6802280CBF1B695B690B600020704756
:10E0C80002207047701C002030B58FB00024054630
:10E0D8000CA80994FFF78CFF9DF8373007939DF83B
:10E0E800363006939DF8353005939DF83430049307
:10E0F8009DF8333003939DF8323002939DF8313008
:10E1080001939DF830300093224621461E4B022091
:10E1180002F080F80AA8FFF7B1FF9DF82F300793A7
:10E128009DF82E3006939DF82D3005939DF82C30E0
:10E1380004939DF82B3003939DF82A3002939DF8A1
:10E14800293001939DF82830009322460F4B214631
:10E15800022002F05FF809A92846FFF7A7FF9DF8FB
:10E16800243003939DF8253002939DF826300193BF
:10E178009DF8273000932246054B2146022002F0E5
:10E1880049F80FB030BD00BF98150108D615010831
:10E198001416010808B50020FFF7F8FD0120FFF765
:10E1A800F5FD0920FFF7F2FD0820FFF7EFFD00203D
:10E1B800FFF78AFF002008BD10B504460B20FFF7C3
:10E1C800E5FD0C20FFF7E2FD0920FFF7DFFD082041
:10E1D800FFF7DCFD0A20FFF7D9FD2046FFF774FFA3
:10E1E800002010BD014B1860704700BF3C010020A3
:10E1F8000B4A30B514680B4D43F2390305FB043361
:10E208001360091A6FF00042B3FBF2F2C2EBC2725C
:10E2180001319B1A93FBF1F201FB1233184430BD14
:10E228003C0100206D4EC64101380A44914200D19C
:10E23800704711F8013B00F8013FF7E710440A4422
:10E24800914200D1704711F8013B00F8013DF7E712
:10E2580002F020BD30B530B10A4D01444FF0FF3314
:10E26800814201D1D84330BD10F8012B5340082218
:10E2780043F30004013A2C4092B284EA5303002A83
:10E28800F6D1EDE72083B8ED01207047054B4FF438
:10E2980000529A62044B1B6813B15B6803B11847BC
:10E2A800704700BF00040048741D0020054B4FF460
:10E2B80080529A62044B1B6813B1DB6803B118479C
:10E2C800704700BF00040048741D002001207047FB
:10E2D8000120704701F048B901F036B910B501F0D6
:10E2E80019FE0E21044640F61F1001F02DF92046B4
:10E2F800012101F0F9FDBDE8104001F0D7BA000096
:10E3080070B50C4E01EB40030D46B3654FF6FF7137
:10E31800002304461A46084601F05EFB96F85600AC
:10E32800002101F0E1FD29462046BDE8704001F0DA
:10E3380095BA00BF901D002010B5044601F0AAFE52
:10E3480001281CD101F0AEFE34B11248214602F07A
:10E3580017FB104802F0DAFA0F4C104B00214FF46B
:10E368008052A1659A6194F8560001F0BDFD63786A
:10E378006BB16FF07F40BDE8104001F053BA002345
:10E3880040F262211A46084601F026FBDCE7A06845
:10E398008001F0E7781D0020901D0020000400484F
:10E3A800002001F0BFB9000008B501F0C7F8043833
:10E3B800C0B2032896BF024B0020185C08BD00BFFE
:10E3C800C817010808B501F0BAFD033008BD01F00F
:10E3D80049B901F009B908B501F000FD00B208BD5E
:10E3E80038B50D46144601F05DFB284601F092FD54
:10E3F8000E21054640F61F1001F0A6F82846012117
:10E40800074D01F071FD01F051FA4FF47A71614343
:10E41800284602F0B5FA2846BDE8384002F076BA38
:10E42800EC1D002001F03EBB08B5084B002193F815
:10E43800560001F059FD00234FF4C0711A460846F2
:10E4480001F0CAFABDE8084001F024BA901D002086
:10E4580010B5044601F01EFE01281CD101F022FE71
:10E4680034B11248214602F08BFA104802F04EFAF5
:10E478000F4C104B00214FF48052A1659A6194F81B
:10E48800560001F031FD63786BB16FF07F40BDE855
:10E49800104001F07DB9002340F262211A46084677
:10E4A80001F09AFADCE7A0688001F0E7781D002007
:10E4B800901D00200004004808B54FF0040001F04A
:10E4C80017F9BDE808400220F4F7F2BA08B50023AE
:10E4D8001A461946184601F07FFABDE8084001F0CF
:10E4E8006DB900001D4B73B51D4D186000241D4803
:10E4F8006C70C5E90144AC6501F098FAAC8101F093
:10E5080003FA2146204601F04BFC21460422012053
:10E5180001F0FCFA144E154D4FF6FF7123462246C2
:10E52800084601F059FAFFF7C7FF2246104B00943E
:10E538004FF0FF31304602F03DF90E4B0094224671
:10E548004FF0FF31284602F035F9304602F090F9D5
:10E55800284602B0BDE8704002F08AB9741D002058
:10E56800901D002035F50008EC1D0020781D0020C6
:10E5780095E20008B5E200080128084805D1084BD3
:10E58800C17719700E3001F0A7BB437D012B03D171
:10E59800034B81751970F5E7704700BF901D002087
:10E5A800400100200D4B10B5044618735873012024
:10E5B80000F016F85CB134214FF4E86000F0C4FFB5
:10E5C8004421BDE8104040F2417000F0BDBF142165
:10E5D8004FF4E86000F0B8FF2421F2E7901D002016
:10E5E80038B5114C0546207001F061FD052D04D8A1
:10E5F800DFE805F0090B03171709032001F070FA8B
:10E608000023637338BD0020F8E7012001F068FAA1
:10E61800207B637B8342F5D06073BDE83840FFF709
:10E62800C1BF0220EAE700BF901D00202DE9F0439A
:10E638001E4687B000230546CDE901330C46174630
:10E6480001F027FD032D61D8DFE815F07B00C3003A
:10E658000E010400A27C082A04D94FF0FF3007B04D
:10E66800BDE8F083A16801A801F0DCFE216800295B
:10E67800F3D042F210729142E37C864D51D80322C6
:10E68800AA7385F83820E96385F844304FF002080A
:10E698006368A17DDB002B820423AB74A37CDB00C1
:10E6A800EB7402294FF000032B75637D02D0227DA5
:10E6B800022A42D103F10F02D2B2012A01D9012B59
:10E6C800CBD1754B754A196803944FF0010903A81B
:10E6D8008DF8149001F0DAFC0028BED1287685F870
:10E6E80017906875FFF75CFE4046FFF779FF6C48A6
:10E6F80001F086FA6B4801F0EFFA01A800F084FFF8
:10E70800208A00F055FFA08900F09AFF384601F0F2
:10E7180001FC604C84F8560001F0C0FC66600020E3
:10E728009DE74FF00008E963890885F80E8085F8B1
:10E73800388085F844302964AAE7EB7529766A752C
:10E74800D0E72368002B88D0A27C082A85D8514DB1
:10E75800A16801A801F066FE002385F83830226818
:10E76800EA63E27C85F84420A269AB732A64626894
:10E77800A17DD2002A820422AA74A27C2B75D20021
:10E788000229637DEA7402D0227D022A1DD103F199
:10E798000F02D2B2012A02D9012B7FF45EAF3E4BA1
:10E7A8003E4A196803944FF0010803A88DF81480B5
:10E7B80001F06CFC00287FF450AF287685F81780AC
:10E7C8006875FFF7EDFD00208FE7EB7529766A7510
:10E7D800F7E7304D012185F83810227885F8502068
:10E7E800637885F85130A37885F85230E3788B4206
:10E7F80002D0022B03D03BB985F8533004E00B3A22
:10E80800012A29D885F853104FF0010885F80E80A1
:10E81800A388AB83A379AB77E37985F82030237A93
:10E8280085F82130FFF7BCFD4046FFF7D9FE1C48AC
:10E8380001F0E6F91B4801F04FFA95F85130062B24
:10E8480040F689000AD100F08FFE00F0FB0140F687
:10E85800890000F079FE59E70023CDE700F084FE37
:10E8680040F00401C9B2F2E72368013BB3F57A7FAF
:10E87800BFF4F3AE0320FFF7B3FE0648022380F887
:10E88800383023688364162380F84C30383001F020
:10E89800B7F93BE7901D0020741D0020EC1D0020F7
:10E8A800C81D00209E1D00202DE9F041002686B0DD
:10E8B8001F461446CDE9016680460D4601F0E9FB86
:10E8C800B442764C16BF0123334637466370B8F11D
:10E8D800000F06D0B8F1010F7CD0002006B0BDE8CB
:10E8E800F081AB68002B00F0D680EB68002B00F0BD
:10E8F800D280AA7F082A00F2CE80296901A801F0F7
:10E9080091FD2868003818BF012000F0D9FF84F86D
:10E918003880AB68E36395F8203084F84430686841
:10E9280001F05AFB84F80E8084F84500EB68DB00A0
:10E938002382EB7FA374AB7FDB00E37495F821306F
:10E94800237595F82230002B3ED12A7D95F82410A6
:10E95800A275022995F8232001D0022B36D102F1A5
:10E968000F03DBB2012B02D9012A40F09480002367
:10E978008DF814304A4B4B4A1968049503A801F0E6
:10E9880085FB002840F0878001232076E3756075B9
:10E99800FFF706FD0020FFF723FE434801F030F99A
:10E9A800424801F099F901A800F02EFEA88B00F06A
:10E9B800FFFD288B00F044FE4FF4FA53AA687B430E
:10E9C800B3FBF2F3A36088E7FF22BFE7E275217685
:10E9D8006375DDE72B8E002B5DD095F83230A86A81
:10E9E800012B0CBF95F814804FF0FF08003818BFB2
:10E9F800012000F065FFF8B200F06EFF012184F8F5
:10EA0800381095F82C2084F8502095F82D3084F88B
:10EA1800513095F82E3084F8523095F82F308B42CB
:10EA280002D0022B03D03BB984F8533004E00B3AF0
:10EA3800012A28D884F853102B8EA38395F83230F6
:10EA4800A377AB8E23840126A67384F81F80FFF773
:10EA5800A7FC3046FFF7C4FD134801F0D1F813486E
:10EA680001F03AF994F82130B34240F236700CD1F3
:10EA780000F07AFD00F0FB0140F2367000F064FD12
:10EA88004FF6FF739EE70023CEE700F06DFD40F0E0
:10EA98000401C9B2F0E74FF0FF301FE7901D0020D6
:10EAA800741D0020781D0020C81D00209E1D002018
:10EAB8002DE9F04F85B082460E9DBDF840B09DF817
:10EAC80044709DF84890019288461E4601F0E1FA8C
:10EAD800BAF1010F524C54D0BAF1040F00F09180F2
:10EAE800BAF1000F3AD10B22304684F8442084F85A
:10EAF80038A0E56301F070FA019B23644FEACB0369
:10EB0800B9F1000F238241F60403638214BFF22394
:10EB18000123E37587F001070123237684F8450074
:10EB280084F80EA084F814A06775FFF739FC5046E6
:10EB3800FFF756FD04F1380001F062F804F10E0009
:10EB480001F0CAF8374A1068516802AB03C302A83B
:10EB580000F05AFD40F2FF1000F02AFD404601F097
:10EB6800D9F90E2184F8560040F61F1000F0ECFC8D
:10EB780094F8560001F092FA169B636005B0BDE860
:10EB8800F08F294984F838A0EAB2895D84F85020CA
:10EB980076BB0B3D012D8CBF00250125053A012AC6
:10EBA80004D8BBF10C0F38BF4FF00C0B1F4B9DF86E
:10EBB8003C201B7884F85350E37701259DF85430A6
:10EBC80084F8511084F8522084F82130A573A4F8F1
:10EBD8001CB0A77784F82090FFF7E2FB2846FFF7E0
:10EBE800FFFC134801F00CF8124801F075F8B5E77E
:10EBF800012E04D1A5F10C035D425D41CEE700254D
:10EC0800CCE75046FFF7ECFC022384F8383004F1D7
:10EC180038001623A56484F84C3000F0F1FF9DE716
:10EC2800901D0020900E0108961701084001002051
:10EC3800C81D00209E1D00202DE9F04F87B0DFF889
:10EC4800B4B29DF864A09DF84C90029314469DF8C8
:10EC580054309DF85020BDF84880039205468BF843
:10EC680001A0BDF8446001930F4601F012FABAF111
:10EC7800000F18BF4FF00008DFF87CA2039AB9F123
:10EC8800000F08BFFF22012D8AF8002000F0C8807D
:10EC9800052D48D0002D40F0C080284600F010FE19
:10ECA8000B2238468BF844208BF83850CBF83C4080
:10ECB80001F092F9019B8BF8450041F60402002B04
:10ECC800ABF812209AF800208BF8162014BFF22215
:10ECD80001228BF81720F600012289F001098BF830
:10ECE80018208BF80E50ABF810608BF814508BF886
:10ECF8001590FFF755FB2846FFF772FC0BF138001B
:10ED080000F07EFF0BF10E0000F0E6FF7B4908687B
:10ED1800496804AA03C204A800F076FC40F2FF1078
:10ED280000F046FC71E0012000F0CAFD09224FF016
:10ED380000098BF8442038464FF44872CBF840203D
:10ED48008BF83890CBF83C4001F046F94FF48052EC
:10ED5800ABF812209AF800208BF845008BF81620A3
:10ED680028460122F6008BF817208BF80E90ABF896
:10ED78001060ABF814908BF81890FFF731FC0BF18A
:10ED8800380000F03DFF0BF10E0000F0A5FF5B49D5
:10ED98008868C96804AA03C204A800F035FC40F2D8
:10EDA800FF1000F005FC40F6B80000F0DDFB00F0B5
:10EDB800EF0140F6B80000F0C7FB042140F6B900A7
:10EDC80000F0C2FB40F69B0000F0CEFB00F0E30130
:10EDD80041F0080140F69B0000F0B6FB40F2D1601C
:10EDE80000F0C2FB40F01801C9B240F2D16000F057
:10EDF800ABFB40F2AC6000F0B7FB00F08F0141F0D4
:10EE0800500140F2AC6000F09FFB4FF4FA5202FB55
:10EE180008F2B2FBF4F2CBF8082007B0BDE8F08F97
:10EE2800002000F04DFD36498BF83850E2B2C95D3C
:10EE38008BF85020002F4DD10B3C012C8CBF0024A7
:10EE48000124053A012A02D80C2E38BF0C26029B51
:10EE58009AF800208BF852308BF85340019B8BF8BE
:10EE68001F2001249DF860208BF821208BF8511079
:10EE78008BF820308BF80E40ABF81C608BF81E9096
:10EE8800FFF78EFA2046FFF7ABFB1E4800F0B8FEEE
:10EE98001D4800F021FF5FFA88F000F01DFD40F6E4
:10EEA800A30000F061FB00EA040140F6A30000F0B3
:10EEB8004BFB9BF82120A24240F2367013D100F0A0
:10EEC80053FB00F0FB0140F2367000F03DFB4FF6BB
:10EED800FF72A0E7012F04D1A4F10C035C425C414E
:10EEE800AFE70024ADE700F03FFB40F00401C9B2F2
:10EEF800E9E700BF901D002040010020900E0108A6
:10EF080096170108C81D00209E1D0020F0B58BB083
:10EF18000D46044617461E46FFF742FA0020FFF743
:10EF28005FFB204600F0BEFD00240123CDE9084325
:10EF380003234FF4167229462046CDE90644CDE94D
:10EF48000444CDE90244CDE900532346FFF774FE9B
:10EF58002046FFF77DFAFFF735FAF3F7A9FD01F030
:10EF680043FC0446204601F049FCB04205D3012485
:10EF7800FFF716FA20460BB0F0BD00F02FFF00B2E5
:10EF88008742EFDA0024F3E7F7B500230C4640F296
:10EF980001211A460646084600F01EFD644B654DE1
:10EFA8004FF400529A6195F85600012100F09CFF39
:10EFB8002B78012B40F6890013D195F85130062B98
:10EFC8000FD100F0D1FA00F0FB0140F6890000F003
:10EFD800BBFA2B78042B6CD8DFE803F0524B527F36
:10EFE800090000F0C1FA40F00401C9B2EDE7524A45
:10EFF800731E1046C6F101074FF0000CF9188C4239
:10F008006FDC0022E7001346BA4271D19A0142EA46
:10F01800C3125B0183F020031343661C0355F6B249
:10F0280002234648AB73AE7600F056FE0021F1206D
:10F0380000F08AFA0021F02000F086FAAB6C642B0D
:10F0480070D17021F32000F07FFA1D21F22000F02A
:10F058007BFAE1008C1CF420090A00F075FA04F030
:10F06800FE01F52000F070FA33486FF07F42314618
:10F078001DE0EC77314800F02FFE0022214615E014
:10F0880001F008F80128074625D121460DF10702AD
:10F09800304601F004F80446A0B99DF80730274827
:10F0A800AB7500F019FE9DF807102246304600F0B7
:10F0B80065FB6968224801F063FC214801F026FCE1
:10F0C800002006E01F4B3A460021022001F0A2F87A
:10F0D800032003B0F0BDAC75CCE70223AB73AC766C
:10F0E800C8E713F8011FC943197002F801CB85E777
:10F0F800D1106FEA020C715C0CF0070C013241FA76
:10F108000CF101F001014FEAE20C4B40D14310F839
:10F118000CE001F0070103FA01F141EA0E0100F8E1
:10F128000C1071E7E121F32000F00EFA04218DE7BD
:10F1380000040048901D0020741C00209E1D002023
:10F14800EC1D002038170108F0B5BDF814409DF8F3
:10F1580018709DF81CE09DF8205040B1012814D08B
:10F168000122002398180138B0FBF2F0F0BD87F0B7
:10F178000107E30003EBC70318330EEB450503EB68
:10F18800C5034FF47A714B43ECE7501F012803F194
:10F19800040302D80C2C38BF0C24D1B9A2F10B0CF3
:10F1A800BCF1010F8CBF4FF0000C4FF0010C28018F
:10F1B800002F00EBCE0014BF00251425A0EB820021
:10F1C800062A4FEA82062844A2F102070DD83546DE
:10F1D80010E0012906D1A2F10C00D0F1000C4CEB93
:10F1E800000CE4E74FF0000CE1E70830BCF1000F39
:10F1F800EDD0BD000028ACBF2E182E1C701E90FB51
:10F20800F5F003FB0044094B062A5A5C8CBF0C340A
:10F218000E340A2A09D8A30001334FF47A71BB408F
:10F228004B43034951F822209CE7FFDE961701085B
:10F238009C17010808B5094B012193F8560000F006
:10F2480053FE4FF4D7602D2100F07EF900F033FB18
:10F25800BDE80840024800F07BBA00BF901D0020BE
:10F26800FFFF0F0073B5A44CB4F854300025202BD1
:10F278008DF80350019500F01B8114D8082B0DD888
:10F288007BB1013B072B0CD8DFE813F042005B0091
:10F298000B00CD000B000B000B00FD00102B00F045
:10F2A800008102B070BDB3F5807F00F0988011D85E
:10F2B800402B00F01081802BF3D1284600F032FA61
:10F2C8008E4B1B68002BECD09B69002BE9D028469D
:10F2D8009847E6E7B3F5007FE3D1894B0122294639
:10F2E800022000F097FF00F029F9042840F08580FB
:10F2F800844B85484FF400529A6201F0B9FA2846C7
:10F3080000F010FA7D4B1B68002BCAD05B6814E034
:10F318007C4B7D484FF400529A6201F0A9FA002014
:10F3280000F000FA00F0B8FE012801D100F0BDFE9F
:10F33800724B1B68002BB4D01B68002BB1D09847C8
:10F34800AFE7704B71484FF480529A6201F090FA1F
:10F35800657895B9284600F0E5F9294640F6021087
:10F3680000F0F2F840F6441000F0FEF840F0020118
:10F37800C9B240F6441000F0E7F8FF220DF103018E
:10F3880063485E4D00F05AFD624800F071FD2B683D
:10F39800002B86D09E68002E83D094F82430012B51
:10F3A80008D194F9313094F930209DF80310584869
:10F3B800B04776E7E06B01A900F022FE019B9DF8BB
:10F3C800031053484FF47A7203F5FA7393FBF2F380
:10F3D8002A685BB2956894F92920A84761E728460E
:10F3E80000F0A0F9454B1B68002B3FF45AAF9B690E
:10F3F800002B3FF456AF01206AE700F09FF805287C
:10F408007FF44FAF3F4B41484FF480529A6201F06E
:10F418002FFA284600F086F9384B1B68002B3FF47A
:10F4280040AFDB6889E700213B4B0122022000F056
:10F43800F1FEA16D00293FF434AFC1F3074140F656
:10F44800031000F081F894F8591040F6041000F009
:10F458007BF894F8581040F6051000F075F840F65F
:10F46800021000F081F840F00101C9B240F6021024
:10F4780000F06AF8002340F262211A460846A365A4
:10F4880000F0AAFA0DE7254B01220021022000F026
:10F49800C1FE00F0FFFD01287FF403AF00F006FE77
:10F4A800FFE61F4B01220021022000F0B3FEF8E620
:10F4B800164801F0DDF9607808B900F033F90F4B10
:10F4C8001B68002B3FF4EDAEDB68002B3FF4E9AE80
:10F4D8009847144BE6E7144B01222946022000F016
:10F4E80099FE607808B900F01DF9044B1B68002BE1
:10F4F8003FF4D7AE1B6920E7901D0020741D002043
:10F508004D17010800040048EC1D0020781D00205C
:10F51800741C0020B41D0020611701086A17010837
:10F52800741701087D17010886170108024BA3F814
:10F538005400FFF797BE00BF901D0020014B1878BC
:10F54800704700BF0A1E002007B501238DF8071079
:10F558000DF1070201460348F7F786F803B05DF896
:10F5680004FB00BF4C03002007B5012301460DF141
:10F5780007020448F7F7B1F89DF8070003B05DF8F3
:10F5880004FB00BF4C03002010B50446F4F726FD29
:10F5980001280CD140F62310FFF7E6FF00F0F9012F
:10F5A800214340F62310BDE81040FFF7CDBF10BD42
:10F5B80010B50C4B1B7804469BB94FF4D760FFF786
:10F5C800D3FFC4F3002100F0FE0001434FF4D760DD
:10F5D800FFF7BAFFE1B240F2B960BDE81040FFF7AB
:10F5E800B3BF10BD0B1E002010B51346EFF31084F7
:10F5F80072B60A4601460348F7F736F884F31088CE
:10F6080010BD00BF4C03002008B5014608224FF486
:10F61800D860FFF7E9FF002008BD000007B5074BD9
:10F628001B7840BAADF804002BB9022201A940F2B8
:10F63800BC60FFF7D9FF03B05DF804FB0B1E002088
:10F6480007B5074B1B7840BAADF804002BB9022266
:10F6580001A940F2BE60FFF7C7FF03B05DF804FBE5
:10F668000B1E002010B51346EFF3108472B60A463D
:10F6780001460348F7F731F884F3108810BD00BF3E
:10F688004C03002010B51346EFF3108472B60A46F7
:10F6980001460348F7F713F984F3108810BD00BF3B
:10F6A8004C0300200A4601460020FFF7EBBF00008C
:10F6B80010B51346EFF3108472B60A4601460348A4
:10F6C800F7F730F984F3108810BD00BF4C03002011
:10F6D80010B51346EFF3108472B60A460146034884
:10F6E800F7F736F884F3108810BD00BF4C030020EC
:10F6F80013B504460020F4F74BFC0220FFF744FF43
:10F7080004F0070401220DF1070184208DF8074059
:10F71800FFF7DEFF024B00221A7002B010BD00BFD7
:10F728000A1E002007B501228DF807000DF1070118
:10F738008020FFF7CDFF9DF80730002B034B0CBF4F
:10F74800012202221A7003B05DF804FB0A1E002091
:10F7580007B5094B8DF8060004221A70030C8DF8C2
:10F7680004300322030A01A983208DF80530FFF72E
:10F77800AFFF03B05DF804FB0A1E002010B5144665
:10F78800FFF790FF2046BDE81040FFF7E1BF0000FB
:10F7980007B5094B8DF8060005221A70030C8DF881
:10F7A80004300322030A01A982208DF80530FFF7EF
:10F7B8008FFF03B05DF804FB0A1E002073B5002616
:10F7C80040F6E2000196FFF7CFFE00F0FE01054685
:10F7D80040F6E200FFF7B8FE40F6E500FFF7C4FE8A
:10F7E80000F07F01044640F6E500FFF7ADFE6FF03C
:10F7F8007F40FFF7CDFF04220DEB020140F6190010
:10F80800FFF730FF3046FFF78DFF294640F6E2004C
:10F81800FFF79AFE214640F6E500FFF795FE0198AE
:10F8280002B070BD13B50C4B04460522972140F673
:10F83800AC001A70FFF788FE230C8DF80430032201
:10F84800230A01A982208DF805308DF80640FFF7BC
:10F858003FFF02B010BD00BF0A1E002007B5030C11
:10F868008DF80030030A8DF801300B0C49BA8DF879
:10F878000200ADF804100622694694208DF8033082
:10F88800FFF726FF024B06221A7003B05DF804FB4F
:10F898000A1E0020002208B51146C520FFF718FFF0
:10F8A800014B07221A7008BD0A1E002000221146CB
:10F8B800D120FFF70DBF00221146D220FFF708BF65
:10F8C80007B501228DF807000DF107019F20FFF70A
:10F8D800FFFE03B05DF804FB07B501228DF80700B1
:10F8E8000DF10701A020FFF7F3FE9DF807103F294F
:10F8F80007D901F0F8010131C9B240F20670FFF7EB
:10F9080023FE03B05DF804FB07B5F4F767FB431E5D
:10F91800584258418DF8070001220DF10701962041
:10F92800FFF7D6FE03B05DF804FB07B500F07F00D3
:10F938008DF8070001220DF107018920FFF7C8FEA5
:10F9480003B05DF804FB0000154B984207B51BD8BF
:10F95800144B98421BD8144B98421BD8134B98420F
:10F968001BD8134B984295BF29226B222B236F2358
:10F978008DF8042001A9022298208DF80530FFF7A0
:10F98800A7FE03B05DF804FBE122E923F0E7D722E4
:10F99800DB23EDE7C122C523EAE775228123E7E7E8
:10F9A80000E9A43580F8A9328044E52D000B6B1BD3
:10F9B80040FC541907B58DF8062004228DF8040080
:10F9C8008DF8051095200DEB02018DF80730FFF733
:10F9D8007FFE03B05DF804FB07B552BAADF804200A
:10F9E80040BA082249BAADF80000ADF802105BBA77
:10F9F80069461046ADF80630FFF76AFE03B05DF8B9
:10FA080004FB07B50B0C042200F0070049BA8DF877
:10FA18000400ADF8061097200DEB02018DF80530B3
:10FA2800FFF756FE03B05DF804FB000010B508B1FF
:10FA3800194B1860F2F73EFF0220FFF7A5FD0024DE
:10FA4800164B20461C70FFF76DFEF4F7C5FA012827
:10FA580017D14FF42071FFF7D4FF40F6111021465B
:10FA6800FFF772FD4FF07F00FFF75FFF0E2140F6B2
:10FA78001F10FFF769FDF4F757FA094B01221A70B6
:10FA880010BD102140F61110FFF75EFD102140F661
:10FA98001210FFF759FDE9E70C1E0020081E002090
:10FAA8000A1E002037B50C4D2B7804461BB9FFF70A
:10FAB8004BFF01232B700023084A6006E109F2F787
:10FAC80023F8042200BA01900DEB02018620FFF70B
:10FAD800FFFD03B030BD00BF081E00200048E8014C
:10FAE80007B5094B8DF807000146187018B940F2A0
:10FAF800AC60FFF729FD01220DF107018A20FFF70D
:10FB0800E7FD03B05DF804FB0B1E0020012873B568
:10FB18000C46164637D10020F4F762FAA042B8BF67
:10FB280044B20E2805461AD101231A4600210420A2
:10FB3800FFF740FF6FF010039C42B8BF1C46182126
:10FB480040F6E700FFF700FD022201A98E208DF89C
:10FB580004408DF80560FFF7BBFD02B070BD0123BE
:10FB68000A28E4B21A464FF0000105D11846FFF7FB
:10FB780021FF033464B2DDE70720C5F10E05FFF766
:10FB880019FF2C44F6E740F6D800FFF7EDFC40F0EB
:10FB98001E01C9B240F6D800FFF7D6FC0120F4F7E1
:10FBA8001FFAA042B8BF44B2142805464FF001031B
:10FBB8004FF000020CD105210320FFF7FBFE0234B1
:10FBC80064B26FF008039C42B8BF1C463821B7E7FF
:10FBD800112805D103210220FFF7ECFE0534EFE7D9
:10FBE8000E2804D102210846FFF7E4FEE9E7C5F133
:10FBF8001605072104202544FFF7DCFE6CB2E0E778
:10FC080013B5314A0446516810686B4603C32F4B3D
:10FC180020781B78834201D0FFF762FF2378032BFB
:10FC280027D8DFE803F00239283C6268284BB3FB89
:10FC3800F2F31A0CA1688DF800208DF802301A0A28
:10FC4800237B8DF80330637B8DF801208DF8043019
:10FC5800204A00234806C909F1F756FF030C40BAA9
:10FC68008DF80530ADF80600082269468B20FFF7AD
:10FC78002FFD02B010BD2269154BB3FBF2F31A0C2D
:10FC88008DF800208DF802301A0A237D8DF80120A6
:10FC98008DF803300422E8E7A3690093FAE7626865
:10FCA8000B4BB3FBF2F31A0C8DF800208DF80230E1
:10FCB8001A0A237B8DF80330637B8DF801208DF8B9
:10FCC80004300522D1E700BFA00E01080B1E00205A
:10FCD8000000093D0048E8011FB52E4A0446D168D6
:10FCE8009068127C01AB03C31A702B4B20781B78E9
:10FCF800834201D0FFF7F4FE2378032B26D8DFE8F0
:10FD080003F002383302637AF12B21D14FF6FF70EA
:10FD1800FFF784FC48F20500FFF792FC0223628893
:10FD2800A188ADF8061052BAE188ADF804208DF824
:10FD38000B30227AA37A8DF80A20ADF808108DF8D6
:10FD48000C30092201A98C20FFF7C2FC04B010BDB9
:10FD5800F22BE4D141F60F50FFF760FC41F221008D
:10FD6800FFF76EFC0623DAE7237B8DF804300122C7
:10FD7800E8E7E389094A5BBAADF80430237C1370DD
:10FD88008DF80630637C8DF80730638AADF808304B
:10FD98000622D7E7A00E01080B1E0020091E00202E
:10FDA80007B502228DF804008DF805108F2001A9EF
:10FDB800FFF78EFC03B05DF804FB000010B5134696
:10FDC800EFF3108472B60A4601460348F6F7F8FCCA
:10FDD80084F3108810BD00BF4C03002007B5012232
:10FDE80001A91520FFF7EAFF9DF8040040424010E2
:10FDF80003B05DF804FB000037B505460C46022247
:10FE080001A91320FFF7DAFF0A4B1B78012B0DD14C
:10FE1800094B1B78012B09D140F20270FFF7A4FBB4
:10FE28009DF805302870237003B030BD9DF804009C
:10FE3800F6E700BF0B1E0020091E0020F7B50D468F
:10FE4800064600240DF10701284617468DF807409D
:10FE5800FFF7D2FF2A78BA4207D89DF80700314643
:10FE6800FFF726FC204603B0F0BD0120FBE70000A9
:10FE780013B50322044601A91420FFF79FFF184B6E
:10FE88001A7822704AB1012A17D01422002120467C
:10FE980000F0D2FA0F2323700DE09DF8043023718F
:10FEA8009DF80530A2605B425B10A3719DF8063097
:10FEB8005B425B10637102B010BD9DF804305B4279
:10FEC8005B1023739DF9053002339B1063739DF813
:10FED80006305B425B10A373024B1B682361EAE7A1
:10FEE8000B1E0020041E0020012908B50346084601
:10FEF8000ED1012B07D10420FFF746FB0220BDE8F5
:10FF08000840F4F745B8022B14BF08460320F6E76B
:10FF18000120F4E738B50446F4F75CF850B102283C
:10FF280014BF01250225284602222146FFF7EEFDCF
:10FF3800284638BD0F2CCCBF02250125F3E70A203F
:10FF480070470000014B01201B6818470C1E002059
:10FF5800014B02201B6818470C1E0020014B402053
:10FF68001B6818470C1E002011B1012904D07047E6
:10FF7800044B1B6880201847024B4FF480701B68A5
:10FF8800F9E700BF0C1E0020024B4FF400701B68FD
:10FF9800184700BF0C1E0020014B20201B68184783
:10FFA8000C1E0020014B04201B6818470C1E002063
:10FFB800014B08201B6818470C1E0020014B10201D
:10FFC8001B6818470C1E0020024B4FF480401B682A
:10FFD800184700BF0C1E002068B1084A002352F8D9
:10FFE8003310814203D902EBC30210797047013301
:08FFF800162BF4D1FEE71F20D7
:020000040801F1
:10000000704700BF5818010873B51D4B0193044693
:1000100040F607000D46FFF7ABFAC0F3C103083303
:100020006B4413F8042C00F00703013302FA03F3C6
:10003000144AB2FBF3F2B2FBF4F007281ED84000DA
:1000400003288CBF022304234FF4D66002FB03F481
:10005000FFF78EFA060240F2B160FFF789FA06F464
:1000600070663043030544BF6FEA00506FEA1050DA
:1000700063094343DB112B6002B070BD0123E3E74A
:1000800004080A0C0048E8014FF0FF3070474FF0B9
:10009000FF3070474FF0FF307047704700207047C7
:1000A0000020704770474FF0FF3070474FF0FF302F
:1000B000704770477047704770B5EFF3108672B69F
:1000C000144B5C8A1A8A944213D1C4F5806292B2AE
:1000D000904206D3844218D901229A7000221C80D3
:1000E0005A825A8A0A800244C2F309025A820020C4
:1000F0000DE006D9C4F58065ADB28542F1D88242E3
:10010000E9E7121B92B28242EBD84FF0FF3086F340
:10011000108870BD10220020EFF3108172B6034AE0
:10012000D38A0133D38281F31088704710220020D4
:10013000EFF3108172B6034AD38A013BD38281F375
:10014000108870471022002010B50848182200219E
:1001500000F076F906484FF48062002100F070F953
:10016000044B05481B68BDE81040184710220020CA
:10017000101E0020400F0108E9020108014B5860E1
:10018000704700BF10220020014B1872704700BF5B
:100190001022002073B5EFF3108572B61C4CE08A74
:1001A00000282FD1FFF7B8FF218A628A914227D019
:1001B000A378012B12D1238820805B1A9BB20221E5
:1001C000A382A17063B9A3702382238A9A428BBF52
:1001D000D21AC3F58063A282A38201E0002BF4D07F
:1001E000238A0C4E1E4485F31088F2F753FC0A4B09
:1001F000A18ADB680193304602B0BDE87040184721
:10020000FFF796FF85F31088002002B070BD00BF95
:1002100010220020101E0020400F010808B4F0B585
:1002200086B00023ADF800302C4B0B9C1D7A854224
:100230004DD3D86881434DD15B681BB112B169467B
:1002400002A898470CAB22464FF400712448019352
:1002500000F0F6FBFFF760FFBDF8003018440DF129
:10026000020180B2FFF728FF01302BD00022BDF839
:100270000030BDF802701B480DF1080C164691B213
:1002800017FA82F58B42ADB216D83B449BB20EB141
:10029000ADF80230BDF80250019B22464FF40071C8
:1002A000284400F0CDFBFFF743FFFFF773FF06B0D4
:1002B000BDE8F04001B070471CF8011B4155013208
:1002C0000126DCE7FFF734FF6FF00200EFE76FF085
:1002D0000400ECE76FF00500E9E700BF1022002002
:1002E00028220020101E002013B5EFF3108472B6F0
:1002F000204B9A78588A022A1DBF1A8A998A521866
:10030000002214BFC2F309029A7090421A8228D0C8
:10031000D98A012925D19978012913D119888A1AF6
:10032000022192B2997000219A82198062B99A7062
:100330001A821A8A90428BBF801AC2F58062988214
:100340009A8201E00029F4D01A8A0B48104484F301
:1003500010880A4A998AD368019302B0BDE8104018
:10036000184784F31088F2F799FB02B0BDE81040FB
:10037000FFF7DEBE10220020101E0020400F0108F3
:10038000024A00231360024A136070472C240020A5
:100390002824002010B5EFF3108472B641B1012972
:1003A00003D1064A13680343136084F3108810BD19
:1003B000024A136823EA0003F6E700BF2C2400205A
:1003C00010B5EFF3108472B641B1012903D1064A8A
:1003D00013680343136084F3108810BD024A136846
:1003E00023EA0003F6E700BF2824002038B5EFF326
:1003F000108572B60A4B0B4C1B6833B123689847C3
:100400006368984785F3108838BD074B1B681BB19C
:10041000A3689847E368F4E7236998476369F0E7BE
:100420002C240020CC0E01082824002001380A4486
:10043000914200D1704711F8013B00F8013FF7E706
:1004400000F02CBC10B5EFF3108472B6064A1368A6
:1004500003431360054A52F83130034342F8313008
:1004600084F3108810BD00BF7C2400207424002079
:1004700070477047030C1B04C3B90004102310F02D
:100480007F4F02BF08330002DBB210F0704F08BF8D
:1004900000014FEA1070064A08BF0433125C08BF1F
:1004A000DBB2C3F11F03981AC0B270470023E6E71E
:1004B000081901082DE9F84F384D394ED5F800805C
:1004C000DFF8E0B0DFF8E0A0DFF8E090D6F800C099
:1004D000374FDBF80010374CDAF80020D9F800303D
:1004E00008EA00002860286800EA020E1EEA0C0FE5
:1004F00001D019421ED04FF0FF333B60FFF7B8FF29
:10050000EFF3108472B63368DBF80020DAF80010DD
:100510000B4029680B4205D1D9F80030134201D1B4
:10052000F2F746FA84F31088FFF7A3FFC5F80080BE
:10053000BDE8F88F236823680340134062681A42BD
:1005400004BF4FF0FF32626060681840FFF792FF0F
:1005500062683860012303FA00F022EA0002626058
:10056000EFF3108172B63A689340326822EA0302D0
:100570003260226822EA0303236081F310880E4A66
:100580003B6852F823309847D6F800C0DBF80010DB
:10059000DAF80020D9F80030A5E700BF44010020B8
:1005A0007C2400203424002048010020382400202E
:1005B00030240020742400203C24002010B5114673
:1005C000EFF3108472B6FFF755FF034B43F820108A
:1005D00084F3108810BD00BF3C24002082B082B09C
:1005E0000DF1080C0CE90600BDF8042003930B4440
:1005F000BDF810100A4491B212B2B2F57A7FA2BFD0
:10060000A1F57A72013312B20360828002B002B0A7
:10061000704782B082B00DF1080C0CE90600BDF8FD
:1006200004200393CB1ABDF81010521A91B212B2E3
:10063000002ABEBF01F57A7203F1FF3312B20360E4
:10064000828002B002B0704730B585B0114D6B4664
:1006500083E8030000230293ADF80C3003A82B6954
:100660009847009BBDF804400290181ABDF80C3062
:10067000E41AA3B224B2002CBEBF03F57A731CB2F5
:1006800000F1FF302B689847AB682046984705B0CB
:1006900030BD00BF000F010873B5114E00230546A1
:1006A0000093ADF8043001A833699847F3680090CF
:1006B0009847736804469847009B1844BDF8043077
:1006C00023449AB21BB2B3F57A7FA2BF0130A2F5E0
:1006D0007A731BB228602846AB8002B070BD00BFA1
:1006E000000F010837B500230093ADF80430074B25
:1006F00004461B6901A898476D46009095E80300E1
:1007000084E80300204603B030BD00BF000F01089D
:1007100037B50F4D02AB03E90300EB6898476B68F0
:1007200004469847BDF80430009A1B1B99B21BB2CF
:10073000002BA2EB0002BEBF01F57A7102F1FF327D
:100740000BB24FF47A7000FB023003B030BD00BF33
:10075000000F01082DE9F0414FF47A75B1FBF5F572
:10076000C5EB4513DFF83C8005EB8303A1EBC30326
:100770009CB2D8F80C3006469847D8F804300746A3
:100780009847E31999B21BB2B3F57A7F2844A2BF08
:10079000A1F57A7301301BB23060B3803046BDE8FA
:1007A000F08100BF000F0108024B00221A60024BCB
:1007B0001B68184780240020140F0108F8B5044670
:1007C000174608461E467CB173B1084B00255B6A8C
:1007D00025609847069B60602581A572E6602361CD
:1007E000E77265612846F8BD0120FCE7140F010897
:1007F00010B5034CE3699847A36ABDE81040184759
:10080000140F010870B5064DEB69064698476B6AF0
:10081000044630469847AB6A201ABDE87040184736
:10082000140F0108054B1B680BB91846704783422B
:1008300001D05B69F8E70120704700BF80240020E9
:100840002DE9F3410B4E336A044698470123B769FB
:100850002372D4F800800546B8472844804502D268
:10086000B84728442060B3682068019302B0BDE80F
:10087000F0411847140F010870B520B3EFF310864C
:1008800072B6124D2B680122827253B1002242725D
:1008900098425C690ED102723CB120462C60FFF791
:1008A000CFFF86F31088002070BD094BDB689847A6
:1008B0002C60F6E71A465B69002BF2D09842F9D11A
:1008C00043695361EDE70120EEE700BF802400207B
:1008D000140F0108084B10B51A685369516911B912
:1008E0005061416110BD046819688C4202D91A46F2
:1008F0005B69F3E71946F3E780240020044A136894
:100900000BB10021197243611060FFF799BF00BF5E
:10091000802400202DE9F041044600282DD0FFF767
:1009200081FF50BB657A45BBEFF3108872B6144E59
:100930006768336A984787422CBF27602060114F51
:10094000A5724FF4807323813B684BB93369984794
:100950002046FFF7D3FF88F310882846BDE8F081D2
:10096000B3699847236818443B6820601B68984225
:100970002046EED3FFF7AEFFEDE70125EDE700BF20
:10098000140F01088024002010B5044608467CB1ED
:10099000084B5B6A984760602046FFF743FF40B111
:1009A0002046FFF769FF2046BDE81040FFF7B2BFC1
:1009B000012010BD140F01082DE9F041EFF310875D
:1009C00072B61D4E1D4D73699847336904469847AA
:1009D0002B684BB94FF000082B688BB9286828BBEF
:1009E00087F31088BDE8F081011B241A1A688A4237
:1009F0008CBF121900221A605B69002BF6D1E9E75F
:100A00001C681CB1B36998478442E7D22C686369BB
:100A10002B60A4F80880D4E9033098476389B3F5C4
:100A2000807FD9D12046FFF775FFD5E7037A002BE9
:100A3000D6D1FFF705FFD3E7140F0108802400206B
:100A40002DE9F04F97B000298046039140F30E81C5
:100A50009A46044603991378A4EB0800013923B998
:100A60000023237017B0BDE8F08F8842F8DA252BF9
:100A700004D004F8013B1646721CEBE792F801C063
:100A8000ACF13003D3F1000E4EEB030EACF13003AA
:100A9000092B02F1010629D8324600254FF00A0938
:100AA000164612F8013BA3F13000092819D9337812
:100AB000692B00F09C801CD8632B28D0642B00F09D
:100AC0009680582B5BD0252B19D13378002B00F062
:100AD000928004F8013BA4EB08038B4280F28980EA
:100AE000CAE709FB0533A3F13005D9E74FF0FF351D
:100AF000DDE7752B7DD0782B43D0732B1ED02523BB
:100B000004F8013BA4EB08038B4272DADDE7002D09
:100B100005F1FF39D8BF4FF000094A462046202191
:100B200000F0BCF85346A144002D53F8042B89F87B
:100B30000020D8BF01252C449A469DE74C4B5AF81B
:100B4000047B002F08BF1F463846F0F739FCA5EBA1
:100B5000000B8542B8BF4FF0000B5A46814620215A
:100B6000204600F09BF8A34400234B4502DB0BEB2F
:100B7000090481E7FA5C0BF803200133F5E74EF036
:100B8000400E1020DFF8EC903B4F1EF0400F08BFE6
:100B90004F465346BCF1300F0197A4EB08020CBF3F
:100BA000302720271EF0020FA1EB0202029753F814
:100BB000041B22D0002920DA4942013D4FF02D0EBE
:100BC00005AF009700278946DDF804A0B1FBF0F1DE
:100BD00000FB119B48451AF80BB0DDF800A00AF89D
:100BE00001BB07F10107CDF800A0ECD90EE04EF0F3
:100BF000020E0A20C6E7013E6DE711B14FF0000E6C
:100C0000DEE730208DF814008E460127BCF1300F4E
:100C1000A5EB070504D02020002D05F1FF3509DCE8
:100C2000BEF1000F04D02D21013A04F8011B83D03E
:100C300025440AE0013A04F8010BEDD17CE7029962
:100C400004F8011B013A3FF477AF291B0029F6DCB9
:100C500005A9394422442744A7423FF46DAF11F857
:100C6000010D04F8010B9442F6D165E70020F9E686
:100C7000181901081F1901084419010810B5013994
:100C80000244904201D1002005E0037811F8014FA1
:100C9000A34201D0181B10BD0130F2E70244034605
:100CA000934200D1704703F8011BF9E770B50D4D71
:100CB0000D4C641BA4100026A64209D10B4D0C4C10
:100CC00000F0B2F8641BA4100026A64205D170BD46
:100CD00055F8043B98470136EEE755F8043B984732
:100CE0000136F2E74C1A01084C1A01084C1A0108A7
:100CF000501A010800F003B8002200F00EB80A44B0
:100D0000914200F1FF3300D1704710B511F8014B4B
:100D100003F8014F9142F9D110BD13460A46194616
:100D2000FFF7BCBF00000000C1F30A522DE9F843F1
:100D3000A2F2FF36132E0B4607460C46054632DC60
:100D4000002E14DA34A3D3E90023F0F747FB002286
:100D50000023F0F777FD38B1002C56DA24F0004478
:100D6000254355D02E4C002523462F4625E02D4AFD
:100D700042FA06F801EA080202431ED026A3D3E98C
:100D80000023F0F72BFB00220023F0F75BFD002887
:100D9000EAD0002CBEBF4FF480133341E41824EA9C
:100DA00008040025E0E7332E0BDDB6F5806F04D193
:100DB0000246F0F713FB07460B4638461946BDE8D6
:100DC000F883A2F213424FF0FF3828FA02F810EA33
:100DD000080FF2D010A3D3E90023F0F7FFFA0022A6
:100DE0000023F0F72FFD0028BED0002C0ADA142EC5
:100DF00001D1013406E0C6F134060123B3401D449D
:100E0000AF42F6D825EA0805AEE700252C46ABE749
:100E10004FF00044A8E700BF9C7500883CE4377E93
:100E20000000F0BFFFFF0F00F8B500BFF8BC08BC22
:100E30009E467047F8B500BFF8BC08BC9E46704798
:100E4000000000000100000002000000000000009F
:100E50008813000010270000204E000030750000AD
:100E6000409C000050C3000060EA0000C0D40100B4
:100E700080A903000053070000EA063700000000C5
:100E80005000000040F7093700000000500000004B
:100E9000C194C10000000000B22700000000000063
:100EA0000000000000000000000000000000000042
:100EB00000000000B5010008F1010008B40E0108AF
:100EC000FC7F003F00350113C4120008732700089F
:100ED000552700083927000859270008352700083A
:100EE000852700085975336E3148344F3152354EDD
:100EF000395332543653256473253033643A000035
:100F0000612C0008012D0008712C00080D2D00082F
:100F1000D12C0008192D000800000000812C0008C9
:100F2000392C0008052C0008BD2B0008152C0008E2
:100F3000292C0008C92B0008CD2B0008E12B000844
:100F4000C12F0008E92F00086D2F0008592F000855
:100F500052464143005056585858002159756E4822
:100F60006F726E2053545320526576697665210066
:100F70000100000003000000050000000100000067
:100F800001000000060000000A0000002000000030
:100F90000200000004000000080000001000000033
:100FA000400000008000000000010000000200007E
:100FB0000000000000000000000000000000000031
:100FC0000100000002000000030000000400000017
:100FD000A0860100400D0300801A060000350C00B9
:100FE00040420F0080841E0000093D0000127A007C
:100FF0000024F40000366E010048E801006CDC02B9
:1010000000000000000000000000000000000000E0
:101010000402080010101004101010021010100824
:10102000010002000400060008000A000C00100085
:1010300020004000800000010804020408010101B2
:1010400001010103070100006572726F723A2052BC
:101050006567696F6E206973206E6F7420646566C2
:10106000696E656420696E20746865204D573A206A
:10107000736574206C6F726177616E5F636F6E660B
:101080002E68206163636F7264696E676C790D0A04
:10109000004D414320727854696D654F75740D0A97
:1010A000004D414320747854696D654F75740D0A85
:1010B000004D4143207278446F6E650D0A004D412A
:1010C00043207478446F6E650D0A00080A0C0D0EFB
:1010D00010121415181A1B1D1E21240305020501E8
:1010E00006020205000006000001050404000000DD
:1010F00048E8010048E8010048E8010048E801002C
:1011000048E8010048E8010090D00300000000001A
:10111000030000000201000C0B0A09080707320057
:1011200000000000000102010000000000020302B4
:101130000100000000030403020100000004050494
:10114000030201000005060504030201000607066C
:101150000504030201070707060504030207070247
:10116000020202020202020202020202020203025E
:101170000202020202030403020202020204050444
:101180000302020202050605040302020206070624
:1011900005040302020707070605040302070733D5
:1011A000337373F2F2F2F200000B357DF2F2F23398
:1011B000337373DEDEDEDE52585F2573206F6E20E0
:1011C0006672657120256420487A2061742044523B
:1011D0002025640D0A005258206F6E2066726571DA
:1011E00020256420487A2061742044522025640D13
:1011F0000A005458206F6E206672657120256420A5
:10120000487A2061742044522025640D0A00310080
:1012100032004D756C74695F43004D756C74695F85
:10122000500000000E12010810120108530F0108AF
:1012300012120108201201081A120108C6F8EEF66F
:10124000FFD6DE916002CE56E7B54DEC8F1F89FACE
:10125000EFB28EFB41B35F452353E49B75E13D4CF8
:101260006C7EF5836851D1F9E2AB622A0895469D00
:1012700030370A2F0E241BDFCD4E7FEA121D583463
:1012800036DCB45BA476B77D52DD5E13A6B900C12F
:1012900040E379B6D48D67729498B085BBC54FEDA5
:1012A000869A66118AE904FEA078254BA25D800526
:1012B0003F2170F16377AF4220E5FDBF811826C35F
:1012C000BE35882E9355FC7AC8BA32E6C0199EA363
:1012D00044543B0B8CC76B28A7BC16ADDB6474145D
:1012E000920C48B89FBD43C43931D3F2D58B6EDA26
:1012F00001B19C49D8ACF3CFCAF447106FF04A5CF7
:1013000038577397CBA1E83E96610D0FE07C71CC06
:101310009006F71CC26AAE6917993A27D9EB2B22BF
:10132000D2A907332D3C15C987AA50A50359091A1C
:1013300065D784D082295A1E7BA86D2CA584998DEF
:101340000DBDB1545003A97D1962E69A459D4087B1
:1013500015EBC90BEC67FDEABFF7965BC21CAE6AE2
:101360005A41024F5CF434089373533F0C52655E4C
:1013700028A10FB509369B3D2669CD9F1B9E742E73
:101380002DB2EEFBF64D61CE7B3E7197F568002CD9
:10139000601FC8EDBE46D94BDED4E84A6B2AE5167D
:1013A000C5D75594CF100681F044BAE3F3FEC08A46
:1013B000ADBC4804DFC17563301A0E6D4C14352F77
:1013C000E1A2CC3957F28247ACE72B95A098D17FA8
:1013D000667EAB83CA29D33C79E21D763B564E1E0E
:1013E000DB0A6CE45D6EEFA6A8A4378B324359B7D5
:1013F0008C64D2E0B4FA0725AF8EE918D5886F72F5
:1014000024F1C751237C9C21DDDC86859042C4AA4F
:10141000D8050112A35FF9D0915827B93813B33317
:10142000BB7089A7B622922049FF787A8FF880177F
:10143000DA31C6B8C3B07711CBFCD63A637C777B80
:10144000F26B6FC53001672BFED7AB76CA82C97DC0
:10145000FA5947F0ADD4A2AF9CA472C0B7FD932651
:10146000363FF7CC34A5E5F171D8311504C723C355
:101470001896059A071280E2EB27B27509832C1A99
:101480001B6E5AA0523BD6B329E32F8453D100EDF3
:1014900020FCB15B6ACBBE394A4C58CFD0EFAAFBD7
:1014A000434D338545F9027F503C9FA851A3408F9F
:1014B000929D38F5BCB6DA2110FFF3D2CD0C13ECB7
:1014C0005F974417C4A77E3D645D197360814FDC4C
:1014D000222A908846EEB814DE5E0BDBE0323A0A30
:1014E0004906245CC2D3AC629195E479E7C8376DB4
:1014F0008DD54EA96C56F4EA657AAE08BA78252ED9
:101500001CA6B4C6E8DD741F4BBD8B8A703EB56661
:101510004803F60E613557B986C11D9EE1F8981152
:1015200069D98E949B1E87E9CE5528DF8CA1890D41
:10153000BFE6426841992D0FB054BB1623232323E5
:10154000232320257320253032583A253032583A4B
:10155000253032583A253032583A253032583A251B
:101560003032583A253032583A253032583A253000
:1015700032583A253032583A253032583A253032EE
:10158000583A253032583A253032583A25303258B8
:101590003A253032580D0A002323232323232044E5
:1015A00065764555493A20202020202025303258A4
:1015B0003A253032583A253032583A253032583AA6
:1015C000253032583A253032583A253032583A25AB
:1015D0003032580D0A002323232323232041707027
:1015E0004555493A202020202020253032583A25E0
:1015F0003032583A253032583A253032583A253070
:1016000032583A253032583A253032583A2530325D
:10161000580D0A00232323232323204465764164A5
:1016200064723A2020202020253032583A2530326A
:10163000583A253032583A253032580D0A00417058
:10164000704B65793A2020202020004E776B4B6547
:10165000793A2020202020004E776B534B65793A51
:101660002020202000417070534B65793A202020C3
:1016700020004442496E744B65793A202020004D89
:1016800043526F6F744B65793A2020004D434B45B0
:101690004B65793A20202020004D43417070534B18
:1016A00065795F303A004D434E776B534B65795FF8
:1016B000303A0000000000004150505F3E16010823
:1016C000010000004E574B5F4B1601080800000058
:1016D0004E574B5358160108090000004150505313
:1016E000651601080A0000004442495F72160108AD
:1016F0000B0000004D4352547F1601080C000000FF
:101700004D434B458C1601080D0000004D434B30F6
:10171000991601080E0000004D415330991601083A
:101720000F0000004D4E5330A616010810000000B7
:101730005A45524F73170108526164696F53656EC1
:1017400064204F76657273697A650D0A00495251BB
:101750005F52585F54585F54494D454F55540D0AD8
:1017600000505245204F4B0D0A0053594E43204F15
:101770004B0D0A00484452204F4B0D0A004844527A
:10178000204B4F0D0A004952515F4352435F45526F
:10179000524F520D0A00040506000000841E00008E
:1017A000093D0000127A000024F4000048E801001E
:1017B00090D0030020A1070000000000B128000025
:1017C00061510000C3A2000002010003EDE4000823
:1017D000B1E30008E9E500082DE4000815EF000872
:1017E000D5E4000841EC0008B9EA000891E20008DD
:1017F00051F1000891EF0008C1E40008A9E30008D6
:1018000059E4000831E40008E9E30008DFE30008D8
:10181000E1E20008DDE20008DBE30008D7E30008AE
:1018200081E50008ADE50008CDE300086DF2000891
:1018300041E3000809E300083DF20008E5E2000882
:10184000B1E8000835E60008890001088F000108AA
:10185000D5E20008D9E20008C01200001F00000015
:10186000A816000017000000841C00000F000000F4
:10187000E42500001E000000B42D0000160000004A
:10188000083900000E0000002C4C00001D00000074
:10189000685B000015000000747200000D0000007D
:1018A000589800001C00000034B70000140000002D
:1018B000E8E400000C000000783101001B0000008B
:1018C000686E01001300000034CA01000B00000024
:1018D000286202001A00000040DB02001200000033
:1018E0003C9303000A000000C0C20400190000007D
:1018F00060B3050011000000382007000900000057
:1019000020A1070000000000040302020101010100
:1019100000000000000000003C4E554C4C3E0030E2
:10192000313233343536373839616263646566671E
:1019300068696A6B6C6D6E6F7071727374757677AF
:1019400078797A003031323334353637383941429C
:10195000434445464748494A4B4C4D4E4F505152DF
:0C196000535455565758595A00000000C7
:10196C00000000000000000000000000000000006B
:10197C000000000000000000002B7E151628AED2DF
:10198C00A6ABF7158809CF4F3C012B7E151628AE58
:10199C00D2A6ABF7158809CF4F3C082B7E1516281D
:1019AC00AED2A6ABF7158809CF4F3C092B7E151686
:1019BC0028AED2A6ABF7158809CF4F3C0A00000021
:1019CC00000000000000000000000000000B000000
:1019DC0000000000000000000000000000000C00EF
:1019EC000000000000000000000000000000000DDE
:1019FC0000000000000000000000000000000000DB
:101A0C000E000000000000000000000000000000BC
:101A1C00000F0000000000000000000000000000AB
:101A2C00000010000000000000000000000000009A
:081A3C000000000000000000A2
:081A4400FC00FF7F010000001F
:041A4C005D01000830
:041A50003901000850
:101A54000200000000000000C6040020C0D4010001
:101A6400B5290008E5290008FD290008692A0008AD
:101A7400753200084D320008E1310008A334000833
:101A8400000000007D340008B5310008913E0008D4
:101A94009931000897310008A9340008E931000899
:101AA4009D310008A93100084934000800020100F2
:101AB400000000000000000000000000040000001E
:101AC400401F00001027000000180101054D3C4D87
:101AD4000400002008190F28040A413F00050A01E8
:101AE4000000050203FFFFFFFFFFFFFFFFFFFF0FE3
:101AF40001030002000000000000000000000000DC
:101B0400000000000000000000093D00100000007B
:101B1400040800200000FF00000000000000000096
:101B2400040800200000000000000000FF00000086
:101B34000000000004080020000000000000000075
:101B4400000000000000000000000000E0000000B1
:101B540095850008C5840008D1840008FD84000828
:101B64000000000000000000ED850008DD8400088E
:101B74005D89000800000000000000000000000073
:101B840000000000000E0F0D010908110100000003
:0C1B9400FF000000FFFFFFFFFFFFFFFF4E
:0400000508003FF5BB
:00000001FF
